:020000040800F2
:1000000000A000204510000891100008B948000821
:1000100091100008911000089110000800000000E5
:100020000000000000000000000000009110000827
:10003000911000080000000091100008FD57000812
:10004000911000089110000891100008911000080C
:1000500091100008911000089110000891100008FC
:1000600091100008911000089110000891100008EC
:100070009110000891100008FD220008911000085E
:10008000911000083D23000891100008911000080D
:1000900091100008911000089110000891100008BC
:1000A000AD2A0008B92A0008C52A0008752A0008E8
:1000B000812A0008892A0008952A00089110000862
:1000C000911000089110000891100008911000088C
:1000D00091100008F1230008FD230008911000088A
:1000E000911000089110000891100008911000086C
:1000F0009110000891100008A12A00089110000832
:100100000000000000000000000000009110000846
:10011000911000089110000891100008911000083B
:10012000911000089110000891100008911000082B
:10013000911000089110000800000000000000006D
:1001400091100008911000089110000800000000B4
:10015000000000000000000000000000000000009F
:10016000000000000000000091100008911000083D
:1001700091100008000000000000000000000000D6
:080180000000000091100008CE
:1001880010B5054C237833B9044810B10448AFF3CF
:1001980000800121217010BDD4050020000000005E
:1001A800C02A010808B5064B1BB106480649AFF33B
:1001B80000800648016811B1054A02B1904708BDA0
:1001C80000000000C02A0108D8050020D40500203E
:1001D8000000000081F0004102E000BF83F000430E
:1001E80030B54FEA41044FEA430594EA050F08BFCA
:1001F80090EA020F1FBF54EA000C55EA020C7FEA8E
:10020800645C7FEA655C00F0E2804FEA5454D4EB0A
:100218005555B8BF6D420CDD2C4480EA020281EAD4
:10022800030382EA000083EA010180EA020281EA0C
:100238000303362D88BF30BD11F0004F4FEA01315E
:100248004FF4801C4CEA113102D0404261EB41016D
:1002580013F0004F4FEA03334CEA133302D05242F3
:1002680063EB430394EA050F00F0A780A4F10104AF
:10027800D5F1200E0DDB02FA0EFC22FA05F28018E9
:1002880041F1000103FA0EF2801843FA05F35941CF
:100298000EE0A5F120050EF1200E012A03FA0EFC4E
:1002A80028BF4CF0020C43FA05F3C01851EBE37178
:1002B80001F0004507D54FF0000EDCF1000C7EEB95
:1002C80000006EEB0101B1F5801F1BD3B1F5001FD3
:1002D8000CD349085FEA30004FEA3C0C04F10104F2
:1002E8004FEA445212F5800F80F09A80BCF1004F1B
:1002F80008BF5FEA500C50F1000041EB045141EA9D
:10030800050130BD5FEA4C0C404141EB010111F49D
:10031800801FA4F10104E9D191F0000F04BF014648
:100328000020B1FA81F308BF2033A3F10B03B3F126
:1003380020020CDA0C3208DD02F1140CC2F10C02B6
:1003480001FA0CF021FA02F10CE002F11402D8BF14
:10035800C2F1200C01FA02F120FA0CFCDCBF41EAE0
:100368000C019040E41AA2BF01EB0451294330BDAF
:100378006FEA04041F3C1CDA0C340EDC04F114048C
:10038800C4F1200220FA04F001FA02F340EA030063
:1003980021FA04F345EA030130BDC4F10C04C4F1A9
:1003A800200220FA02F001FA04F340EA0300294689
:1003B80030BD21FA04F0294630BD94F0000F83F4D3
:1003C800801306BF81F480110134013D4EE77FEAB6
:1003D800645C18BF7FEA655C29D094EA050F08BF02
:1003E80090EA020F05D054EA000C04BF19461046E3
:1003F80030BD91EA030F1EBF0021002030BD5FEA27
:10040800545C05D14000494128BF41F0004130BD4E
:1004180014F580043CBF01F5801130BD01F00045A2
:1004280045F0FE4141F470014FF0000030BD7FEA15
:10043800645C1ABF194610467FEA655C1CBF0B4610
:10044800024650EA013406BF52EA033591EA030F27
:1004580041F4002130BD00BF90F0000F04BF00211F
:10046800704730B54FF4806404F132044FF0000552
:100478004FF0000150E700BF90F0000F04BF0021CB
:10048800704730B54FF4806404F1320410F0004531
:1004980048BF40424FF000013EE700BF42004FEA2C
:1004A800E2014FEA31014FEA02701FBF12F07F43A9
:1004B80093F07F4F81F06051704792F0000F14BFA6
:1004C80093F07F4F704730B54FF4607401F00045EA
:1004D80021F0004120E700BF50EA010208BF704741
:1004E80030B54FF000050AE050EA010208BF704736
:1004F80030B511F0004502D5404261EB41014FF49F
:10050800806404F132045FEA915C3FF4DCAE4FF0A2
:1005180003025FEADC0C18BF03325FEADC0C18BF89
:10052800033202EBDC02C2F1200300FA03FC20FADA
:1005380002F001FA03FE40EA0E0021FA02F1144427
:10054800C1E600BF70B54FF0FF0C4CF4E06C1CEA3C
:1005580011541DBF1CEA135594EA0C0F95EA0C0FB1
:1005680000F0DEF82C4481EA030621EA4C5123EA24
:100578004C5350EA013518BF52EA033541F4801153
:1005880043F4801338D0A0FB02CE4FF00005E1FB06
:1005980002E506F00042E0FB03E54FF00006E1FB50
:1005A80003569CF0000F18BF4EF0010EA4F1FF0493
:1005B800B6F5007F64F5407404D25FEA4E0E6D41D3
:1005C80046EB060642EAC62141EA55514FEAC520E4
:1005D80040EA5E504FEACE2EB4F1FD0C88BFBCF560
:1005E800E06F1ED8BEF1004F08BF5FEA500E50F111
:1005F800000041EB045170BD06F0004646EA0101D7
:1006080040EA020081EA0301B4EB5C04C2BFD4EB08
:100618000C0541EA045170BD41F480114FF0000E01
:10062800013C00F3AB8014F1360FDEBF002001F06F
:10063800004170BDC4F10004203C35DA0C341BDCE9
:1006480004F11404C4F1200500FA05F320FA04F0BB
:1006580001FA05F240EA020001F0004221F00041EF
:1006680010EBD37021FA04F642EB06015EEA430E62
:1006780008BF20EAD37070BDC4F10C04C4F1200592
:1006880000FA04F320FA05F001FA04F240EA020045
:1006980001F0004110EBD37041F100015EEA430E16
:1006A80008BF20EAD37070BDC4F1200500FA05F236
:1006B8004EEA020E20FA04F301FA05F243EA0203B5
:1006C80021FA04F001F0004121FA04F220EA0200C4
:1006D80000EBD3705EEA430E08BF20EAD37070BD0A
:1006E80094F0000F0FD101F00046400041EB0101EA
:1006F80011F4801F08BF013CF7D041EA060195F0CC
:10070800000F18BF704703F00046520043EB030385
:1007180013F4801F08BF013DF7D043EA0603704772
:1007280094EA0C0F0CEA135518BF95EA0C0F0CD07D
:1007380050EA410618BF52EA4306D1D181EA0301C3
:1007480001F000414FF0000070BD50EA410606BFBD
:100758001046194652EA430619D094EA0C0F02D102
:1007680050EA013613D195EA0C0F05D152EA033647
:100778001CBF104619460AD181EA030101F0004165
:1007880041F0FE4141F470014FF0000070BD41F0AE
:10079800FE4141F4780170BD70B54FF0FF0C4CF488
:1007A800E06C1CEA11541DBF1CEA135594EA0C0FA7
:1007B80095EA0C0F00F0A7F8A4EB050481EA030EF4
:1007C80052EA03354FEA013100F088804FEA0333DB
:1007D8004FF0805545EA131343EA12634FEA0222A9
:1007E80045EA111545EA10654FEA00260EF000416A
:1007F8009D4208BF964244F1FD0404F5407402D2BC
:100808005B084FEA3202B61A65EB03055B084FEA4C
:1008180032024FF480104FF4002CB6EB020E75EB49
:10082800030E22BFB61A754640EA0C005B084FEA71
:100838003202B6EB020E75EB030E22BFB61A7546EE
:1008480040EA5C005B084FEA3202B6EB020E75EB39
:10085800030E22BFB61A754640EA9C005B084FEAB1
:100868003202B6EB020E75EB030E22BFB61A7546BE
:1008780040EADC0055EA060E18D04FEA051545EAAD
:1008880016754FEA06164FEAC30343EA52734FEA56
:10089800C2025FEA1C1CC0D111F4801F0BD141EACF
:1008A80000014FF000004FF0004CB6E711F4801F34
:1008B80004BF01430020B4F1FD0C88BFBCF5E06F14
:1008C8003FF6AFAEB5EB030C04BFB6EB020C5FEA24
:1008D800500C50F1000041EB045170BD0EF0004E79
:1008E8004EEA113114EB5C04C2BFD4EB0C0541EAAB
:1008F800045170BD41F480114FF0000E013C90E6A8
:1009080045EA060E8DE60CEA135594EA0C0F08BF6B
:1009180095EA0C0F3FF43BAF94EA0C0F0AD150EA6A
:1009280001347FF434AF95EA0C0F7FF425AF1046FD
:1009380019462CE795EA0C0F06D152EA03353FF425
:10094800FDAE1046194622E750EA410618BF52EAA2
:1009580043067FF4C5AE50EA41047FF40DAF52EA76
:1009680043057FF4EBAE12E74FEA4102B2F1E043F0
:1009780024BFB3F5001CDCF1FE5C0DD901F0004C7E
:100988004FEAC0024CEA5070B2F1004F40EB8300CE
:1009980008BF20F00100704711F0804F21D113F1FA
:1009A8003872BCBF01F00040704741F480114FEA33
:1009B8005252C2F11802C2F1200C10FA0CF320FABC
:1009C80002F018BF40F001004FEAC1234FEAD323D9
:1009D80003FA0CFC40EA0C0023FA02F34FEA430343
:1009E800CCE77FEA625307D150EA01331EBF4FF0CC
:1009F800FE4040F44000704701F0004040F0FE40E7
:100A080040F40000704700BF80F0004002E000BFE3
:100A180081F0004142001FBF5FEA410392EA030FE1
:100A28007FEA226C7FEA236C6AD04FEA1262D2EB2B
:100A38001363C1BFD218414048404140B8BF5B4230
:100A4800192B88BF704710F0004F40F4000020F0C9
:100A58007F4018BF404211F0004F41F4000121F0DF
:100A68007F4118BF494292EA030F3FD0A2F1010229
:100A780041FA03FC10EB0C00C3F1200301FA03F167
:100A880000F0004302D5494260EB4000B0F5000F8A
:100A980013D3B0F1807F06D340084FEA310102F149
:100AA8000102FE2A51D2B1F1004F40EBC25008BFFB
:100AB80020F0010040EA03007047490040EB0000C5
:100AC80010F4000FA2F10102EDD1B0FA80FCACF1F4
:100AD800080CB2EB0C0200FA0CF0AABF00EBC250F3
:100AE80052421843BCBFD0401843704792F0000FE1
:100AF80081F4000106BF80F400000132013BB5E734
:100B08004FEA41037FEA226C18BF7FEA236C21D0A9
:100B180092EA030F04D092F0000F08BF084670470E
:100B280090EA010F1CBF0020704712F07F4F04D1DC
:100B3800400028BF40F00040704712F100723CBFEF
:100B480000F50000704700F0004343F0FE4040F419
:100B5800000070477FEA226216BF08467FEA2363D7
:100B68000146420206BF5FEA412390EA010F40F4C2
:100B7800800070474FF0000304E000BF10F000430E
:100B880048BF40425FEA000C08BF704743F09643F5
:100B980001464FF000001CE050EA010208BF704710
:100BA8004FF000030AE000BF50EA010208BF704797
:100BB80011F0004302D5404261EB41015FEA010CAC
:100BC80002BF84460146002043F0B64308BFA3F1A4
:100BD8008053A3F50003BCFA8CF2083AA3EBC25386
:100BE80010DB01FA02FC634400FA02FCC2F12002A5
:100BF800BCF1004F20FA02F243EB020008BF20F0DC
:100C08000100704702F1200201FA02FCC2F1200241
:100C180050EA4C0021FA02F243EB020008BF20EA36
:100C2800DC7070474FF0FF0C1CEAD0521EBF1CEA64
:100C3800D15392EA0C0F93EA0C0F6FD01A4480EA52
:100C4800010C400218BF5FEA41211ED04FF000633B
:100C580043EA501043EA5111A0FB01310CF0004067
:100C6800B1F5000F3EBF490041EAD3715B0040EA8D
:100C7800010062F17F02FD2A1DD8B3F1004F40EB5D
:100C8800C25008BF20F00100704790F0000F0CF030
:100C9800004C08BF49024CEA502040EA51207F3AF4
:100CA800C2BFD2F1FF0340EAC250704740F40000CF
:100CB8004FF00003013A5DDC12F1190FDCBF00F0C0
:100CC80000407047C2F10002410021FA02F1C2F16E
:100CD800200200FA02FC5FEA310040F1000053EA0A
:100CE8004C0308BF20EADC70704792F0000F00F058
:100CF800004C02BF400010F4000F013AF9D040EA5E
:100D08000C0093F0000F01F0004C02BF490011F4F1
:100D1800000F013BF9D041EA0C018FE70CEAD153EF
:100D280092EA0C0F18BF93EA0C0F0AD030F0004C6F
:100D380018BF31F0004CD8D180EA010000F0004023
:100D4800704790F0000F17BF90F0004F084691F0E1
:100D5800000F91F0004F14D092EA0C0F01D142021B
:100D68000FD193EA0C0F03D14B0218BF084608D1E4
:100D780080EA010000F0004040F0FE4040F400002E
:100D8800704740F0FE4040F4400070474FF0FF0CC1
:100D98001CEAD0521EBF1CEAD15392EA0C0F93EA08
:100DA8000C0F69D0A2EB030280EA010C49024FEA5A
:100DB800402037D04FF0805343EA111143EA101313
:100DC8000CF000408B4238BF5B0042F17D024FF4CB
:100DD800000C8B4224BF5B1A40EA0C00B3EB510FA6
:100DE80024BFA3EB510340EA5C00B3EB910F24BF8F
:100DF800A3EB910340EA9C00B3EBD10F24BFA3EB14
:100E0800D10340EADC001B0118BF5FEA1C1CE0D1DB
:100E1800FD2A3FF650AF8B4240EBC25008BF20F08E
:100E2800010070470CF0004C4CEA50207F32C2BFE2
:100E3800D2F1FF0340EAC250704740F400004FF07F
:100E48000003013A37E792F0000F00F0004C02BFB0
:100E5800400010F4000F013AF9D040EA0C0093F07A
:100E6800000F01F0004C02BF490011F4000F013BD4
:100E7800F9D041EA0C0195E70CEAD15392EA0C0F3C
:100E880008D142027FF47DAF93EA0C0F7FF470AF74
:100E9800084676E793EA0C0F04D14B023FF44CAFB7
:100EA80008466EE730F0004C18BF31F0004CCAD14C
:100EB80030F000427FF45CAF31F000437FF43CAF88
:100EC8005FE700BF4FF0FF3C06E000BF4FF0010CAA
:100ED80002E000BF4FF0010C4DF804CD4FEA40028C
:100EE8004FEA41037FEA226C18BF7FEA236C11D0D6
:100EF80001B052EA530C18BF90EA010F58BFB2EB89
:100F0800030088BFC81738BF6FEAE17018BF40F008
:100F1800010070477FEA226C02D15FEA402C05D1BC
:100F28007FEA236CE4D15FEA412CE1D05DF8040B41
:100F3800704700BF844608466146FFE70FB5FFF7D4
:100F4800C9FF002848BF10F1000F0FBD4DF808ED8C
:100F5800FFF7F4FF0CBF012000205DF808FB00BF7D
:100F68004DF808EDFFF7EAFF34BF012000205DF8D7
:100F780008FB00BF4DF808EDFFF7E0FF94BF012024
:100F880000205DF808FB00BF4DF808EDFFF7D2FF21
:100F980094BF012000205DF808FB00BF4DF808ED64
:100FA800FFF7C8FF34BF012000205DF808FB00BF31
:100FB8004FEA4002B2F1FE4F0FD34FF09E03B3EB5E
:100FC80012620DD94FEA002343F0004310F0004F9E
:100FD80023FA02F018BF404270474FF000007047F4
:100FE80012F1610F01D1420205D110F0004008BF93
:100FF8006FF0004070474FF00000704742000ED27B
:10100800B2F1FE4F0BD34FF09E03B3EB126209D43B
:101018004FEA002343F0004323FA02F070474FF0F1
:101028000000704712F1610F01D1420202D14FF066
:10103800FF3070474FF00000704700BF002100F0FC
:1010480004B80C4B5B58435004310B480B4B421807
:101058009A42FFF4F6AF0A4A00F003B8002342F8B8
:10106800043B084B9A42FFF4F9AF0AF01FFA03F069
:1010780019FC7047E42A010800000020D40500206C
:10108800D4050020801F0020FFF7FEBF084B9842C0
:1010980001D1084904E0084988420CBF07490849BA
:1010A8000A88501C83B20B80098888B2704700BF39
:1010B80000300140F205002000380040F40500200F
:1010C800F005002038B5054641F201041148022117
:1010D8000AF0F2FC20B9601E84B2002CF6D10EE0B2
:1010E8000C4829460AF0DFFC41F2010409480121B5
:1010F8000AF0E2FC40B9013CA4B2002CF6D1054844
:10110800FFF7C4FFC0B238BD0248BDE838400AF056
:10111800CEBC00BF003001402DE9F041012188B06C
:101128004FF480500AF0FAFB01214FF400300AF026
:10113800E9FB05210A464FF090400AF0A0F9062184
:1011480005224FF090400AF09AF9052207214FF046
:1011580090400AF094F902200026E02303258DF838
:10116800080001A94FF0904001938DF809508DF8BF
:101178000A608DF80B600AF031F901214FF4001074
:101188000AF0C0FB8DF80950394D0824394F4FF04B
:101198000108284601A901948DF808808DF80A6095
:1011A8008DF80B600AF01AF9214628460AF063F90F
:1011B80038460AF0EBFB07204FF482714FF4E062E7
:1011C8004FF40073ADF80E10ADF81C0003A93846B3
:1011D800ADF81020ADF81630ADF80C60ADF812601F
:1011E800ADF81460ADF81840ADF81A600AF000FCCC
:1011F80038464FF480510AF04BFC384641460AF015
:101208003BFC214628460AF038F92420FFF75AFF0C
:101218008020FFF757FF214628460AF02CF9642062
:1012280004F010FB214628460AF027F92020FFF792
:1012380049FFAF20FFF746FF214628460AF01BF971
:10124800404604F0FFFA214628460AF016F9232002
:10125800FFF738FF5020FFF735FF284621460AF0F0
:101268000AF9642004F0F9FA08B0BDE8F08100BF7B
:10127800001000480030014037B5082105461948DC
:101288000AF0FBF8E820FFF71DFF00240020FFF715
:1012980019FF0DF804000134062CF7D11148082174
:1012A8000AF0E9F89DF800209DF8013043EA022091
:1012B80001B2082391FBF3F29DF802009DF8031098
:1012C8002A8041EA002210B290FBF3F19DF8052034
:1012D8009DF80400698042EA002108B290FBF3F30C
:1012E800AB803EBD00100048034B0449044A03602C
:1012F8004160C26001207047211100088112000876
:101308001944923113B506220446282132206B462F
:1013180000F058FAF0B19DF801209DF8003043EA3A
:10132800022001B2022391FBF3F29DF803009DF81D
:101338000210228041EA002210B290FBF3F19DF8DE
:1013480004209DF80500618042EA002108B290FB64
:10135800F3F3A3801CBD000008B5242180223220AD
:1013680000F0B6F9642004F078FA202197223220A0
:1013780000F0AEF90A2004F070FA1022232132207E
:1013880000F0A6F9642004F068FA024B4FF480528A
:101398001A8008BD0400002013B501220446272145
:1013A80032200DF1070300F00DFA20B10248034B7B
:1013B8006060236001201CBD0D1300086113000844
:1013C800044B054903EB4000427831F8123098B2DB
:1013D800704700BFB8140020B214002030B55C4D2F
:1013E8005C4B2878062207211A7099700822811C04
:1013F800441C9BB01A7159715870DC70C31C564854
:101408002B70564C0BF044F80FA80BF0D9F82A783B
:10141800534810940024012A8CBF802121460F9044
:1014280014914FF480604FF400514FF48073ADF87D
:10143800482016902022189147480FA91792159313
:101448001194139419940BF09BF8012142480BF066
:10145800C4F868460AF005F803200F238DF8040045
:101468006946404800938DF8074009F0B7FF01210D
:101478004FF0A0400AF0A0FB0A2004F0EEF94FF06C
:10148800A04021460AF08DFB4FF0A0400AF084FBF3
:101498004FF0A0400AF08DFB04460028F8D1214601
:1014A8004FF0A0400AF088FB02A80AF065FB4FF451
:1014B80000414FF44032022304914FF0A04002A9AA
:1014C8000392059302948DF818400AF025FB07A8AB
:1014D8000AF016FB1E4A4FF40050117807908DF859
:1014E80038104FF0A04007A9089409940A940B9467
:1014F8000C940D940AF0E6FA154B1878A0420BD913
:10150800144A4FF0A04012F814100134E4B22246F5
:1015180006230AF05EFBEFE74FF0A04001210AF036
:1015280032FB4FF0A04001210AF0C9FB0028F8D097
:1015380002214FF0A0400AF0BAFB4FF0A040012171
:101548000AF0ACFB4FF0A0400AF0A3FB1BB030BD83
:10155800F6050020B814002008000240B21400204C
:101568004000005000080048024B1A88501C81B205
:1015780019807047F805002070B5494B8AB0984229
:10158800054637D14FF4802001210AF0BBF94FF40A
:10159800001001210AF0CEF901214FF480200AF051
:1015A800B1F910200AF094F93E480621042209F006
:1015B80066FF042207213B4809F061FF01A809F0F2
:1015C80050FF03A80AF030FF0224032640218DF8BB
:1015D80008408DF80960019132480126002401A9CC
:1015E8008DF80A608DF80B4009F0F8FE8022019210
:1015F8002C483CE02C4885424FD14FF480200121F3
:101608000AF080F94FF4800001210AF093F90121D2
:101618004FF484000AF076F924480AF059F924486E
:101628000621042209F02BFF0A2104224FF09040E2
:1016380009F025FF01A809F014FF03A80AF0F4FE39
:1016480002218DF80810032240231948012600249E
:1016580001A98DF809208DF80A608DF80B400193D7
:1016680009F0BCFE4FF4806001904FF0904001A952
:1016780009F0B4FE03A80AF0D7FE0E4B284603A9CA
:1016880006940494059407940894099403930AF023
:101698009BFE284631460AF0D2FE0AB070BD00BF54
:1016A800005400400004004800580040200000108A
:1016B800001400487A25E0000148FFF75DBF00BF2D
:1016C80000540040014B188880B27047F80500208C
:1016D8003A4BF7B516464FF4204205460F461A60B6
:1016E80037484FF400410AF0CAFE344C40B1236831
:1016F800581E2060002BF3D1FFF736FF00205BE077
:101708004FF40050009029462D4801224FF0807375
:101718000AF09EFE4FF420412160294802210AF078
:10172800AEFE264C28B921684A1E22600029F4D151
:10173800E2E7234839460AF09DFE4FF42042226032
:101748001F4880210AF09BFE1C4C28B92368581EAC
:101758002060002BF4D1CFE70023009318482946D6
:1017680001224FF000730AF073FE4FF4204020600E
:10177800134802210AF083FE104C28B921684A1E3A
:1017880022600029F4D1B7E731460D480AF072FE0D
:101798004FF4204121600A4820210AF070FE30B938
:1017A800064A1368581E1060002BF4D1A4E70448B9
:1017B80020210AF06AFE0120FEBD00BFFC050020C2
:1017C800005400402DE9F3411F463E4B14464FF4A8
:1017D800204280460D461A603B484FF400410AF00B
:1017E8004EFE384E034640B133685A1E3260002B15
:1017F800F2D1FFF7B9FE002061E04FF400500090ED
:101808004146314801220AF023FE4FF4204131605D
:101818002D4802210AF033FE2A4E28B93168481EA5
:1018280030600029F4D1E4E7012C88BF45F0800539
:10183800254829460AF01EFE4FF42042326022480D
:1018480040210AF01CFE30B91E480268531E03608E
:10185800002AF4D1CDE74FF4105300931A484146BB
:1018680022464FF000730AF0F3FD16484FF420416A
:101878000160CCB1144804210AF001FE30B9114AC4
:101888001368591E1160002BF4D1B2E70E480AF014
:10189800F3FD013C07F8010BE4B2E6E7094A1368D7
:1018A800581E1060002BA4D0074820210AF0E7FD3D
:1018B8000028F3D0044820210AF0E7FD0120BDE804
:1018C800FC8100BFFC05002000540040F8B5134B14
:1018D80005469B890E461446ECB116B116F8017BF5
:1018E80000E0FF270D4802210AF0E6F80028F9D0A9
:1018F8000A4839460AF0D9F8084801210AF0DCF804
:101908000028F9D005480AF0D4F8C0B20DB105F89E
:10191800010B013CE0E70120F8BD00BF00380040A2
:101928002DE9F047012188B04FF480400AF002F811
:10193800364C01214FF480400AF014F803204FF48C
:1019480020434FF0020A8DF8030069462046ADF89F
:1019580000308DF802A000F05DF84FF480410025BA
:101968002B4FADF80010204669464FF480564FF0D3
:1019780001098DF8025000F04DF869462046ADF88F
:1019880000608DF8029000F045F8384609F0FEFF37
:1019980007214FF482724FF400704FF4E063ADF802
:1019A8000E20ADF816001022ADF81C10384603A919
:1019B800ADF81030ADF81820ADF80C50ADF81A504D
:1019C800ADF812A0ADF814900AF012F8384649465E
:1019D8000AF052F89F238DF804308DF805508DF8E1
:1019E80006508DF8075001A90422268502A8FFF7A2
:1019F8006DFFA6619DF80900A846B0F1EF014A42C3
:101A080052EB010008B0BDE8F08700BF00040048B1
:101A18000038004073B506460D460024012303FA3A
:101A280004F229880A421AD0A878E978009200F0CE
:101A380003028DF804208A1ED1B299429CBF0A4B3A
:101A48005B5C800800F00C028DF8053030460023FE
:101A580069468DF806308DF8072009F0BFFC01347F
:101A6800102CDBD17CBD00BF240201082DE9F8430E
:101A7800044643796278002B14BF0220002002B18B
:101A880001303849002551F82090A8462F462E46A7
:101A980019F80620FF2A02F00F0002F0F0035FD0C9
:101AA800A17821B1A0F1080CBCF1030F55D902F0BF
:101AB8002002D2B21AB12278002A08BF002303F00C
:101AC8001002D2B21AB16278002A08BF0023E27865
:101AD8004AB162793AB909B1011F01E0A0F10801E0
:101AE800012998BF802322792AB1617919B9021F87
:101AF800032A98BF802303F01001CAB212B100F084
:101B0800C9F92AE003F02001CAB222B1F9B200F003
:101B18008BF9013721E003F04001CAB282B1228972
:101B2800114B4FEA0010B2F5FA7F1844E9B2A389C5
:101B380002D900F0DFF801E000F0F2F801350CE01E
:101B48001B060AD5084B5FFA88F103EB001062897F
:101B5800E38900F0FBF808F1010801360E2E97D151
:101B6800BDE8F88340020108A0020108064BA1F570
:101B78007A7153F82000838802684B434FF47A70D7
:101B880093FBF0F11160704704060020024B53F8F4
:101B98002000026811607047040600202DE9F04F0C
:101BA800044646488E46057889B0691C01709246FD
:101BB80011462068724601930C2600F0A7FEA26821
:101BC8004FF0020802A96E436068ADF808208DF84E
:101BD8000A808DF80B80FFF71DFF03A8384F256892
:101BE80094F80CB00AF0CEF97023019A03930120FF
:101BF80000214FF4807307EB0609ADF81000ADF82B
:101C080012100592ADF81880ADF81C30BBF10C0F1E
:101C18002BD8DFE80BF0072A2A2A102A2A2A192AA1
:101C28002A2A2200284603A90AF0DCF828460821B7
:101C38000AF0B2F919E0284603A90AF011F9284672
:101C480008210AF0AFF910E0284603A90AF03EF986
:101C5800284608210AF0ADF907E0284603A90AF04A
:101C680069F9284608210AF0AAF9A07B18B120686A
:101C780001210AF03AFA012120680AF0A6F8217B2E
:101C88000C2914D8DFE801F0071313130A131313F0
:101C98000D13131310002268343207E0226838321B
:101CA80004E022683C3201E022684032BA51A9F8C7
:101CB80004A0484609B0BDE8F08F00BF0006002028
:101CC8005406002008B5044B53F820301BB10B28EC
:101CD80001D89A68904708BD04060020044B53F8C1
:101CE80020201AB107289CBF12681160704700BFF6
:101CF8003406002010B50C460649B1FBF2F292B248
:101D08000821FFF74BFF044B044943F82400816086
:101D180010BD00BF00127A0004060020751B0008E1
:101D280010B50C460649B1FBF2F292B20121FFF759
:101D380035FF044B044943F82400816010BD00BFFF
:101D480040420F0004060020951B000810B50C4601
:101D5800054991FBF2F292B20121FFF71FFF034BF5
:101D680043F8240010BD00BF40420F003406002095
:101D78000A4A0B4813681160C91A40F68C2291422E
:101D88000360084B01DD002006E01A78072A9CBF93
:101D9800054820F81210501C18707047880700205A
:101DA800E40600209C0700208C0700207FB504462D
:101DB80001A80D4616460AF009F90020032101235F
:101DC800ADF80A00ADF80C10204601A9ADF8045092
:101DD800ADF80660ADF808300AF02DF97FBD0000B7
:101DE8000F4B142210B502FB00308278036932B918
:101DF8004160012181701868197B02220BE0446858
:101E08008160084A091B4478C16022F81410002236
:101E180082701868197BBDE81040FFF7C7BF00BF84
:101E2800E80600208C0700202DE9F34114220D4616
:101E38006A43154F4FEA0018144908EB07040126B6
:101E48008B188E54E17BA2685D701C616068022368
:101E58008DF8061001A98DF80730ADF80420FFF7BA
:101E6800D9FD58F80700217B0022FFF79FFF204685
:101E780032464FF6FF7100F069FD20462946044AB4
:101E880000F026FDBDE8FC81A0020108E80600205C
:101E9800E91D0008F7B5124E0701BC19A168114BDE
:101EA8000025E27B1D701C6160680223ADF80410F8
:101EB80001A98DF807308DF80620FFF7ABFDB8595A
:101EC800217B2A46FFF772FF204601224FF6FF7159
:101ED80000F03CFD20462946034A00F0F9FCFEBD0F
:101EE800A0020108E8060020791D0008014B33F81C
:101EF800100070478C070020036B13B15A68006C00
:101F080001E0026AC069101A18BF01207047436BCC
:101F180013B190F844007047826A406A111A4B4224
:101F280053EB01007047026B034610B5406942B19C
:101F38001A6CD9688C1A013A18BF1146005D1964E9
:101F480010BD196ADA68405C0131B1FBF2F402FB9A
:101F58001411196210BD0000F0B51D465A4B93B01C
:101F680098420F46164604D11046294600F004F957
:101F780007E05649884240F0A3801046294600F001
:101F880061F9044605F0040200206571A660A0719D
:101F980001962062E061A0626062E762029002F04E
:101FA800FF062AB14FF4005703974FF4806600E00C
:101FB80003960023049615F00106069301D10596B1
:101FC80001E00421059105F0020505F0FF071DB1A8
:101FD800059840F00802059201A9206D0AF0DAF888
:101FE80007A80AF0EDFAE36C00254FF48051802031
:101FF8000793109111950B950D950C900E9536B38E
:10200800206BD8B16369E668202208930F92ADF877
:10201800286009950AF03CFA206B07A90AF0B0FA83
:10202800206B01210AF0D9FA206D402101220AF023
:102038001EF9206B0AF0DEFA206408E0206D2449BE
:102048000AF034F9206D224901220AF018F907A88C
:102058000AF0B6FA4FF48055A16C10958026002539
:10206800079111950B950D950C960E951FB3606B06
:10207800E0B1226910230993ADF828200F950AF0E2
:1020880007FA606B07A90AF07BFA0122606B02214C
:102098000AF0B3FA606B29460AF0AAFA606B314677
:1020A80045600122206D0AF0E2F804E0206D09493C
:1020B80001220AF0E4F8206D01210AF0CBF800E0D3
:1020C8000024204613B0F0BD003801400044004011
:1020D800050105000701070007B5024651710B46C7
:1020E80081790091D16A006D9268FFF735FF0EBDC6
:1020F80013B504460A46A160817943790091006DC1
:10210800E16AFFF729FF1CBD836A8169426BC91820
:10211800D160416A994203D9CB1A5360816204E0C5
:102128000169CB1A536000228262002180F84410B2
:10213800406B01210AF051BA10B5426A8469A15472
:10214800416A02690131B1FBF2F402FB1411426BDE
:10215800416232B11368DA070AD4BDE81040FFF7CC
:10216800D3BF006D03490122BDE810400AF087B8CB
:1021780010BD00BF0701070030B52C4B0D462C4998
:102188002C4A986099612C482C491A6058614FF480
:1021980080722B4819652431DA601A610A1D85B0EE
:1021A80018639A64143801225863D96403200223FF
:1021B80000218DF80F20AA078DF80C308DF80D003E
:1021C8008DF80E100FD504AC4FF4007344F8083D99
:1021D8004FF090400921072209F051F94FF0904043
:1021E800214609F0FBF8EB070FD504AC4FF48060EB
:1021F80044F8080D0A214FF09040072209F03FF9F2
:102208004FF09040214609F0E9F801220E2101A87B
:102218008DF804108DF805208DF806208DF807201C
:1022280009F084FF014805B030BD00BF200A002036
:102238009D070020700201081D0900200038014098
:102248005800024030B5254B254A986080200D463D
:10225800D860402123481A601961234A234985B070
:10226800986100205A6119650322022301218DF823
:102278000E00A8078DF80C308DF80D208DF80F1082
:102288000CD504AC202344F8083D19480521072241
:1022980009F0F5F81648214609F0A0F8E9070CD529
:1022A80004AC402244F8082D11480621072209F001
:1022B800E6F80F48214609F091F8262001218DF80B
:1022C800040001A88DF805108DF806108DF8071088
:1022D80009F02CFF014805B030BD00BF740A00208A
:1022E80070020108C80A00209D0800200044004030
:1022F800000C004810B54FF400500C4C0AF086F959
:1023080000210B480AF069F90021606B0AF065F9B1
:10231800626AA36A9A4204D02046BDE81040FFF7DB
:10232800F3BE012084F8440010BD00BF200A00203D
:102338004400024010B54FF000700C4C0AF066F9EA
:1023480000210B480AF049F90021606B0AF045F9B1
:10235800626AA36A9A4204D02046BDE81040FFF79B
:10236800D3BE012084F8440010BD00BF740A0020C9
:102378008000024038B5026B036D0446DD69A2B9DE
:10238800AA0612D5C16A19B19A8C90B288470CE096
:102398009B8CE2694069D9B28154E069E368421CC8
:1023A800B2FBF3F103FB1120E061626BCAB92B06A3
:1023B80017D5A36A616A8B420DD0A069C15C206DF4
:1023C80009F051FFA26A2369501CB0FBF3F103FB2B
:1023D8001102A26238BD206D0249BDE8384009F0FB
:1023E8004EBF38BD070107000148FFF7C3BF00BF54
:1023F800200A00200148FFF7BDBF00BF740A002073
:1024080041717047426A806A131A594251EB0300BE
:1024180070477FB5044601A80D46164609F0D6FD5B
:1024280000200123ADF80A00ADF80C0001A92046F0
:10243800ADF80450ADF80660ADF8083009F0FBFDC2
:102448007FBD437913F001010BD0026AC3699A4238
:1024580005D09CBFC0681218D01AC0B270470020BF
:10246800704708467047437910B513F001010446D8
:102478000ED0FFF7E6FF60B1E3696269E168D05CFE
:102488004A1E934201D2013300E00023E36110BDEC
:10249800084610BD43799A070AD5436A8269D15420
:1024A800416A03694A1CB2FBF3F103FB1122426241
:1024B80070478379012B03D1D1F1010138BF002185
:1024C800D0F83401426811B183689361704701897B
:1024D8001185704707B5034699680422ADF80410C2
:1024E8000223406801A98DF806208DF80730FFF710
:1024F80091FA0EBD2DE9F74391464FF4127242430B
:1025080098463B4B0646D41808B93A4802E00128D9
:1025180004D1394820631030C4F83401374D0327FB
:10252800D55067710023D4F83471012584F83C3202
:1025380084F8393284F8385284F84662E1624FF4FC
:102548008071E1602161B96804F1340204F59C707E
:102558002362E361A3626362A4F84232A4F84432BE
:102568006261A06102227868ADF80410C4F808908E
:1025780001A984F806808DF807208DF80650FFF72A
:1025880049FA206BFFF7A6FF20462946FFF791FF7F
:10259800322003F062F91A4BD4F8347118680346F4
:1025A800B3FBF9F1B1F5803F03D3012BF8D95B08F0
:1025B800F6E7144D89B2B0FBF5F2D2B2384600F016
:1025C800C5F938463146104A00F082F9256BB8F152
:1025D800010F14BF022200222868297BFFF719FF88
:1025E80028463146094A00F073F92046BDE8FE83C3
:1025F800C0140020200301084003010888020108D4
:102608006C01002040420F0041280008C92600083C
:1026180003460A4690F84602D96A9B79FFF76ABFD3
:10262800C268036A511E8B4201D3002300E00133C4
:102638000362704710B590F83C220446AAB9836A31
:10264800416A994225D080692169C05C01338B4277
:10265800A36228BFA26242000A2342F4007084F8F1
:102668003D32A4F83E02012311E090F93D3273B1E6
:10267800B0F83E124A08A0F83E2201F00101FFF727
:1026880018FF94F83D02431E84F83D3210BD84F8CB
:102698003C3210BD90F83B3210B583B990F83A320D
:1026A80090F8392293420AD2012101FA03F1B0F8D5
:1026B800404201332143A0F84012DBB2F2E710BDDB
:1026C8002C4B10B54FF4127404FB00346079C10729
:1026D8004ED594F8381219B3236B0021186809F005
:1026E80072FB94F83C1221B1B4F84202421CA4F8DF
:1026F8004222236BA2791868197B012A0CBF022297
:102708000022FFF786FE0020012184F83B1284F89E
:10271800390284F83A02A4F8400284F8380210BD5D
:1027280094F83B222046012A04BF94F8392284F801
:102738003A22FFF7AFFF94F83B02236B50B9012010
:10274800A27984F83B021868197B012A0CBF02227F
:10275800002209E0002184F83B12A2791868197B4D
:10276800012A14BF02220022BDE81040FFF751BE23
:1027780010BD00BFC014002090F83B1200230122B6
:10278800012980F8393280F838220BD180F83B32A1
:10279800036B8279197B1868012A14BF0222002270
:1027A800FFF737BE7047427908B5D20703461BD5F5
:1027B800B0F8402202F4007189B209B9D10705D4F2
:1027C800B3F84402421CA3F8442208BDC16AC2F30C
:1027D800470211B11046884708BD4169036ACA54C7
:1027E800BDE80840FFF71CBF08BD10B590F83832A7
:1027F8000446002B1ED190F839124A1CD3B2092B7B
:1028080080F8393203D1BDE81040FFF743BF0A2BE7
:1028180010D190F83B0228B9B4F8401241F00102F7
:10282800A4F840222046FFF7BEFF2046BDE810402E
:10283800FFF7A2BF10BD0000064B10B54FF412748D
:1028480004FB00342046FFF7F5FE2046BDE81040A3
:10285800FFF7CBBFC014002030B500240E4D55F84B
:102868002450854202D00134E4B2F7E700200B4D32
:1028780035F810508D4202D0451CE8B2F7E707251D
:1028880005FB0040C0B21B2805D8054C04EB00101E
:1028980083600171027330BD800301089C03010845
:1028A800080B00200C2912D8DFE801F007111111DC
:1028B800091111110B1111110D00022104E004215D
:1028C80002E0082100E01021012209F017BC70473E
:1028D80038B504460D461346217B00682A46FFF7A3
:1028E800BBFF2068217BBDE83840FFF7DBBF07B599
:1028F8008DF80400012000238DF806008DF80700EC
:1029080001A88DF8053009F011FC0EBD7FB504460D
:1029180001A80D46164609F04DFA0A4B0A485E43CF
:1029280001680023B1FBF6F2013D561E204601A9BD
:102938000295ADF80460ADF80C30ADF8063009F03A
:10294800F3F97FBD40420F006C01002010B504462A
:102958000068FFF7DBFF2068012109F036FA607B89
:10296800BDE81040FFF7C3BF00230C4A52F82320EC
:10297800824202D00133DBB2F7E70022084830F880
:102988001200884202D00132D2B2F7E7072101FBD8
:1029980002330448DAB200EB0210704780030108E2
:1029A8009C030108080B002070B5044600262E4B36
:1029B8009D5D95B90221204609F0A9FB01284FD158
:1029C8002046022109F0ADFB29462046FFF7CCFF3F
:1029D8000546204609F002FB3DE0042D12D12046B1
:1029E800294609F094FB01283AD12046294609F0E6
:1029F80098FB29462046FFF7B7FF0546204609F011
:102A0800EFFA28E0082D12D12046294609F07FFB6D
:102A1800012825D12046294609F083FB294620466E
:102A2800FFF7A2FF0546204609F0DCFA13E00C2D5B
:102A380016D11021204609F06AFB012810D1204642
:102A4800102109F06EFB29462046FFF78DFF054649
:102A5800204609F0C9FAAA6801460AB1287B9047BE
:102A68000236082EA3D170BD9C0301080148FFF768
:102A78009BBF00BF002C01404FF08040FFF794BF80
:102A88000148FFF791BF00BF000400400148FFF76D
:102A98008BBF00BF000800400148FFF785BF00BF9B
:102AA800003401400148FFF77FBF00BF00400140EC
:102AB8000148FFF779BF00BF004401400148FFF714
:102AC80073BF00BF00480140024800214FF4E07284
:102AD8000BF0FCBD080B00202E4B2DE9F3410546F9
:102AE8001878002838D0002426462746A0463221E8
:102AF800082253206B46FEF765FE9DF801109DF8ED
:102B08000000013400EB01239DF803109DF802003A
:102B18001AB200EB01239DF805109DF80400E4B2F9
:102B280090441AB200EB01239DF80710BF18202C1F
:102B38001AB2164401F07F0001D00028D7D1164BF5
:102B480098FBF4F897FBF4F796FBF4F6A5F80080E9
:102B58006F80AE801C701AE0322106226B4653202B
:102B6800FEF730FE9DF801209DF800109DF8030047
:102B780001EB02239DF802202B8002EB00219DF837
:102B880004309DF80500698003EB0022AA80BDE8A7
:102B9800FC8100BFC80C0020C90C002008B5134BED
:102BA80053201B782D2108227BB1FEF791FD31219E
:102BB8000A225320FEF78CFD2C210C225320FEF70D
:102BC80087FD53203821902209E0FEF781FD31214D
:102BD8000A225320FEF77CFD53202C210A22FEF7FF
:102BE80077FD034840F20912028008BDC80C002096
:102BF8000400002037B5104B05461A680F480C46EC
:102C0800002182428DF8071001D1002013E05320E3
:102C180001220DF10703FEF7D5FD0028F5D09DF838
:102C28000710E529F1D12A780548064B06492060A6
:102C38001A70616001203EBD68010020001BB700CA
:102C4800A52B0008C80C0020E12A000813B50622AD
:102C5800044602216B461820FEF7B4FD9DF80030AB
:102C68009DF8012098089DF8023000EB02219DF89C
:102C7800032098089DF80430218000EB02219DF87C
:102C880005209808618000EB0221A1801CBD00008E
:102C980008B50F2108221820FEF71AFD0E22182069
:102CA8001021FEF715FD024B4FF480521A8008BD23
:102CB8000400002037B5002402AB054603F8014D97
:102CC800182021460122FEF77DFD50B19DF80730FE
:102CD800FB2B05D10348044928606960012000E006
:102CE80020463EBD992C0008552C000813B5062235
:102CF800044601216B461C20FEF764FD9DF8002068
:102D08009DF8013043EA022040F38D01042391FB32
:102D1800F3F29DF802009DF80310228041EA002298
:102D280042F38D0090FBF3F19DF805209DF8040017
:102D3800618042EA002141F38D0090FBF3F3A38008
:102D48001CBD000037B52023022500244FF0904019
:102D580001A9ADF804308DF807508DF80640FEF74C
:102D680059FE2A2122461C20FEF7B2FC0E212A46D3
:102D78001C20FEF7ADFC0F2103221C20FEF7A8FC47
:102D88002B2112221C20FEF7A3FC2C212A461C20F2
:102D9800FEF79EFC2D2101221C20FEF799FC2E2116
:102DA80022461C20FEF794FC05221C202A21FEF74F
:102DB8008FFC02484FF4807202803EBD0400002060
:102DC80013B5044610481149026800238A428DF859
:102DD800073001D1002015E01C200D2101220DF142
:102DE8000703FEF7EFFC0028F4D09DF807302A2BE4
:102DF80001D01A2BEED10648064A074920606260C6
:102E08000B7001201CBD00BF68010020001BB7002B
:102E18004D2D0008F52C0008CA0C002013B502221D
:102E280004461B2101AB6820FEF7CCFC9DF804206A
:102E38009DF8053043EA022000F54E5110314FF459
:102E48008C7291FBF2F3233323801CBD13B5062249
:102E580004461D216B466820FEF7B4FC9DF800204F
:102E68009DF8013043EA022001B2042391FBF3F2FA
:102E78009DF802009DF80310228041EA002210B25A
:102E880090FBF3F19DF805209DF80400618042EA6B
:102E9800002108B290FBF3F3A3801CBD08B51920EC
:102EA80002F0DBFC682015210022FEF711FC10B9A6
:102EB800032002F0D3FD0C4B16211A78682042F04B
:102EC8001802FEF705FC172100226820FEF700FC17
:102ED8003D2101226820FEF7FBFB68203E210122EC
:102EE800BDE80840FEF7F4BB0000002038B50546F1
:102EF80019200C4602F0B1FC682015210022FEF7CB
:102F0800E7FB18B3124B13481349144A622C2B6081
:102F18006860A960EA60124B0FD004D80A2C12D05E
:102F2800142C0CD10DE0BC2C04D0B4F5807F06D154
:102F3800002009E00120187038BD022004E00320B9
:102F480002E0042000E005201870012038BD00BF11
:102F5800A52E0008552E0008252E00081844923189
:102F680000000020064B187820B1012806D14FF444
:102F7800805201E04FF4006202490A80704700BFA6
:102F8800CB0C00200400002007B5232002F065FCCC
:102F98006820752101220DF10703FEF713FC30B1FB
:102FA8009DF80700B0F16803594251EB03000EBDCC
:102FB80013B50622044643216B466820FEF702FC3F
:102FC8009DF800209DF8013043EA022001B2042355
:102FD80091FBF3F29DF802009DF80310228041EA6C
:102FE800002210B290FBF3F19DF805209DF8040033
:102FF800618042EA002108B290FBF3F3A3801CBD74
:1030080013B5062204463B216B466820FEF7DAFB1F
:103018009DF800209DF801309DF8021043EA022037
:103028009DF80320208042EA01239DF804009DF8C2
:103038000510638041EA0022A2801CBD07B5204A22
:1030480002204FF40053ADF804308DF807001368E0
:103058001C48002183428DF8061001D11A4803E06C
:103068001A498B4203D11A4801A9FEF7D3FC6B21F8
:1030780080226820FEF72CFB052002F0EEFB1921C8
:1030880000226820FEF724FB6B2103226820FEF74C
:103098001FFB372102226820FEF71AFB0D4A1A216E
:1030A80068201278FEF714FB1B2118226820FEF70F
:1030B8000FFB68201C211022FEF70AFB0EBD00BF83
:1030C8006801002000127A0000040048001BB700C5
:1030D800000800480100002030B585B00446FFF71D
:1030E80053FF002841D006210A46682002ABFEF7AC
:1030F80069FB9DF80B309DF80D5003F0010105F0B8
:1031080001004A0042EA80059DF8090000F0010329
:103118001D4307D0012D164801D1002318E0022DC8
:103128000CD114E00C21682001220DF10703FEF7F1
:1031380049FB9DF8071011F00F0203D1052002F09A
:103148008DFC06E0042A0A4801D1057001E001233C
:103158000370074807490378074A2160002B14BF0A
:103168006E216F2162602172012005B030BD00BF61
:10317800CB0C00206D2F00080930000838B5054633
:103188000C46FFF701FF28B3134B14481449142CBD
:103198002B606860E960134B15D004D8052C16D055
:1031A8000A2C0ED111E0BC2C08D0B4F5807F03D0D6
:1031B800622C06D102220BE0002209E001201870DF
:1031C80038BD032204E0042202E0052200E00622C2
:1031D8001A70012038BD00BF45300008B92F00081B
:1031E800194492310100002013B506220446A82193
:1031F8006B466820FEF7E6FA9DF800209DF801303E
:1032080043EA022001B2042391FBF3F29DF8020085
:103218009DF80310228041EA002210B290FBF3F1DE
:103228009DF805209DF80400618042EA002108B25B
:1032380090FBF3F3A3801CBD08B5642002F00DFBDE
:1032480068202321F022FEF743FA10B9032002F088
:1032580005FC052002F001FB044B68201A782021A8
:1032680042F00F02BDE80840FEF732BACC0C00204D
:1032780037B5054619200C4602F0EFFA68200F21F1
:1032880001220DF10703FEF79DFA9DF80730D32BB5
:1032980016D10C480C490D4A4E2C28606960EA602A
:1032A8000B4B07D05D2C09D0362C01D0002002E052
:1032B800402000E080201870012002E0C020FAE7DA
:1032C80000203EBD41320008F1310008DDE9A73198
:1032D800CC0C002010B5FDF751FC0A49FDF7A2FC03
:1032E8000949FDF753FD094B044618680078FDF7B6
:1032F80045FC01462046FDF795FCFDF77FFE80B2B0
:1033080010BD00BF3333534000F07F45E00C002070
:1033180038B50D4C00202578FEF752F80B4A05F019
:10332800070322F813000135002325701846D15AE7
:1033380002334018102B80B2F9D1C008FFF7CAFF3A
:10334800034A107038BD00BFCD0C0020CE0C002001
:1033580050190020074B084A19781088884207D36B
:10336800064B1A68907888428CBF0020012070476D
:10337800002070475019002052190020E00C00204E
:1033880038B5114B2024186000250020FEF718F8E6
:103398002D180A2002F061FA013CF6D1C5F34F104E
:1033A800FFF798FF084901230A6851786418A0427A
:1033B80002D30133062BF9D10448927803705343A2
:1033C80003490B8038BD00BFE00C0020020000203C
:1033D800521900202DE9F04F0446008885B048B9FD
:1033E800B4F9023043B9B4F90420D2F1010138BF6D
:1033F800002102E0002100E0014611F0010377D12D
:103408003D4D00B22B7000F0B7FD0646B4F902003E
:1034180000F0B2FD0546B4F9040000F0ADFD044625
:10342800304609F0FDF80746304609F06DF9804648
:10343800284609F0F5F80646284609F065F90546D4
:10344800204609F0EDF88246204609F05DF9394634
:1034580081465046FDF7E6FB394683464846FDF768
:10346800E1FB514601904046FDF7DCFB49460290DE
:103478004046FDF7D7FB314603905046FDF7D2FB97
:103488001E4C4946206006F10040FDF7CBFB29465B
:103498006060A5600298FDF7C5FB01460198FDF73D
:1034A800B9FA2946E0600398FDF7BCFB0146584687
:1034B800FDF7AEFA3146206108F10040FDF7B2FB96
:1034C800294660615846FDF7ADFB01460398FDF7B4
:1034D8009FFA2946A0610198FDF7A4FB01460298CE
:1034E800FDF798FA3946E0613046FDF79BFB20620C
:1034F80005B0BDE8F08F00BF03000020E40C0020F9
:103508002DE9F8434D4B0C460168013A1960808853
:103518009880072A30D8DFE802F004080F14191E33
:103528002226188820805A8803E0598821801A8822
:10353800524262809A881EE01988484220805A8840
:10354800F6E75988484220801A88F2E719884842E5
:10355800208058880CE05A882280188808E019884A
:1035680021805A8803E05988484220801A885042AE
:1035780060809B885A42A280314B1A78002A5AD11F
:10358800B4F90000FDF7FAFA8046B4F90200FDF735
:10359800F5FA0746B4F90400FDF7F0FA294D064696
:1035A80029684046FDF73EFBE96881463846FDF745
:1035B80039FB01464846FDF72DFAA9698146304690
:1035C800FDF730FB01464846FDF724FA09F05CF8A0
:1035D800696820804046FDF725FB29698146384601
:1035E800FDF720FB01464846FDF714FAE9698146D4
:1035F8003046FDF717FB01464846FDF70BFA09F080
:1036080043F8A96860804046FDF70CFB696980466D
:103618003846FDF707FB01464046FDF7FBF9296AE6
:1036280007463046FDF7FEFA01463846FDF7F2F93F
:1036380009F02AF8A080BDE8F88300BF080D002033
:1036480003000020E40C002070B5144D06462B78CA
:10365800134CABB102F0F0F82268B31898421CD3AF
:103668000020287002F0B4F802F0E6F820600D4857
:10367800017809B14A1E02700B4B0120187070BD09
:1036880002F0DAF821683231884206D30120287026
:1036980002F09EF802F0D0F8206070BD0F0D0020F7
:1036A8001C0D0020110D0020100D002037B58DF8DD
:1036B800051022498DF807300B788DF8040002A810
:1036C8008DF80620C21812F8044C0D46443CE0B2AE
:1036D8000A282CD81A49022B31F8104003D814B103
:1036E8002046FFF7B1FF2B78022B0BD9154D2D681B
:1036F80002F0A2F8021B954204D21049124B002096
:1037080008701870114802780146012A00D094B94F
:103718000A4B1878022801D8421C1A700020087039
:103728000B49087003B0BDE8304002F051B83224AC
:10373800022BD5D9D7E703B030BD00BF120D00204A
:10374800A40301081C0D0020110D0020100D0020FD
:103758000F0D0020014B1860704700BF140D0020AA
:1037680070B53F4B04465A7B3E4802B101220270B5
:103778004FF4007000F070F9002828D03A4E3B4B07
:10378800316858780D68003018BF01206A68904782
:1037980048B13368364D18680121C26829709047CE
:1037A80008B102212970304D2B681868826890474B
:1037B80028B12E494B7813B92D4A02201070296878
:1037C8000B689869804710B1294900220A702020A7
:1037D80004F04EFE60B12248264B827A0AB9C17ABB
:1037E80021B12248C27A0AB9012100E000211970EA
:1037F8001F4B1878022802D14C204E211DE00128C9
:1038080007D14D2153204C220B46BDE87040FFF7ED
:103818004DBF184A1178012903D1532001464E2281
:1038280006E0104B1878012804D1532001460246BF
:103838004D23EAE724B153204D210A464423E4E707
:103848000D4A117821B13220BDE87040FFF7FCBE67
:103858000A4B20461C70BDE8704001F0B9BF00BF9C
:10386800141F00200E0D0020140D0020031F00203F
:10387800180D0020190D0020110D00200F0D00203B
:10388800014B1870704700BF110D00200E4B1A78BD
:10389800422A16D15888B0F56C7F12D11979BE2901
:1038A8000FD193F8AD230020EF2A0CD113F8011B98
:1038B800064A48409342F9D1D0F1010038BF0020B0
:1038C800704700207047704700F80308B0FB0308F2
:1038D800C82314211E22038001238170C270037142
:1038E80064214FF496722823C18002814381704776
:1038F80010B50446272005F00BFE2070102005F0B7
:1039080007FE6070002005F003FEA070002005F09F
:10391800FFFD4FF4E133E07052206360A360E36081
:10392800207510BD7FB51B4D1B4C284604F0D6FDF5
:103938002146284604F0ECFD1F3D04F1240001F067
:10394800ABFD2E4604F1680005F07AF916F8C20BB3
:1039580002F096FA304603F0CBFC681C03F086FDB3
:1039680005F1B80000F00CFE04F1280001F08EFD0E
:1039780004F1490304F1380005F1C00100930190F6
:10398800029105F17800A11D224605F1BE0302F05F
:1039980009FF7FBD271D0020241A002008B5054B0C
:1039A800D02202FB0030044900F59E700AF0E0FDC9
:1039B80008BD00BF54190020081D0020224A38B550
:1039C800422313704FF46C700023BE21EF24508003
:1039D800117182F8AD4382F8AE331D461A4A985CDD
:1039E8000133B3F56C7F85EA0005F7D182F8AE5351
:1039F80008F062FC04250024691E11F0FF0516D0AA
:103A0800342008F06FFC114808F0C0FC0F4C042863
:103A18000BD10F4A2046A15808F090FC0D4B0434F6
:103A28009C42F4D10428044601D00446E4E708F097
:103A380051FC042C02D1FFF729FF20B90A20BDE868
:103A4800384002F00BB838BD5419002000F80308BC
:103A58005421FC17B0FB0308034B996808420CBFBC
:103A680000200120704700BF54190020024B9A68BB
:103A780010439860704700BF541900202DE9F04F9B
:103A8800A84AA94D85B010685168A84C02AB03C379
:103A98004FF46C72002128460AF018FED02200214B
:103AA80020460AF013FE4220032128700220697183
:103AB800FFF7DCFF2A232021A5F8EE304FF4FA7037
:103AC8002B2385F8F41040F24C41FA22A5F8F600B1
:103AD80085F80531212001F54873A5F8F22085F80D
:103AE80006016E2240F27E40A5F816314FF47A7333
:103AF80000274FF001094FF4167685F80421A5F840
:103B0800141140F2DC5200F52F71A5F8D00003F52E
:103B1800CB70A5F81221A5F8F060A5F8D21085F8A9
:103B2800AC73A5F8FA70A5F8F870A5F8FC7085F8DC
:103B3800E27085F8E37085F8E470A5F8E670A5F8FA
:103B4800E870A5F8EA7085F8ED7085F8EC9085F8CE
:103B5800077185F8387185F83A7185F8397185F8F3
:103B6800107185F8187185F8197185F81A91A5F8FA
:103B7800D430A5F8D6006C30A5F8D8004FF4C8703A
:103B8800322340F2B451A5F8DE0005F590709B464B
:103B9800A5F8DA10A5F8DC30A5F8E030019285F830
:103BA8001C7185F81D71FFF7A3FE1E2117235520F0
:103BB80040F6AC52E17263752173A3750B2114238F
:103BC800AA81E0702D2208206171A3710E2163740F
:103BD80050234FF0280862732074A2766420E171A4
:103BE800E3765A2178234FF00A0A22754122A372FC
:103BF80021722077E177AF7385F81B71277084F8FD
:103C0800018084F80280E77584F804B0A7732776EA
:103C1800E773677684F812A084F8098084F81E9008
:103C280084F8202084F8237084F8247084F82570A0
:103C3800019904F12A00E18484F821B084F8227003
:103C480002F00AF904203A4A84F82E0039493A4821
:103C5800152384F83430A263E163206405F5847188
:103C68003648278584F82F8084F8308084F844907B
:103C780004F08EFD4FF44873C8224FF4966140F269
:103C8800D9303E4684F8707084F8717084F8728078
:103C980084F8739084F87670A4F8743084F8B8A027
:103CA80084F8B920A4F8BA10A4F8BC004FF47F73C4
:103CB8004FF4FA62A4F8783007F108006B46A2F5D1
:103CC800FA71A4F87A20C25CA4F87C100137FF21AD
:103CD80084F87E2084F87F100834082FE6D1134832
:103CE800012480F8BE4080F8BF4080F8C040C23050
:103CF800FFF7EEFD00200C4B0021C2181030C02841
:103D08001161F8D100240E48D02220180749D03478
:103D18000AF02EFCB4F51C7FF5D105B0BDE8F04FD4
:103D2800FFF74CBE0402010854190020081D0020AA
:103D38009A99193FF6287C3F3D0A773FBA03010854
:103D4800901A002008B5FFF7A1FD18B9BDE8084092
:103D5800FFF794BE08BD0000024B9A6822EA0000F3
:103D68009860704754190020314B10B59A681404B4
:103D780009D4D00707D4110705D4D20303D44FF4CC
:103D88000040FFF773FE2A488168044611F4803F1B
:103D980012D00B0702D50820FFF7DEFFA36818042E
:103DA80003D54FF40040FFF7D7FF214A9068C107B9
:103DB80002D50120FFF7D0FF1D498B680C4613F090
:103DC800080F0BD01A0403D54FF40040FFF7C4FFC7
:103DD800A268D30702D50120FFF7BEFF144848F2B6
:103DE8000103816848F201040B40A342044603D151
:103DF8004FF40040FFF7B0FFA26848F240001040BF
:103E080048F24001884202D14020FFF7A5FF094847
:103E180004F0BEFB084805F06DFC074805F006FCF9
:103E280020B90548BDE81040FFF762BD10BD00BFCE
:103E3800541900205C1A0020741A002010B5FFF7EE
:103E480025FD10B90A2001F009FE0F4C0F49204644
:103E58004FF46C720AF08CFB94F8AC33022B02D945
:103E6800002084F8AC0394F8AC13D02202FB014381
:103E7800074803F59E710AF07BFBFFF775FFBDE865
:103E88001040FFF74FBD00BF5419002000F8030889
:103E9800081D002008B5FFF7D1FF0F2014210122CB
:103EA800BDE8084007F072BA08B5054B93F8AC03B3
:103EB800FFF774FDFFF782FDBDE80840FFF7EABF92
:103EC80054190020014B9868704700BF541900200E
:103ED800884203DB8242B4BF114601460846704758
:103EE8000023036170472DE9F04106690446013655
:103EF800012E0D46066105D10023616021608360B3
:103F0800BDE8F081D0F8008008464146FCF780FD06
:103F180007463046FCF732FE01463846FCF736FFC6
:103F280001464046FCF776FD064660603146284665
:103F3800FCF76EFD01463846FCF774FEA168FCF7F5
:103F480069FD2660E060A060BDE8F08110B5044618
:103F58000069012807DD0138FCF710FE0146E0681A
:103F6800FCF714FF10BD002010BD08B5FFF7EEFFE9
:103F7800BDE8084008F056BC08B5FCF77DFA04A374
:103F8800D3E90023FCF7DEFAFCF7EEFC08BD00BF1E
:103F9800399D52A246DF913F2DE9F041069C064625
:103FA8000F46002B0CBF4FF020084FF0300820467A
:103FB80010F8013B0BB9154603E0002AFBDD013A76
:103FC800F6E7002D04DD30464146B847013DF8E7E5
:103FD80014F8011B11B13046B847F9E7BDE8F08184
:103FE800014B186801F0C0BB280D00202DE9F043F3
:103FF80089B006460F4603921C46039A134613F8E7
:10400800011B0393002900F08A80252901D030463E
:1040180083E0002004905578911C302D039105D140
:104028009578033203924FF0010800E08046A5F12D
:104038003003D8B2092806D8284603A90A2204ABB7
:1040480000F02AF905466C2D05D10399012211F8D3
:10405800015B039100E00022642D2FD010D8582D69
:104068003AD006D8002D5AD0252DC6D1304629463B
:1040780053E0632DC1D130462178251DB8474AE069
:10408800752D0DD0782D27D0732DB6D1251D246818
:10409800304600943946049A0023FFF77DFF3AE042
:1040A800251D20680A2122B1002205AB00F07EF808
:1040B80002E005AB00F0AAF82C4623E005AD04F1B8
:1040C80004092068294612B100F095F801E000F0D3
:1040D800C2F84C46009517E004F104092068102145
:1040E80042B1B5F15804634253EB040205AB00F04A
:1040F8005DF806E0B5F158035A425A4105AB00F0A5
:1041080085F84C4605A8009030463946049A43463F
:10411800FFF742FF71E72C466FE7B8476DE709B034
:10412800BDE8F0830FB407B5094904AB086809492D
:1041380053F8042B09680193FFF758FF064B1868DA
:1041480001F031FB0028F9D0BDE80E4004B07047FB
:10415800240D0020200D0020280D0020034A044BC8
:10416800044900201A600860704700BFE93F000852
:10417800200D0020240D0020014B1860704700BF5F
:10418800280D002070B50646B6FBF2F40846154621
:1041980014B12046FFF7F6FF05FB1464024B195DC6
:1041A80000F8011B70BD00BFC3030108F0B501246E
:1041B800B0FBF4F58D4201D34C43F9E70026C4B1B6
:1041C800B0FBF4F504FB1500B4FBF1F41EB9002DA7
:1041D80001DC002CF4D1092DEFB204DD002A0CBF5C
:1041E8005725372500E03025ED1903F8015B013626
:1041F800E5E71C70F0BD00280B4603DA2D2240428B
:1042080003F8012B0A210022FFF7D0BFF0B50124E3
:10421800B0FBF4F58D4201D34C43F9E70026C4B155
:10422800B0FBF4F504FB1500B4FBF1F41EB9002D46
:1042380001DC002CF4D1092DEFB204DD002A0CBFFB
:104248005725372500E03025ED1903F8015B0136C5
:10425800E5E71C70F0BD00280B4603DA2D2240422A
:1042680003F8012B0A210022FFF7D0BFA0F1300389
:10427800DAB2092A01D818467047A0F16101052968
:1042880001D857387047A0F14103052B01D83738BA
:1042980070474FF0FF3070472DE9F8430D6804462A
:1042A8000F469046994600262046FFF7DFFF002874
:1042B80006DB404504DC08FB060615F8014BF3E76E
:1042C8003D602046C9F80060BDE8F883931E222BA4
:1042D80088BF0A22031E10B50C4603DA2D2001F808
:1042E800010B5842FFF74EFF00210170204610BD18
:1042F80030B587B005460C4603A800210C220AF009
:10430800E5F928460021FCF749FE20B1284629494D
:10431800FCF780FB03E028462649FCF779FB264991
:10432800FCF780FCFCF744FE054685EAE570A0EB47
:10433800E5700A226946FFF7C9FF002D01DB20233B
:1043480000E02D2368468DF80C300BF0F3F80128B7
:1043580007D130228DF80D208DF80E208DF80F2012
:104368000CE0022805D130218DF80D108DF80E10C3
:1043780004E0032802D130208DF80D00694603A817
:104388000AF0D6FF03A80BF0D5F8C51EEDB22A46F1
:1043980003A920460BF06CF9002363552046074912
:1043A8000AF0C6FF03A9204649190AF0C1FF2046B2
:1043B80007B030BD6F12033A00007A44340E01088A
:1043C8002DE9F041027803460130202AFAD0092A63
:1043D800F8D02D2A02D10346414D04E02B2A08BF0C
:1043E80003464FF07E551E460024334616F8010B4F
:1043F800A0F13007F9B209290DD83A492046FCF74F
:1044080011FC04463846FCF7B9FB01462046FCF788
:1044180001FB0446E9E72E2817D1324F334616F838
:10442800010B3038C2B2092A0FD8FCF7A7FB39466E
:10443800FCF7ACFC01462046FCF7ECFA2949044697
:104448003846FCF7EFFB0746E8E71878652801D0FF
:10445800452839D15E782D2E02D19F1C012605E012
:104468002B2E01D05F1C00E09F1C00267B1E00271E
:1044780013F8012F303AD1B2092903D80A2000FBDA
:104488000727F5E7B7F59A7F28BF4FF49A77B8461C
:104498004FF07E51B8F1070F07D908461249FCF7CB
:1044A800C1FBA8F108080146F4E707F0070737B190
:1044B80008460C49FCF7B6FB013F0146F7E72EB169
:1044C8002046FCF763FC04E04FF07E512046FCF7E1
:1044D800A9FB01462846FCF7A5FBBDE8F08100BF13
:1044E800000080BF0000204120BCBE4C014B0022D0
:1044F8009A807047300D0020034BB3F90400D0F1C7
:10450800010038BF00207047300D00200649074BD6
:104518000A68B3F90400137805214B439842D4BFC5
:1045280000200120704700BF380D0020300D00200A
:1045380010B50446FFF7EAFF002814BF2046002004
:1045480000F0010010BD0000074B084A1968B2F9D5
:1045580004004B780A78D118052251438842D4BF09
:1045680000200120704700BF380D0020300D0020CA
:10457800024B9A88501C9880704700BF300D00206D
:10458800024B00221860024882807047380D0020D4
:10459800300D0020034B04491860044800220160D4
:1045A800C28070473C0D0020E8030108300D002050
:1045B80008B501F049FC024B00221A7008BD00BF83
:1045C800031F002010B5FFF7A1FF00281ED0104BD5
:1045D8005C78201C18BF0120FFF7AAFF70B10D48B6
:1045E8000D4B01680D484A8901681A805A809A80E3
:1045F8004A88DA800A4BD888411CD980FFF7A4FF83
:1046080000B91CB9BDE81040FFF7D2BF10BD00BF0C
:10461800031F00203C0D00205A1F0020380D0020E9
:10462800300D0020044B9A8811B2142901DD143A88
:1046380000E000229A807047300D002003280B4BC1
:104648000AD80B4A126892888A4205D2012101FAD7
:1046580000F01A78104318701B780F2B04D1034808
:1046680000210170FFF7DEBF704700BF2C0D00204E
:10467800380D002030B5814C89B0FFF76FFDFFF78A
:1046880061FBFFF7DBFBA07B003018BF012001F0C6
:10469800EFF894F8073133B1012B01D0092B02D17F
:1046A8008DF80C3004E000218DF80C1084F8071107
:1046B80003A8FCF793FE0220FFF7CEF910B170486B
:1046C800FEF75EFE6F48FEF785FE022003F0DAFE75
:1046D8006D4D6A4AB5F9283002F1E200B2F8EE10E1
:1046E80092F8ED2000F0AEFF10B9032001F0B6F902
:1046F800664C4FF488404FF48853A0610A252385FF
:10470800624C013DA18A8AB282F48840A082A38AC1
:10471800192099B281F48852A28201F09EF80120F2
:1047280001F056F8192001F098F8002001F050F82F
:1047380015F0FF05E4D14FF488434FF488502085E5
:1047480023854E4C01F028FC04F11001607902F039
:1047580089F8FEF7B9F904F5907005F041F8617928
:104768000E2901D0082903D101228DF8152001E076
:104778008DF815504020FFF76FF98DF812004FF4AF
:104788000040FFF769F98DF810000120FFF764F980
:104798008DF8110002F08CFC8DF813003A4890F85F
:1047A800C0304FF47A70C3F380048DF81440334C52
:1047B800ADF81C00B4F8DE10B4F8E0204FF48040E7
:1047C800ADF81810ADF81A20FFF746F918B1B4F88B
:1047D800DA30ADF81C30BDF81810B1F5FA7F02D9FF
:1047E8000022ADF81C20B4F8120194F80741ADF886
:1047F8001E00012C04D0092C01D1072400E000245C
:1048080004A88DF81640FDF731F92148FFF7C2FEDC
:10481800204C2060FEF79EFF1D48216803F0F2FE41
:104828004FF48070FFF718F958B114481A4B90F8F4
:104838001D1190F81C21009300F59070C13302F00F
:1048480065FE4FF40060FFF707F908B104F07CFA41
:1048580000F0D8FF0949114B4A791860052A03D19D
:104868004FF4C87000F000FD4FF47A7000F01AFEA3
:104878000B4B0120587309B030BD00BF54190020FC
:10488800581A00203A1A0020081D0020001000487D
:104898005C1A0020DC1D0020091D0020480D0020A6
:1048A800031F002008B5FFF7E5FE00F0E5F9FCE777
:1048B80008B5034BB3F9D40002F0EAF8FEE700BFED
:1048C8005419002008B500F0F3FD0B4B50B19A784D
:1048D80042B1597879B901225A70084B08491888A9
:1048E800088008BD587830B90220FF210122BDE8B0
:1048F800084006F04BBD08BD031F0020261E0020FF
:10490800EC1D00202DE9F04FB64BB74AB3F906006D
:10491800D18C85B088420FDBB0F5FA6F92F825404C
:1049280007DA451A6C43A1F5FA6694FBF6F4643489
:1049380003E0C4F1640400E06424AC4AAA4BB2F872
:10494800127192F9EC2093F823100097574293F8CC
:104958007050019193F87160B9B293F824300291C4
:10496800002103930A469F4FDDF8008031F907C004
:1049780040F2E637C8EB0C0303F2F31EBE4503D83A
:10498800002BB8BF5B4201E04FF4FA73022ADFF84C
:1049980068822CD025B1AB42CCBFC5EB0303002302
:1049A8006427DFF87CA293FBF7FE6FF0630B3AF8FD
:1049B8001E900BFB0E3B0EF1010E3AF91EA00FFAEA
:1049C80089FECEEB0A0E0EFB0BFE9EFBF7FEF144B2
:1049D80028F80190DDF8048003FB08FE844B9EFB59
:1049E800F3F3DB199BB2634393FBF7F712E026B1AD
:1049F800B342CCBFC6EB03030023029F5F43A8F872
:104A08000470039F002BB8BF5B427B43784F93FB36
:104A1800F7F76437744B02EB030E9EF8019064239A
:104A280007FB09F898FBF3F9DFF8F88102F808901A
:104A38009EF80B909EF815E007FB09F807FB0EF7A8
:104A480098FBF3F9DFF8E08197FBF3F302F808909D
:104A5800DDF80080674FC445D35503DA664BCF5A5B
:104A68007F42CF5201320231032A7FF47CAF5F4C80
:104A78004FF4FA62B4F81411FFF72AFAB4F8146183
:104A88004FF47A75801B4543C6F5FA63B5FBF3F519
:104A980064215A4895FBF1F36FF0630630F8132050
:104AA80006FB0355013330F9130013B2C01A45430E
:104AB800534B514C95FBF1F1587A8A18E280002843
:104AC80038D0504F504D3E882988721A10B2FFF7DF
:104AD80053FA074607F0A4FD0646384607F014FEC9
:104AE8000546B4F90200FCF749F80746B4F9000096
:104AF800FCF744F831468046FCF794F8294681468D
:104B08003846FCF78FF801464846FBF781FFFCF76B
:104B18004FFA314620803846FCF784F82946064685
:104B28004046FCF77FF801463046FBF773FFFCF779
:104B38003FFA60800220FEF78FFF90B133480622CB
:104B48000378591CCBB20370B3FBF2F002FB1031AF
:104B580011F0FF0F05D1FEF7DBFBFEF7FBFB2C4B3B
:104B680018702B4A1078003018BF0120FEF7F8FDA6
:104B780000F080FB18B100F09BFC60B904E0022053
:104B880003F076FC0028F6D0224B9A8A91B281F481
:104B9800885098820EE01A4B997819B11D4A4FF443
:104BA800885010855B781BB11A484FF48851816191
:104BB80004F0A4F8184B194A196810680B1A002B4E
:104BC80036DB0F4B587B88BB9870124B01F5F421EC
:104BD800988A80B280F48850988201F590731360A7
:104BE80026E000BF5A1F0020081D0020541900208D
:104BF8000CFEFFFF1F1E00202A1F0020321F00206E
:104C0800031F0020261E0020EC1D00204D0D002053
:104C1800440D002000100048400D0020580D0020D1
:104C28004A1F0020221E00201C1E0020012199700E
:104C380004F0E6FD0C4A107830B94FF40060FEF736
:104C48000BFF08B104F094F8202003F011FC18B110
:104C58000649086803F0F0FB054B9A680AB1054855
:104C6800904705B0BDE8F08F10140020400D0020DB
:104C7800041E0020E01D002038B50820FEF7ECFED9
:104C880010B19E4803F0F8FC04464FF48030FEF75C
:104C9800E3FE10B103F09CFD0446994B994A18684D
:104CA8001168431A002B02DA002C00F01C8200F570
:104CB8009C44203491489449146003F0EDFC4FF46F
:104CC8008040FEF7C9FE20B1904D2A780AB901F05C
:104CD800BBF88F4991F81B01B0B18E4CC31C34F955
:104CE80013504FF47A720021A5F57A70FFF7F0F8A7
:104CF800FBF744FF8849FCF749F88849FBF792FF1E
:104D0800FCF77CF9864A10804FF40070FEF7A4FE89
:104D180020B18449086803685C69A0477C4D00227B
:104D2800B5F81401B5F8164113467A499B08555E43
:104D38008542C4BF63F07F03DBB2A542B8BF43F02E
:104D480040030232082AF0D17748784A04780546A9
:104D58009C4204D11078F92803D8411C00E00021B6
:104D680011704FF480402B70FEF776FE68B1684DE5
:104D7800684BB5F81211B5F8DC20B3F90640881A6B
:104D8800844202DD8B189C420CDB4FF48040FEF716
:104D980063FED8B95F4C5E49B4F90650B1F81421E6
:104DA800954213DA01F05CF801F062F86048B0F857
:104DB80046305BB1554C5F492578002D00F02082C4
:104DC8000A78002A00F01C82FFF77CFD574B1C78FC
:104DD800142C40F0CB80574D6C78ECB1544BB3F8A1
:104DE80046502DB950490C785F2C01D101F02CF8B0
:104DF800474A92F81801002800F0B8804C4BB3F8E5
:104E08004650002D40F0B28047490C787D2C40F088
:104E1800AD8001F019F8A9E0434D2978572911D13F
:104E28004FF47A7000F03EFB4FF48070FEF714FEEA
:104E380008B102F0C9FA082003F01AFBE0B93E4BAA
:104E4800188019E00420FEF707FEA8B12A785A2A2C
:104E580012D13A48037823B104703948012202700C
:104E68000AE0384C257885F00101217009B102204B
:104E780000E00320FEF704FD2B4C25785D2D00F0A3
:104E8800C6815B2D00F0C5815E2D00F0C481284BE2
:104E9800B3F8465035B924490C786F2C02D1FFF786
:104EA80011FD15E01A4A204B92F8180118B115B9EE
:104EB8001D787E2DF3D01978972904D14FF4C87046
:104EC80000F0D2F904E0A72902D11A4A0124947308
:104ED80015480378BB2B03D11548818D8D1C04E040
:104EE800B72B04D11248838D9D1E858532E0BE2BD9
:104EF8002AD10F4D6A8D941C2BE000BF5C1A00204C
:104F0800400D0020500D0020581F0020141F0020C5
:104F1800541900205A1F002000007A4400C07F4422
:104F2800EA1D0020DC1D00204C0D0020630D002030
:104F3800081D0020031F0020261E0020620D0020EF
:104F4800540D00204F0D0020BD2B0FD1744D698DDD
:104F58008C1E6C85734C94F8AC03FEF71FFDFEF7AE
:104F68002DFDFEF797FF7048002202700420FEF71F
:104F780073FD00282CD06D4B1A788AB16C4845789F
:104F880075B16C49674AB1F90640B2F81401844218
:104F980006DD694D2C781CB9684932220A801C70DC
:104FA800654B587C50B1664B1D782DB9654C2278FD
:104FB80012B9624832210180012008E0614D2C7845
:104FC80034B15B4A517819B95F4B297001201870C8
:104FD80000235E4C1A4634F8020F40F2135501B212
:104FE800A942CCBF0025012505FA03F5A0F215500A
:104FF800B0F5C77F8CBF002001202A435D1C00FA52
:1050080005F0024340F2A4608142D4BF002101218F
:10501800981C01FA00F103330A430C2B92B2DAD13F
:1050280000233F49444C01EB4300B0F846100A42C4
:105038000CBF0020012018550133152BF1D16278DF
:1050480022B1022003F014FA68B914E04FF400709A
:10505800FEF702FD78B13E4C2168086883689847DE
:105068000028EED107E0324CE17839B900F0F8FEBB
:105078000120E07002E02E4C0022E2702E4B2C4CF6
:10508800987830B121790022E27019B900F0E8FE71
:1050980001202071284B26491A780AB90120087086
:1050A800CA782C4B12B92249087918B14FF48841B3
:1050B800996102E04FF488421A85202003F0D8F95C
:1050C80008B103F05BF91C4B19481A7B02B10122A5
:1050D800144982724B79082B01D00E2B45D1144A02
:1050E8000020507241E01C480268042A3DD8DFE8DD
:1050F80002F00305080B35000121016003685A1C02
:10510800026001684B1C036013480268511C01606F
:105118004FF48070FEF7A0FC00B302F029FB24E0F6
:10512800081D002054190020630D00204F0D002099
:10513800031F00205A1F0020141F0020680D0020A4
:105148004E0D0020620D0020540D0020601F00202D
:10515800DC1D002000100048640D0020364B0020A4
:1051680018604FF40050FEF777FC00F04BFB334B10
:1051780033499A890860334B1AB11968411A0029D2
:1051880059DB84181C6001F00BF9FFF7BBFB00F03A
:1051980039FB2D4B2A4A19681060441A18602B48AD
:1051A8002B4A90F87630148053B12A49CC780CB940
:1051B8000A792AB12848294BC48819880A19C28053
:1051C800202003F055F940B12248C3790BB9017A80
:1051D80019B1047B0CB103F047F82148214A174B59
:1051E80000F11E011468B3F8F62000F12903A04766
:1051F80001F060FC01F0DCFBBDE8384001F034BC94
:10520800487800283FF4E2AD00F01EFEDEE50121FB
:1052180002E0022100E00321CCB20848621E80F8B7
:10522800AC23FEF7CBFBFEF709FE0220282122461D
:1052380006F0ACF82BE638BD640D002054190020A8
:10524800400D00205C0D0020480D0020081D0020A6
:10525800600D0020031F00202A1F0020780E002068
:10526800091D002008000020014B1880704700BF6E
:10527800720D0020034B1888D0F1010038BF0020C0
:10528800704700BF720D0020F8B51E4B0022196848
:1052980013461D4C2588B5F5C87F1C4D01D1002645
:1052A800EE501B4EEF5832F906C0184C6744EF50C9
:1052B8000025043395538D5202320C2BE9D1124B41
:1052C8001A88012A18D1236803F1C8024FF4C87359
:1052D80092FBF3F20A806268C83292FBF3F24A80CA
:1052E800A268C83292FBF3F30A4A12889B1A8B8091
:1052F80000F0B2FDFEF7D8FD034801884A1E02807F
:10530800F8BD00BF740D0020720D00208C0D002028
:10531800401E002004000020F8B5354B04461888CC
:1053280032280ED13349344D0A68344816885788D4
:105338009388218862882E806F80AB8001804280AC
:1053480001E0002834D02B4D00222E681346284F48
:105358002B493888322801D10025CD502948CD580D
:10536800175EED19CD50002104331152B1520232AB
:105378000C2B0D46EBD11E480188012914D1224B74
:10538800224A022011701D70FEF77AFA1A4A19484B
:105398001188036850889288198058809A80174B22
:1053A8001988588821806080114B1A88511E1980ED
:1053B80017480378DBB10F4900220B6810490270C7
:1053C8000868322290FBF2F01880486890FBF2F0EF
:1053D800588089680F4891FBF2F201882046521ADA
:1053E8009A8000F039FDBDE8F840FEF75DBDF8BDD4
:1053F800680D0020740D00206C0D0020780D002031
:105408007C0D0020401E00204E0D0020620D002063
:10541800540D002004000020064B02881988891AC0
:10542800198042885988891A5980808899880A1A67
:105438009A807047401E00200F4B10B559680446EB
:105448000E4888470D480E4A01461278FEF758F86C
:105458000C48038813B12046FFF716FF0420FEF717
:10546800FBFA10B12046FFF757FF07490868BDE867
:105478001040FFF7D1BF00BFF01D0020401E0020E4
:105488006A0D0020720D0020740D0020014B186079
:10549800704700BF740D0020014B1860704700BFB3
:1054A800A00D0020014B1880704700BFA40D0020FC
:1054B800034B1888D0F1010038BF0020704700BFA7
:1054C800A40D00202DE9F8433C4B3D485968884716
:1054D8003B483C4A01461278FEF712F83A480388DE
:1054E800002B42D0394C256800242F7826462546C3
:1054F80035490A88B2F57A7F08D1354B354A0020FC
:105508001421E85001FB0620FEF7EAFCDFF8B08022
:105518002F4B38F90400E9584FF014090A18EA50DB
:105528002C4B09FB0639FBF729FB01464846FEF7D9
:10553800DAFC002024F80800DFF88C802649B8F847
:1055480000206052012A2FD14846FEF70EFD814601
:10555800DFB13846FBF712FB01464846FBF71EFD54
:1055680098B14FF47A73A8F80030154B1A4A188886
:105578001188401A1880518858889288401A99884A
:105588005880881A9880BDE8F883114B4FF47A72D6
:10559800E858114B00F5FA7191FBF2F0E0520F2137
:1055A8000A20012205F0F2FE013604350234032EEA
:1055B8009ED105490A88501E0880D6E7041E00209F
:1055C800281E0020F00D0020A40D0020A00D0020B2
:1055D800E40D0020A80D0020680E002010B50D4B2A
:1055E800044600220C4821461A70FDF7C7FD78B919
:1055F80009482146FDF73CFE50B907482146FDF70A
:1056080075FC28B904482146BDE81040FBF76CBE7C
:10561800012010BDF00D0020041E002003780BB1FE
:10562800054A1370417809B1044B1970807808B1A4
:10563800034A1070704700BFF00D00206A0D00206B
:105648009C0D00202DE9F3410646084614461D46E8
:10565800FFF7C4FF002876D03C4A00231370072CBC
:105668003BD8DFE804F0080818212A333A0402205E
:1056780002F010FF31E04FF44870ADF806003449ED
:1056880001A88DF80430FDF7B5FA10B1314B0121AE
:105698001970012C21D02E48FDF71EFD20B10222E1
:1056A8002C489442027018D02948FDF789FB20B194
:1056B8000321284B8C4219700FD02548FDF7FAFAC0
:1056C80020B1042223489442027006D02048FBF7F8
:1056D80063FE10B11F4B052119701E4A107828B9B6
:1056E8000CB10446B8E7022002F0D4FE3046FFF7BA
:1056F80095FF022002F0BCFE10B1154C21688847C6
:10570800154B164C1A689047082002F0B1FEB8B144
:10571800642795FBF7F63046FBF730FA07FB16517E
:10572800804608B2FBF72AFA0D49FBF77BFA0146D7
:105738004046FBF76FF90B49FBF774FA206001E06C
:10574800002020600120BDE8FC8100BF6A0D002018
:10575800F01D0020880D0020041E00209C0E002053
:105768008988883C0000204108B503681A6890477A
:1057780008BD38B505460C4614F8011B19B1284672
:10578800FFF7F2FFF8E738BD08B50368596888479E
:1057980008BD08B503689968884708BD08B5036857
:1057A800DA68904708BD08B503681969884708BDD5
:1057B80008B503685A69904708BD0000034B4FF4C9
:1057C800085208B19A6170471A857047001000485E
:1057D80008B5024B1968884708BD00BFF40D0020C2
:1057E800024A034B00201A60FFF7F2BFC5570008B2
:1057F800F40D0020024B1A68501C1860704700BF57
:10580800F80D002010B5094A094913688C6810681A
:105818008342F8D1074A106811684FF47A725043EE
:10582800001BB0FBF1F102FB031010BDF80D0020C6
:1058380010E000E0FC0D0020014B1868704700BF25
:10584800F80D002038B50446FFF7DCFF0546FFF7E2
:10585800D9FF401BA042FAD338BD10B504462CB17D
:105868004FF47A70FFF7EEFF013CF8E710BD000037
:1058780030B56B4D9DB002AC0FCD0FC495E8030059
:1058880084E8030005F040FE4FF4D87006F010F8E5
:105898000121644806F04EF801214FF4CD2006F0AE
:1058A8003DF8012160481CAC06F02CF806F066F8BB
:1058B80041F6FF7024F86C0D032321464FF0904009
:1058C8008DF80630FCF7A6F84FF6FF71ADF8041016
:1058D80056482146FCF79EF8554D21465548FCF799
:1058E80099F821465448FCF795F828462146FCF7D4
:1058F80091F8082106224FF0904005F0C0FD0821DC
:1059080001224A4805F0BBFD09210122474805F05C
:10591800B6FD06210422474805F0B1FD07210422FF
:10592800444805F0ACFD04224248082105F0A7FDD3
:105938000C214148022205F0A2FD3F480D21022218
:1059480005F09DFD3C480E21022205F098FD3A48DD
:105958000F21022205F093FD01210A464FF09040E5
:1059680005F08DFD4FF090400221012205F087FDE2
:105978002E480021022205F082FD2C480121022236
:1059880005F07DFD02224FF09040042105F077FDDF
:105998000024FFF725FF4FF488524FF488432A85E7
:1059A8002B8525462548264A016802AB914205D138
:1059B80018198179112901D10122827103EBC501DE
:1059C800185904310135FCF725F80834032DE9D1BD
:1059D80008A805F0EBFD1B48089B1B4AB3FBF0F138
:1059E8001A48116001684FF47A73B1FBF3F2501E44
:1059F800B0F1807F09D2164B164AF021586082F820
:105A0800231000200721986019601348FBF754FE03
:105A1800FBF786FF6420FFF720FF1DB030BD00BFF5
:105A28000C0201080700420001003E100004004873
:105A38000010004800080048000C004868010020D9
:105A4800001BB70040420F00FC0D00206C01002035
:105A580010E000E000ED00E00058004010B540F212
:105A6800DB1460430F4B4FF488424FF488519A611E
:105A7800841E19850B48838A9AB282F488418182F0
:105A8800838A9AB282F4885181822046FFF7E5FE24
:105A98000120FFF79DFE1920FFF7DFFE0020FFF72A
:105AA80097FEE7E70010004810B1034A034B1A605D
:105AB80003480449C8607047EFBEADDEF04F0020D0
:105AC8000400FA0500ED00E02DE9F04F89B00793D6
:105AD800754B07460692B3F90000B3F90220002877
:105AE800B8BF4042002AB8BF524200248242B8BF21
:105AF800024605922546A146A0460494A24626469B
:105B08006A49CB7813B90A79002A38D0022E36D0E0
:105B1800674B6548EA5EDDF818B0295E02EB410084
:105B2800CBF100015A46FEF7D3F96249DDF81CC0F3
:105B38006B5E3CF90520C01A8318F879FA7E584341
:105B480064214FF0050E90FBF1F06FF00401514312
:105B58000EFB02F20393FEF7BBF9DFF878B1039B63
:105B6800824654F80B00544942F210721818FEF796
:105B7800AFF97A7C44F80B005043011304914B4869
:105B8800C3781BB102790AB9022E2FD14649502099
:105B980035F90180DFF828B100FB08F2BB5DDFF8BA
:105BA800389135F90B0092FBF3F154F809300A1AD1
:105BB800D01842494FF47A52FEF78AF935F90B109A
:105BC80049F804000029B8BF4942B1F5207F02DD39
:105BD800002049F8040059F80420B9197D23887A6F
:105BE80092FBF3FC00FB0CFE4FEAAE192F4B1A791F
:105BF800B2B1022E14D0DDF814B0DDF810C00BFBE2
:105C080008F0CBF5FA7303FB0A020BFB09F003FB60
:105C18000C034FF4FA7192FBF1F293FBF1F308E0F5
:105C2800D97809B1022E02D14B46424601E0049BC5
:105C380052462349DFF8A4B0695A16F80BC008B2D7
:105C48000CFB00FB6FF04F0C9BFBFCFC94441D4AC3
:105C5800CDF800C035F902C0A952CCEB00001A4AB1
:105C6800DFF87CC0019054F80C10A0584018019936
:105C780002904018A15844F80C100199A150134AF9
:105C88000434B15C202201FB00F090FBF2F1581AB9
:105C9800009B0F49C21801366A520235032E7FF461
:105CA8002FAF09B0BDE8F08F2A1F0020031F002086
:105CB80092100020A00E0020F0D8FFFF80C1FFFF47
:105CC800940E00200C0E0020280E00201F1E00201D
:105CD800161E0020200E0020000E0020221E00208C
:105CE800140E00202DE9F04F002485B003930546DB
:105CF8008946924606462346474AD17809B910791B
:105D0800B8B1022C17D0454B454F33F9140037F979
:105D18001420CAF1000102EB40005246FEF7D8F801
:105D28004049039F31F9143037F91420C01A8318F9
:105D38000AE0022C08D1394A99F80570B2F9041022
:105D48001B374F43791114E03348C17871B9334F89
:105D580099F8042037F914101B324A4300791111BD
:105D680038B16A7C5A4301EB222102E0EF795F43A4
:105D780039112D4FDFF8C4C037F91400BCF80020E2
:105D88000F1A295D7A437943DFF8B480D0124FEABD
:105D9800E11B58F82420B17A01FB0020234948F878
:105DA80024004FF400120293CDF804C0FEF790F8D7
:105DB8001F4BDDF804C053F8241043F82470791AF7
:105DC800BCF800704FF6FF723B09B2FBF3F74F4384
:105DD800184BDFF870C048F824005CF8241053F81A
:105DE8002480BF1108EB010243F82470337DD119D8
:105DF80059430BEB6030104A00EB21214CF824800A
:105E080022F8141001340136032C029B7FF474AF7E
:105E180005B0BDE8F08F00BF031F00202A1F002037
:105E280092100020A00E0020940E00200000E0FF39
:105E3800400E00204C0E0020161E0020600D002091
:105E4800000E0020340E0020024B5A780AB10020C0
:105E580058707047031F0020002303804380704759
:105E6800024B00221A605A60704700BF200E0020C3
:105E7800024B00221A605A609A607047000E002098
:105E88000128034B14BF034A034A1A60704700BF36
:105E980008000020D15A0008ED5C0008000000004E
:105EA8002DE9F84F384E04463768384606F0B8FBF7
:105EB8000546384606F028FC76688046304606F0E7
:105EC800AFFB8346304606F01FFCD4F80490064624
:105ED80029464846FAF7A6FEA7688246414638464C
:105EE800FAF7A0FE01465046FAF792FD216882466D
:105EF8005846FAF797FE414604464846FAF792FE96
:105F08003146FAF78FFE01462046FAF783FD3146FF
:105F180004463846FAF786FE2946FAF783FE014614
:105F28002046FAF777FD0146504606F079FC1749F6
:105F3800FAF778FEFAF7B2FA11A3D3E90023FAF7D1
:105F48002BFC134B044618680D46FAF7A7FA0246CD
:105F58000B4620462946FAF743F900220D4BFAF77B
:105F68001BFCFAF701FD06F08FFB81B20A0444BF5F
:105F780000F5B47189B208B2BDE8F88FAFF30080BC
:105F8800182D4454FB2109405C0E00200000E14418
:105F98009C0E00200000244010B5194C2088FAF708
:105FA800EDFD1849FAF73EFE06F06EFB164B188019
:105FB8002088FAF7E3FD01461448FAF7E7FE14498A
:105FC800FAF7E4FE134908601348B0F87400FAF7CA
:105FD800D5FD01461148FAF7D9FEFAF75FFA06A38C
:105FE800D3E90023FAF7AEFAFAF7BEFC0C4A1060C0
:105FF80010BD00BFAFF300803B597E90A9E78140F8
:1060080004000020C903683F580E00200AE81C411C
:1060180000401C463C1E0020081D00200000614472
:10602800581E0020AFF300802DE9F04104460068B7
:106038000D460146FAF7F6FDD4F8048006464146B7
:106048004046FAF7EFFD01463046FAF7E3FCA76849
:10605800064639463846FAF7E5FD01463046FAF76E
:10606800D9FC06F0DFFB00210646FAF76FFF70B98E
:1060780020683146FAF78AFE314628606068FAF7E8
:1060880085FE31466860A068FAF780FEA860BDE822
:10609800F0812DE9F04F0C68836889B0D0F800A032
:1060A800D0F804800646204603938B4606F0B8FADB
:1060B8000746204606F028FBDBF8044081462046C8
:1060C80006F0AEFA0546204606F01EFBDBF808206F
:1060D80004461046019206F0A3FA8346019806F09A
:1060E80013FB394602905846FAF79CFD394604904E
:1060F8000298FAF797FD594605904846FAF792FD37
:10610800029906904846FAF78DFD294607905846A9
:10611800FAF788FD01465046FAF784FD2146834682
:106128000698FAF77FFD01460598FAF773FC0146D1
:106138004046FAF777FD01465846FAF76BFC2146C8
:1061480083460498FAF76EFD01460798FAF760FC53
:1061580001460398FAF766FD01465846FAF75AFCD5
:106168003060029905F10040FAF75CFD014650469F
:10617800FAF758FD214683460798FAF753FD01467A
:106188000498FAF745FC01464046FAF74BFD0146EC
:106198005846FAF73FFC214683460598FAF742FD30
:1061A80001460698FAF736FC01460398FAF73AFDD5
:1061B80001465846FAF72EFC214670605046FAF719
:1061C80031FD2946044609F10040FAF72BFD014646
:1061D8004046FAF727FD01462046FAF71BFC3946E8
:1061E80004462846FAF71EFD01460398FAF71AFDF9
:1061F80001462046FAF70EFCB06009B0BDE8F08F02
:1062080080EAE073A3EBE0738B4206DB002801DD34
:10621800401A704702D040187047002070470000AD
:106228002DE9F041524B86B01A685B6802F10042D2
:1062380003F1004301934F4B0646B3F90000009267
:10624800FAF79CFC00F10040FAF728F946A3D3E9D5
:106258000023FAF777F9FAF787FB474C0290B4F96D
:106268000000FAF78BFC0390B4F90200FAF786FCF9
:106278000490B4F90400FAF781FC6946059003A874
:10628800FFF707FF3D4B93F84430012B16D13C48EC
:10629800417869B93B4C4025226892FBF5F7D01B41
:1062A800FAF76CFC0599FAF7B5FBFAF781FE20605E
:1062B800344B4021186890FBF1F001E0324B18880C
:1062C800FAF75CFC01460598FAF7A2FB0590304600
:1062D800FAF750FC2D490746FAF79CFB0146384669
:1062E800FAF754FD2A4D07462C6805982146FAF717
:1062F8008FFB01463846FAF795FC01462046FAF727
:1063080089FB244C28601D4D07460398D4F800806B
:1063180006F0BAF995F83010FFF772FF08EB0002A3
:1063280004982260D4F8048006F0AEF995F830108D
:10633800FFF766FF08EB000338466360D4F808806F
:1063480006F0A2F995F82F10FFF75AFF1249134BE0
:106358000A684044A0601868B6180E60411C1960AD
:1063680006B0BDE8F08100BF399D52A246DF913FDB
:106378005C0E0020261E0020501E0020081D002054
:10638800031F00207C0E0020040000203661823CA0
:10639800640E0020301E0020740E0020800E0020A5
:1063A8002DE9F04F87B0FFF78DF8022002F060F872
:1063B800002800F0AD81AE48FFF73EF8FFF722FA5B
:1063C800AC4C05462768C71B3846FAF7D3FBAA49E1
:1063D800C968FAF727FC8346A848256090F82E80FC
:1063E80000252C462E46A64A105FFAF7C7FB5946E9
:1063F800FAF718FC03AB5851B8F1000F27D0404604
:10640800FAF7BCFB01464FF07E50FAF7BFFCDFF805
:10641800B092824651464FF07E50FAF7F9FA55F895
:106428000910FAF7FFFB97490346085F0193FAF74B
:10643800A5FB5146FAF7F6FB01460198FAF7EAFA86
:1064480049F80500FAF7B4FD8F4A105303E08D4967
:106458008D4A605AA0528C4B0435E15E0234062CFA
:1064680001FB0166BFD1894A6420138846435B4318
:10647800874803A996FBF3F6FFF70BFE082001F007
:10648800F7FF20B1834803A9FFF703FE07E082481E
:1064980003A9FFF7FEFD80480146FFF7C5FD493E09
:1064A8007E49B4B23B2CB1F8F00007D97B4E0820E6
:1064B800B6F8F25001F0DCFF30BB4FE0FAF75AFBB8
:1064C8004FF07E518046FAF7A5FA01464FF07E500C
:1064D800FAF75CFC002406466D4D404655F814104A
:1064E800FAF7A0FB81466848005FFAF747FB0146C8
:1064F8004846FAF78FFA3146FAF794FB45F8140044
:106508000234062CE8D1D1E7B6F8F200FAF732FBEC
:1065180080462846FAF72EFB4FF07E51FAF77AFAB2
:1065280001464FF07E50FAF731FC00240646594DDB
:10653800404655F81410FAF775FB594A8146105F22
:10654800FAF71CFB01464846FAF764FA3146FAF7AF
:1065580069FB45F814000234062CE8D1514B4C4D28
:10656800B3F90000FAF70AFBAC6801462046012699
:10657800FAF714FD00B906464B4968684E73214680
:1065880006F04EF9494CD5F808802060286800F1DB
:10659800004668680146FAF745FB4146054640460D
:1065A800FAF740FB01462846FAF734FA06F03AF9BA
:1065B8000146304606F034F960602068F9F76EFF4E
:1065C80029A3D3E90023F9F7BDFFFAF7CDF906F0BF
:1065D8005BF8374D28806068F9F760FF22A3D3E99C
:1065E8000023F9F7AFFFFAF7BFF906F04DF8688016
:1065F800082001F03DFF2F4C08B1264800E026484E
:10660800FFF74EFC1D4D20803846FFF709FE95F830
:106618007620002A00F080801D4B18689C6801468F
:106628005F68FAF7FFFA394606463846FAF7FAFA83
:1066380001463046FAF7EEF9214606462046FAF7B3
:10664800F1FA01463046FAF7E5F906F0EBF80146AB
:106658002046FAF79BFB18490446FAF78BFC88B3E7
:1066680016480021018057E03B597E90A9E78140F8
:10667800321D0020900E0020041E0020081D00205E
:10668800281E0020401E0020501E0020040000206C
:106698005C1E0020840E00200C00002054190020ED
:1066A800FC1D0020580E0020031F00205C0E002057
:1066B800A00E0020261E00208FC2753C780E0020F8
:1066C800A40E0020204606F05BF8274B1968FAF75D
:1066D800A9FA05F0D9FFB0F5617FA8BF4FF4617042
:1066E800F9F7CAFE1EA3D3E90023FAF755F8FAF71B
:1066F8003BF906F009F8044695F87600FAF73EFAF1
:106708002146FAF78FFA05F0BFFF184B188003E00F
:10671800174B188058809880164A5379012B164BCE
:1067280007D0164819885A889B8801804280838040
:1067380011E01349B3F90420B1F9000002EB40005D
:10674800032290FBF2F080B20C4A088019885B881B
:1067580090801180538007B0BDE8F08FAFF30080C0
:10676800A2EB0FE5DD169640581E0020780E00209B
:10677800401E002054190020281E0020940E0020DE
:106788007A0E0020AFF3008010B5054C0020218858
:10679800FBF7A4FA61880120BDE81040FBF79EBA18
:1067A8001800002010B5094C20600948016009490B
:1067B80009480A60094A0A491360029B039A036060
:1067C8000848049B0A60036010BD00BFB00E00209B
:1067D8008C0F0020880F0020B80E0020900F00209A
:1067E800C00E0020C40E0020094B1A6802EBC0013D
:1067F800CB79FF2B04D01BB1064830F8130004E016
:106808000728D4BF888840F2DC5000B2704700BF28
:10681800B00E00205A1F0020054B1A6802EBC0007A
:1068280090F9063019420CBF01204FF0FF30704735
:10683800B00E002010B500244FF48040FDF70CF98D
:1068480008B1054B00E0054B1868054A8188A1523C
:106858000234182CF0D110BD8C0F0020880F0020B6
:10686800801E0020F8B53A4B3A4E0546187006EBE4
:10687800C0000F46384C417820202160FDF7ECF825
:1068880008B101222260162D19D10024385900219F
:10689800FAF75CFB28B14FF48040FDF7DDF850BBF8
:1068A80025E02E4A3B1916190FCB86E80F002C4815
:1068B800103401784A1CC02C0270E7D1EBE716F8B7
:1068C800357006EBC506264BD6F804E01F70BEF1FE
:1068D800000FE0D00024BC42DDDA204E200136183B
:1068E8000EEB00010FC9013486E80F00F3E7082D0D
:1068F8001C4B23D124E01A4F3F78012FF7D91A4CAB
:1069080000261034BE42F2DA54F8100C4FF07C51D5
:10691800FAF788F94FF07C5144F8100C54F8140C2D
:10692800FAF780F94FF07C5144F8140C54F80C0C29
:10693800FAF778F9013644F80C0CE2E70E2D01D18C
:10694800012000E000201874BDE8F840FFF772BF8E
:10695800B40E0020B8050108940F0020C80E0020CE
:10696800BC0E0020031F0020D00E0020F0B58C467E
:10697800461C002300224CF803201033C02BF9D109
:106988000A4800EBC6014F6807B9F0BD0024074B61
:1069980013F83620944208DA20010CEB0005391868
:1069A8000FC9013485E80F00F1E7F0BDB80501080B
:1069B800284B10B5186800284AD027490A78531E72
:1069C800142B3DD8DFE803F00B3C3C24403C3C1C36
:1069D8003C3C3C3C3C2C3C3C3C3C3C242C001F4874
:1069E80001684A7832B11E4900204989BDE8104043
:1069F800FBF774B91B4B58780028F4D10146F5E72A
:106A0800174C0020E188FBF769F901202189EDE79F
:106A1800134C00202189FBF761F901206189E5E722
:106A28000F4C0020E188FBF759F901202189FBF779
:106A380055F902206189FBF751F90320A189D5E7AF
:106A48002020FDF709F818B1BDE81040FFF79CBEFB
:106A580010BD00BF940F0020B40E0020900F00203E
:106A680018000020031F002010B50024064B1878DA
:106A7800A04208D90549204631F814100134FBF723
:106A880021F9E4B2F2E710BDBC0E0020681E002018
:106A9800064B1A780023D9B2914204D2044921F84E
:106AA80013000133F7E7FFF7DFBF00BFBC0E00207C
:106AB800681E00202DE9F74FA34B187803280FD93B
:106AC800A249A34CB1F904206FF06305002AB8BFAE
:106AD8005242A91AB4F904006432FDF7F9F9A0800A
:106AE800994A1678012E1DD89A4E3478651E9A4C0C
:106AF800142D00F2C981DFE815F0A400C701C70111
:106B08007B00B300C701C7015A01C701C701C7010C
:106B1800C701C701D000C701C701C701C701C70125
:106B28005F00A1018D488A4B884F0168B7F806B00D
:106B3800B3F800805F88B3F904A0894C019100255F
:106B48001034B542D0D20FFA8BF0FAF717F854F890
:106B5800101CFAF767F8814638B2FAF70FF854F8BC
:106B6800081CFAF75FF801464846F9F753FF8146D3
:106B78000FFA88F0FAF702F854F80C1CFAF752F8F2
:106B880001464846F9F746FF019A814692F9000006
:106B980041420AFB01F0F9F7F1FF54F8041CFAF737
:106BA80041F801464846F9F735FFFAF701FA6D4B07
:106BB80023F815000135C3E701210420FFF72CFE57
:106BC800634D654C6E88704387B204202781FFF7B8
:106BD8000BFE3818208101210520FFF71DFE2B88A8
:106BE800584385B205206581FFF7FEFD2B1826E086
:106BF80002210420FFF710FE554C0121A68870439E
:106C080087B20420FFF708FE6588534C00FB057225
:106C1800042097B2FFF7E8FD3818208102210520EB
:106C2800FFF7FAFD7043012186B20520FFF7F4FD56
:106C380000FB056105208DB2FFF7D6FD2B18638197
:106C480022E101210520FFF7E7FD414A424E9788DE
:106C5800784384B20520FFF7C7FD2018708113E13F
:106C6800414900200D68FFF7BFFD404F95F90630F8
:106C7800B7F902607343322693FBF6F2801820803E
:106C88000120FFF7B1FD95F90E10B7F900506943DF
:106C980091FBF6F3C7186780F6E03549354E4A7818
:106CA800376812B9B888E08108E0284C3988B4F907
:106CB80006007A88FDF70CF9274BD881264D2E4F10
:106CC800E989284A3E681180347854B3264D022059
:106CD800FFF78AFD2B68B3F91010B3F91220FDF7FE
:106CE800F7F82649264B0A68198854890EB2201AE3
:106CF80002B2964203DA3E683278511803E003DDA7
:106D08003F683878091A19802D681D4F95F9163093
:106D1800B7F90000642143430F4A93FBF1F6A41925
:106D28009480134D0C4BAF7A67B1084801880E4A1E
:106D3800D9801981868817685E814488064D9C81B0
:106D480003241FE00248F1E7BC0E00202A1F0020A0
:106D5800161E0020B40E002018000020900F0020FE
:106D6800C80E0020681E0020B00E0020A00E0020D3
:106D7800031F0020880F0020B80E0020C00E00203E
:106D8800B60E002007EBC40393F90600B5F9061008
:106D98006426414391FBF6F6EE802046FFF724FD7A
:106DA80001343218EA800235072CEBD16CE0A54F8C
:106DB800A54B78781E6810B9B588E58108E0A34925
:106DC8007288B1F906003188FDF782F8A04AD081AF
:106DD8009F4C9C4B9F48E7899E7A0780012103209E
:106DE8001EB1FFF719FD994D02E0FFF715FD9A4D09
:106DF8006E880221704387B20320FFF70DFD2D88AE
:106E080000FB05710420E1800121FFF705FD7043B7
:106E1800022186B20420FFF7FFFC00FB0562032075
:106E28002281FFF7E1FC8A4CE388C018E080042047
:106E3800FFF7DAFC2789C519258125E0864A03244E
:106E4800978802212046FFF7E7FC7843012186B2A4
:106E58002046FFF7E1FC804DC4F10603590835F8D8
:106E680011207B4D00FB026086B225F81460204695
:106E7800FFF7BAFC331825F814300134072CE0D199
:106E8800724F744AF98811802020FCF7E5FD00282C
:106E980045D00020FFF7A8FC6D4F0546388001203B
:106EA800FFF7A2FC6D4978800B7A002B37D06C4A2B
:106EB8006C4B14686C4A267806F00201CCB2D4B147
:106EC8001468B3F9001094F90E2094F906404A4367
:106ED800322192FBF1F6B3F90230B2B26642734343
:106EE8006FF0310493FBF4F69419651993FBF1F1F3
:106EF8003D80561811E01168B3F9026091F9064017
:106F08003222664396FBF2F42D193D8091F90E105A
:106F1800B3F900304B4393FBF2F6801978800026D2
:106F2800514F4B4D3B68A85F03EB860233F926109F
:106F3800B2F90220FCF7CCFFA8530236102EEFD18D
:106F4800474C2168087800F00407FBB22BB9414A86
:106F5800464C1688277801231CE0454D2E780E2EC6
:106F68000AD0082E08D0434A02EBC60461780029EB
:106F780014BF0225002500E0042500263E4F7019A5
:106F880007EB4603C0B219890136FAF7A7FE042EAB
:106F9800F4D1DCE7BB4209D22E4C36B234F91310D7
:106FA8000133B142A8BF0E46B6B2F3E70024274624
:106FB8002E490878874272D2234D31B22B685A88FD
:106FC800914204DD2348951B235AEA1822524FF4B4
:106FD8008040FCF741FD1F4DC0B1284A264B106880
:106FE800B3F906104389184A9942254905DD09680D
:106FF8001268285F4988528804E012680B68285F85
:1070080091881A88FCF764FF28533EE0DFF838803F
:10701800285FD8F8003005EB040919885A88FCF76E
:1070280057FF164A144913682853B1F9060099897D
:1070380088422ADA1020FCF70FFDD8F8002008BB98
:10704800108820E0031F0020880F00202A1F00203E
:1070580018000020681E0020161E0020141F0020A3
:10706800C40E0020A00E0020B00E0020BC0E002090
:10707800B40E0020B80501085A1F0020C00E0020D9
:107088008C0F00209088A9F80000064843781BB9A7
:1070980005490648625A22520137023488E7BDE89A
:1070A800FE8F00BF031F0020801E0020681E0020E6
:1070B800024B1868003018BF01207047940F002059
:1070C80044F25063984203DDA0F50C40A0387047A5
:1070D80003498842BCBF00F50C40A030704700BF90
:1070E800B0B9FFFF10B5F9F749FD00210446F9F7DB
:1070F80055FF08B1204601E004F100400549F9F7C1
:1071080045FE0549F9F78EFD05F08AFA034B18602C
:1071180010BD00BF8096184B35FA8E3C2800002021
:1071280010B5044C002320702361FEF785FB6061D5
:1071380010BD00BF04110020F8B51D4614460E46C8
:10714800F9F71CFD6968F9F76DFD3146F9F76AFD35
:107158002168F9F75FFC2060F9F72AFFED68074618
:1071680005F10040F9F724FF06462846F9F720FF05
:10717800314602463846FCF7ABFEF9F7FFFC2060C3
:10718800F9F716FFF8BD0000F8B5101A0C461F46AF
:10719800F9F7F4FC0546381BF9F7F0FC174B079E86
:1071A8001968F9F73FFD294604462846F9F73AFDDC
:1071B800214607462046F9F735FD01463846F9F7D6
:1071C80029FC05F02FFB0E49F9F72CFDF9F716FFFE
:1071D80006990860214605F1004005F021FB0949A0
:1071E800F9F720FD0849F9F715FCF9F7E1FE002841
:1071F800BCBF00F50C40A0303060F8BD280000206E
:107208002C7D8E3FA00CB34500A00C4610B504465B
:10721800002003460D49CA5CA2B12E2A04D10133CD
:1072280094B1C91800220A55084A0A21D25C484379
:10723800A2F13001092901D8303880180E2B02D864
:107248000133E7E710BD002010BD00BF7810002013
:107258002DE9F843224B074648681D68381A0C4642
:107268009146F9F78BFC2946F9F790FD1D492061F5
:107278000A6880469078F9F77DFCF9F70FF916A3AC
:10728800D3E90023F9F75EF902460B4600201649B8
:10729800F9F782FAF9F768FB2946F9F7BBFB0146CB
:1072A8002846F9F773FDA668054631464046F9F7C2
:1072B800AFFB01462846F9F7B5FC01463046F9F719
:1072C800A9FBD9F8081020616760A060F9F7AAFC4B
:1072D800F9F76EFEBDE8F883182D4454FB211940D8
:1072E800A8100020601000200000F03FAFF30080DD
:1072F800014B1860704700BF60100020F8B52D4B97
:10730800187810B1012850D10AE02B4B2B4A587835
:107318002B4B02EB001149681868FEF73FFA41E071
:10732800274D2868FEF73FFA00283ED0224C2178E6
:10733800264601291ED1FEF77FFA06466069321AF1
:10734800632A35D92169042912D81C4F286807EB0C
:1073580001135968FEF722FA607807EB0017B9683D
:107368002868FEF706FA22696661511C21611CE053
:10737800022018E022693AB96478104B286803EBB8
:1073880004114968FEF70AFA33690B4C8B2B09D8AC
:107398000C4A0B48D15C0068FEF7E6F921694B1CE2
:1073A800236102E00320FFF7BBFE034A0020506080
:1073B800F8BD00BF9010002004110020980A0108B1
:1073C8005C1000200A0A010810B50B4CE37A8BB157
:1073D8000A48017804290DD9094A0A4B10685168EE
:1073E80018605960FFF77EFE0748084B02880121A4
:1073F8001A80217310BD00BF031F0020F01E00205B
:10740800D81E0020BC1E0020261E00206810002068
:10741800002370B51C460F48002119521420604300
:107428000D4A0E4E0E4D99520022325059533518BE
:107438000C4E6960AA60325035180B4E01346960F1
:10744800AA6002333518022C32506960AA60E2D172
:1074580070BD00BFA4100020921000201C10002056
:1074680024110020C40F0020C010002070B504466D
:107478000079F9F77FFB1E49F9F788FC1D4D1E4E70
:107488002860A07BF9F776FB1949F9F77FFCEE60D5
:1074980068606079F9F76EFB1849F9F777FC184DC1
:1074A8002860E07BF9F766FB1149F9F76FFC686023
:1074B800607EF9F75FFB1349F9F768FCEE60A86096
:1074C800A079F9F757FB0D49F9F760FC0E4D2860D4
:1074D800207CF9F74FFB0649F9F758FC6860A07E55
:1074E800F9F748FB0749F9F751FCEE60A86070BD51
:1074F8000000C842441000200000FA440000204167
:10750800FC0F002000007A440C1000202DE9F34104
:107518001A4F0E461A491B4D3A701B4A0860002044
:107528001360DDF82080FFF7FBFD6E70FEF784F92D
:10753800A860387800246C60A0420CBF01250325A0
:107548004046FFF793FF114B214603EB06160094C4
:10755800102072682B4602F0F7F80D49086030B920
:107568004FF4807002B0BDE8F041FCF7F5BB012094
:1075780002B0BDE8F041FFF7D3BD00BF9010002076
:10758800301100200411002060100020980A010822
:107598005C100020F7B5264B1D78032D44D1202020
:1075A80001F0C4FF234E044638B102F033F93168C4
:1075B8002046C968FEF7F2F80AE0326800902146D2
:1075C8002020D2682B4602F0BFF8044600282DD0B0
:1075D80019484FF488554FF4884605850685174F96
:1075E8003868FEF7D1F858B1134D4FF48856AE619C
:1075F8003868FEF7CEF801462046FEF7B5F82E8526
:107608002046FEF7C1F80028E9D00B4D0B4B4FF48C
:107618008846AE6120461F68FEF7BBF8014638462B
:10762800FEF7A2F82E85DAE7022000E02846FEBD24
:107638000411002030110020001000485C100020C8
:10764800F7B50368164C174D23600968164E61603C
:107658000068FFF747FD94E80C0014480196009075
:1076680095E80300FFF790FD6B68114A616836687A
:10767800C81A1660F9F782FA0E4A0F4F1168F9F71F
:10768800D1FAF9F795FC2968786020680B4A431A03
:107698000B483B60016816600A4BCA881A80FEBD19
:1076A80070100020D81E0020EC1000209810002038
:1076B8006C1000202800002034110020FC1000204D
:1076C800601000202C110020264BF0B51D680246E2
:1076D80000F1100116781446AB195B78013203F0FB
:1076E8000403DBB263B18A42F4D10020F0BD13B1C8
:1076F8000A225343DBB210F8011B30395B18DBB2A6
:10770800211A0229F3DC0021844209D911B10A2285
:107718005143C9B210F8012B303A8918C9B2F3E7BE
:107728002E2E11D10134042000220A267243267815
:10773800AF197F7807F00407FFB217B1303A9219F2
:1077480001340138F1D100E00022074C6420614384
:1077580000FB021106240548B1FBF4F200FB0320EC
:10776800F0BD00BFA401002040420F0080969800A1
:107778002DE9F04F9A4B8BB01868B8B9994C21781D
:107788004A1E032A00F26585DFE812F0F704F704C1
:1077980042052C052068FDF7FCFF934904460B7849
:1077A800012B00F0DF8008D3022B06D08C4C206818
:1077B800FDF7EAFF0028EDD1E0E7242C07D18B4B39
:1077C8008B4A8C4C0021197011702170C5E02C2C4B
:1077D80002D02A2C40F08280854D844A2978864B35
:1077E800157800205854854AB5B918781570472877
:1077F80068D15978502965D19878472840F017857D
:10780800D978472940F013851B79412B40F00F8523
:107818000120107000F00BBD117801293AD1022D1A
:1078280005D11846FFF750FF754908604AE0032D57
:1078380007D11978532945D171480268534203602A
:1078480040E0042D05D11846FFF73EFF6C4B586009
:1078580038E0052D07D11B78572B33D168494A6882
:10786800504248602EE0062D07D119786548302926
:1078780094BF00210121C17224E0072D04D1FFF734
:10788800C5FC614A10701DE0092D1BD1FFF7BEFC35
:107898005E4B16E0022915D1072D0CD10120FFF708
:1078A800B5FC41F2184250434FF47A71584BB0FB83
:1078B800F1F0188006E0082D04D10120FFF7A6FC9E
:1078C800544B1880494B4A49013500202A2C1D7019
:1078D800087039D15048012404703EE00D2C4E4AFE
:1078E80001D00A2C26D11478FCB1434C2178647855
:1078F800A1F13000C3B2092B84BFA1F13703DBB279
:10790800A4F1300003F00F02C3B21101092B84BFA8
:10791800A4F13703DBB2374C03F00F028918207843
:10792800CBB2C21A514251EB02043B4B00201870F3
:107938007CB912E02E490B780E2B03D82E48C4547C
:1079480001330B70127842B92A4B1A7854401C70D4
:1079580003E02A4A1078012800D00020C00700F16F
:10796800338123E72D4B0022197808293FF61EAFF3
:10797800DFE801F00A05111927607C96A00062284B
:1079880001D1022105E01A70B52C7FF40FAF1C78E5
:10799800611C19700AE72249224A03261E700870E2
:1079A8001070214B0BE01F4E0421197032781E4BCA
:1079B800A1181878CAB2101818701C4B32701C70B5
:1079C800F4E605211970174B174E1A783078A1186C
:1079D800CAB210183070164E1A703480E6E600BF2E
:1079E8005C10002004110020901000206510002079
:1079F800F80F0020F90F002078100020C00F002099
:107A0800D81E0020031F0020F01E0020AA1E002000
:107A1800AE1E0020F8100020021100206610002081
:107A2800001100205810002067100020C10F00200E
:107A3800FA0F00206C4906261E700A786B4BA618B0
:107A48001878F2B210181870694B0A70198801EB8F
:107A58000424A6B2B6F5007F01D81E8003E00022F8
:107A68001A80644B1A700024634983E35E495F4EB1
:107A78000A783078A318DAB2101830705E4E0A709F
:107A880033885B4AC72B98BF5C49108898BFCC5491
:107A98005C1CA1B2884231807FF488AE072107E0E0
:107AA800514808261E700378A3423FF47FAE002198
:107AB800504B6EE74D4E1A70337883427FF476AEA2
:107AC8004F4C207806283BD005D8022813D003282D
:107AD8007FF46CAE23E0122847D030287FF466AEDE
:107AE800464A484C1679454A102E88BF10262670FB
:107AF8002178002347E0414C434E6368A068216920
:107B08007360424B4FF47A723060414C91FBF2F64D
:107B1800187840492680C87201223F4923E0374936
:107B28004A7912F0010004D00E79F41E634253EB37
:107B3800040036490870002839D1364AD07236E038
:107B48002E4EF47A14F0010104D0B07AC21E5342CA
:107B580053EB02012D4E317009B92E4CE1722748C2
:107B68002E4990F82F200A7021E024482C49866974
:107B7800426942F210742B4B96FBF4F00A8018808D
:107B880001222949EFE70C328B4210DA12F8046C13
:107B9800264812F8034C1E54254E26489C5512F8C8
:107BA800014C16781C54244C1E550133EBE71A4936
:107BB8000A78002A3FF4FAAD1B4B1E78002E3FF4DA
:107BC800F5AD00240C701C701C4CA068E060FDF73B
:107BD80033FEA060202000F055FC19490A78012ADC
:107BE80030D100232FE000BF58100020671000207C
:107BF800FA0F002066100020081200204011002013
:107C0800C10F0020F11E0020D81E00202A110020DC
:107C1800AA1E0020031F002064100020F01E002070
:107C2800AE1E0020F810002001110020981E002030
:107C3800C61E0020E01E0020F21E002004110020B5
:107C48002E11002001230B700C787E497E48CA7AD9
:107C5800C480002A3FF4AAAD7C4B1C78042C7FF624
:107C6800A5AD4F7807B90F730D7B15B90FB1FFF7A5
:107C7800ABFB774E05213078764F421C92FBF1F32F
:107C880001FB13243470744E97F800C0734D06EB53
:107C980084020023724873491C58DFF814E2724EBC
:107CA8005C5094FBFEF103EB000A06FB01406F4FAA
:107CB80042F21074DFF8FC91D95190FBF4F7166882
:107CC800BCB253F809701060C6EB0708404405269B
:107CD80043F8090090FBF6F00EFB01016448BCF183
:107CE800010F25F8024F195005D1023CB4F5797FF0
:107CF80098BFCAF8001004331432082BCAD1FDF714
:107D08009BFD5C4D5C4C2A68801AF8F733FF5B4991
:107D1800F9F73CF82060FDF78FFD286025684FF0E3
:107D28007E512846F9F71CF908B94FF07E552560B1
:107D380006A907AC4A48524B0194009103C80CCBE2
:107D4800FFF722FA069A64234E49B2FBF3F0088043
:107D5800079A3C4892FBF3F34B4C027B23800AB909
:107D68000A80228049490C78002C36D0424F4FF0C7
:107D78007E503968F9F70AF8454D394E2B680446A4
:107D88003068C01AF8F7FAFE2146F8F74BFFF9F702
:107D98000FF9726869683F4D0746501AF8F7EEFE0A
:107DA8002968F8F73FFF2146F8F73CFFF9F700F993
:107DB80004B239480225B0F902303FB2E21892FB0A
:107DC800F5F1B0F900208BB2B918344C91FBF5F2FB
:107DD80091B263802180438001802C4B0120204C8C
:107DE8001870184B61682A4A20681C7A5160106024
:107DF8001CB9DA79002A3FF4D9AC294E294D2A4C0E
:107E080001960095164F94E80C00FFF7BDF96168DC
:107E18007868264E081AF8F7B1FE1E4B1968F8F76D
:107E280001FFF9F7C5F870600A48226890F9003038
:107E38003C68012BC4EB020131603DD0022B7FF47A
:107E4800B5ACA0E0031F0020E21D0020F01E0020BA
:107E58003C110020B8100020980F00209A10002034
:107E6800D81E00201C110020806967FFAC1000207C
:107E7800F00F0020B4100020A810002000007A4461
:107E8800BC1E0020B81E0020C41E0020E8100020E0
:107E9800881000202800002054100020BA1000206C
:107EA800EC100020981000207010002034110020E1
:107EB80080969800F0100020002634463546DFF8FA
:107EC80018C3AF4F5CF825B0CDF80CC05846F8F78A
:107ED80055FE3968F8F7A6FEF9F76AF8DFF8DC927C
:107EE800A84934F80920DFF8DC82801A83B21FB26F
:107EF800635238460497A44FF8F740FE3968F8F7FC
:107F080091FEF9F755F84FF0140A0AFB058A82B278
:107F18009E4B0498196805923B4658445246FFF711
:107F28000BF90599DFF8B4B2DDF80CC00A1824F88B
:107F38000B205CF8250051463A46FFF789F9944929
:107F48004FF4FA62FBF7C4FF34F809303BF8042019
:107F5800313399B2622998BF0020801883B22BF878
:107F680004308C4940F6B83218B2FBF7B1FF58F824
:107F78000610894A01352BF80400B1500234143632
:107F8800022D9CD112E4854F2D683E686C08B6F925
:107F98000820A24228BF2246814C97B2268839B2CF
:107FA80030B2814209DD794B7E491868F8F73AFE0C
:107FB800F8F7FEFF8719BFB227807B4A7B4E14680B
:107FC8003168661A3046FFF77BF80028D8BF404270
:107FD80041F293139842CCBF0020012050B33046A1
:107FE800F8F7CCFD7249F8F71DFE04F08DFB064644
:107FF8002846F8F7BFFD01463046F8F713FEF8F7B4
:10800800D7FF6C4A6349108000B240F6B832FBF7DC
:108018005FFF201848F6A044A04203DDA0F50C40FD
:10802800A03804E00028BCBF00F50C40A03062492D
:10803800086001E0604D2C605F4B1D68C5F50C5071
:108048002830F8F79BFD5A49F8F7ECFD064604F08E
:10805800E7FA0990304604F057FB002508902C46B3
:108068002E4638B2F8F78AFD08AA52F82610F8F713
:10807800D9FD80465148DFF80C91005FF8F77EFD86
:1080880001464046F8F7C4FCF8F792FF4FF47A72BD
:1080980024F809004A4900B2FBF71AFF81B20BB273
:1080A800DFF83C8124F8091018460493F8F766FDB8
:1080B800D8F80010F8F7B6FDF8F77AFFDFF8D8A07F
:1080C8004FF0140B0BFB06AB049A30491FFA80FCE7
:1080D8000968434610465A46CDF80CC0FFF72CF8FD
:1080E80042460346594639F904000493FFF7B0F8AD
:1080F800049ADDF80C80801808EB000CDFF8DC80AF
:108108001FFA8CF124F8081008B240F6B832214959
:10811800FBF7DEFE55F80A202A4B013628F8040042
:10812800EA5002341435022E9BD11C480368197991
:1081380031B1214A64201468234A94FBF0F111807C
:10814800224C1B88206898420ED91749174B0A6899
:108158001C68101BFEF7B4FF42F210710028B8BF6C
:10816800404288427FF722AB194B1A4A01201C88EB
:10817800154910700C80FFF719BBFFF7BFF868E0CE
:1081880044100020EC0F0020FC0F0020A810002055
:1081980030F8FFFF48F4FFFFC010002060100020F7
:1081A8002C1100200000C842EC100020FC10002018
:1081B800D3023739281100206C100020BA10002093
:1081C80018FCFFFFC40F0020141E00209810002088
:1081D80068100020B810002034110020241100205D
:1081E8000C10002062686078531C411CCAB263609E
:1081F8000523B2FBF3F003FB10216170FDF71CFBB4
:10820800154AA06015480023C372137001200BE0C3
:10821800FDF712FBA36840F6C411C01A884218D9AA
:10822800202000F037F90420FEF77AFF11E00C490E
:108238008A78522A7FF446ABCB784D2B7FF442AB39
:10824800087943287FF43EAB064A02211170FFF7F4
:1082580039BB0BB0BDE8F08FF01E0020031F0020D3
:1082680078100020C00F00203D4B2DE9F047B3F9EE
:108278000000F8F783FC3B49F8F7D4FC044604F007
:1082880043FA0646204604F0CBF9DFF8EC900546A1
:10829800D9F80000344F90F80380B8F1000F2BD0C4
:1082A800324CB7F90210B4F802A00FFA8AF2881A11
:1082B800FEF706FFC8F100014246FBF709FEB4F8D5
:1082C800008000EB0A03B7F900000FFA88F7C01B1B
:1082D8006380FEF7F5FED9F80010CA785142FBF723
:1082E800F7FD00EB080297B22780B4F90200F8F70F
:1082F80045FC804638B206E0B7F90200F8F73EFCC4
:108308008046B7F90000F8F739FC29460746404689
:10831800F8F788FC314681463846F8F783FC014671
:108328004846F8F775FB1249F8F730FDF8F740FEB4
:10833800104C314620804046F8F774FC2946064622
:108348003846F8F76FFC01463046F8F763FB0849F2
:10835800F8F71CFDF8F72CFE6080BDE8F08700BF39
:10836800261E002035FA8E3C24110020A41000207F
:1083780000002041921000206010002038B5254CE4
:10838800E37A2246002B3ED02348017804293AD9C3
:108398002248817A79B1E179002939D12048214BE5
:1083A800012221721970011DE271FFF749F91E4976
:1083B8000220087038BDC37AE171C3B11B4A106846
:1083C800408900F075F890B1237A002B20D1154828
:1083D8001749037017480A684B680125011D026098
:1083E80043602572FFF72CF90F48057038BD0D481A
:1083F800084B02780021197252B901210170BDE8B9
:108408003840FFF705B80023D3711372064A13707A
:1084180038BD00BF031F0020F01E0020141F0020DD
:10842800BC1E00202C000020B81000206010002086
:10843800D81E0020B01E00200A4B1A68811A002995
:108448000EDB094A117804290AD900F5123000F523
:10845800F8721A60054B998A88B280F488429A8229
:10846800704700BFA0100020F01E00200010004838
:10847800034B196808420CBF00200120704700BF59
:108488000C120020024B1A6810431860704700BF96
:108498000C120020024B1A6822EA0000186070478C
:1084A8000C120020014B1868704700BF0C12002006
:1084B800094BB3F90020002AB8BF5242824209DAB8
:1084C800B3F902100029B8BF49428142ACBF00206D
:1084D80001207047002070472A1F002010B54478FB
:1084E8000078002303FB03F11939614301F6C41135
:1084F8005943414340F6C41291FBF2F1034A22F872
:1085080013100133072BEDD110BD00BF4A1F002007
:108518002DE9F04384780A276743C678C4F1640CD0
:108528001A4D5FFA8CFCC6F1640800231A1B12B2BC
:10853800002A04DCB8BF204602DB012000E06046C8
:1085480002FB02F9404309FB06F999FBF0F04044AD
:1085580042434FF00A0992FBF9F2B81882B26A80D6
:108568000888B1F8029012B2C0EB090902FB09F2BF
:108578000A334FF47A7992FBF9F29BB28018782B80
:1085880025F8020FD2D1BDE8F08300BF301F0020CC
:10859800014B1860704700BF28120020074B19686C
:1085A8000B7A032B09D8DFE803F00202040600F077
:1085B80001BB00F063B900F02BBA70472812002005
:1085C80008B5037A032B12D8DFE803F00202070C80
:1085D8000A490B4A00F0F6FA08E00849084A00F090
:1085E80055F903E00549064A00F01AFA28B90820A7
:1085F800FBF7B2FB02480022026008BD581F0020AA
:1086080024120020174B10B5186004460023608917
:10861800154A98520233242BF9D1144801600820D6
:10862800FBF71AFA10B12046FFF7CAFF4FF4803063
:10863800FBF712FA20B120460D490E4A00F0D2F895
:108648000120FBF709FA28B109480A49BDE810409A
:1086580000F0D4B84FF40040FBF7FEF90028F3D13E
:1086680010BD00BF281200205A1F00202012002031
:10867800581F002024120020037A032B09D8DFE8B2
:1086880003F00202040600F0D5BA00F02DB900F09C
:10869800E5B90020704700002DE9F84F80464FF4F7
:1086A80000708B46FBF7D8F920B1334B1868016886
:1086B8000A6990474FF40040FBF7CEF940B12F4CC0
:1086C800257805F10107FBB2237003F0030A05E0E2
:1086D8000120FBF7C1F90028F1D182460025284C7A
:1086E8004FEA4A0A2F462748026822B9B8F80A20F2
:1086F800254BEA5238E018F8079058464946904703
:1087080006464FF40070FBF7A7F930B11A490B6819
:1087180031461868C26948469047A6F2EE2188B2E9
:1087280040F2DC5398424FF4004088BFB8F80A6022
:10873800FBF792F930B90120FBF78EF910B912480E
:108748002E5211E024F80A6022886188A388501804
:10875800E288C11888180D4983B26B5218B20422F6
:10876800094990FBF2F36B52013702350834082FA0
:10877800B9D1BDE8F88F00BF201200202C120020CC
:108788002E120020241200205A1F00201012002050
:10879800F8B505460F46441E14F8011F49B1054EA9
:1087A800304606F0EBFD0028F6D0861B631BBB5550
:1087B800F2E7F8BDE80A0108014B33F811007047E9
:1087C8005A1F0020014B01221A7070476E120020B8
:1087D800034B187810B100221A700120704700BFAF
:1087E8006E1200200AB1024B13600120704700BFCF
:1087F800C18700080846F9F779BB0000024B0B60F7
:1088080008210170704700BFFD870008034B53F82B
:108818002100410801F5777290B270477812002064
:1088280038B50446FCF7EEFF104B40F6C4111A6841
:10883800821A8A421A460E4B01D9002119701B78F8
:1088480010600BB90F2C10D10A4800210170084A9A
:108858004BB1094D182B1D4405F8014C03D10123D8
:108868000370117038BD0133137038BD70120020C9
:10887800741200207512002098120020024B032168
:108888004360836041737047A086010073B500237D
:10889800044600930E4605230E49154608200E4A45
:1088A80000F052FF62890D4B0D49A2F57774640000
:1088B80008601C605C609C60DC601C615C619C61A1
:1088C800DC610DB10749296008220030327018BFF9
:1088D80001207CBD29880008A086010078120020AC
:1088E800B412002015880008254B10B51A780AB96B
:1088F800002010BD00201870224B997D0A07F7D47C
:1089080058781978204A00F0070441EA04211160D8
:10891800997801F03F04640144EAD0005060DC78A3
:10892800A00040EA9110197901F0010440EA84207E
:108938009060587900F00F04E40144EA5101D160D5
:10894800997901F07F04240144EA10101061DC7960
:10895800600040EAD111187A00F0030441EA44218A
:108968005161597A01F01F04A40144EA9000906112
:108978009B7AD80040EA5111D161012010BD00BF97
:10898800751200209812002078120020024B53F82C
:108998002100C0F3CF007047DC12002010B5044658
:1089A800FCF730FF154B1A68811AB1F57A6F1A4631
:1089B800134B01D9002119701060187820B9A82C20
:1089C8001AD1104B187006E0022802D10E4A147012
:1089D80001E0142801D80D490C540B490130C3B2E9
:1089E8000878074A4100481D8342137004D10023C8
:1089F8000449137001220A7010BD00BFB81200208C
:108A0800FC120020D1120020D8120020BC12002035
:108A18004FF4E133012143608360417370470000E4
:108A280037B5002300930D461446094908204FF432
:108A3800E132012300F088FE064908600CB1064ABD
:108A48002260082300302B7018BF01203EBD00BFF4
:108A5800A5890008D412002095890008124B10B58A
:108A68001A780AB9002010BD1049002018704B78F8
:108A7800012BF7D10E480278082A01D90821017084
:108A880001780C4A0023D8B2023288420AD212F87E
:108A9800010C12F8024C40EA0424074840F823402D
:108AA8000133F0E7012010BDD1120020BC120020D4
:108AB800D8120020BF120020DC120020114B012226
:108AC80010B51A700446FCF79DFE0F4A014610685F
:108AD80011600B1A0D4841F288318B4203600C4B30
:108AE80001D900221A7018780A49E4B20F280C54E8
:108AF80003D109490120087010BD054A431C1370B1
:108B080010BD00BF401300200013002008130020F0
:108B18000D130020431300200C1300201E4B2DE9D9
:108B2800F0411A781AB31D4C1D4D2678077895F830
:108B380000C002231B4A03F10108D45C44FA06F47E
:108B480004F00F04E5B2BD420BD20B2D09D8D55C59
:108B580012F8082005EA0C0502EB0525124A42F82E
:108B680024500233102BE5D10B4B00221A700078E9
:108B780088420ED90D4A107860B10D4B0A481A7810
:108B880050F8211002B1490801F5777398B2BDE891
:108B9800F0810020BDE8F0810C13002004130020B0
:108BA800421300204313002010130020401300201C
:108BB800411300204FF4E133012143608360417386
:108BC8007047000013B5037A14465BB1012B13D12B
:108BD800124A03201070124A0720107011480370BF
:108BE8000C2308E00D4A022010700D4A0320107073
:108BF8000C48037007230B70002100914FF4E132F9
:108C080008200949012300F09FFD084A10600CB1B3
:108C1800074B2360003018BF01201CBD041300203F
:108C28004213002041130020C58A00085413002075
:108C3800258B0008014B1878704700BF0C130020E3
:108C4800014B1860704700BF5C130020034B186885
:108C58000178D1F1010038BF002070475C13002073
:108C6800034B186801784A1E534253EB02007047C1
:108C78005C13002008B54FF40060FAF7EDFE20B150
:108C88000420BDE8084000F017BD08BD084B18785F
:108C980060B108490A68537813B1074A117D01E0A9
:108CA80006484178081C18BF01207047012070470A
:108CB800581300205C130020141F0020031F0020FD
:108CC80008B5FFF7C3FF18B1BDE8084000F062BA65
:108CD800FFF7C6FF18B1BDE8084000F09DBB08BD0E
:108CE80008B5FFF7B3FF08B100F094F8FFF7B8FF35
:108CF80018B1BDE8084000F07FBA08BD0F4B10B5A9
:108D08001878D0B1FFF7C2FF0D4904460A788242AD
:108D180013D070B1FFF79AFF18B10A4B186800F02A
:108D280091F8FFF79DFF30B10648006800F07CFA23
:108D380001E0FFF7D5FF02490C7010BD6013002059
:108D4800591300205C13002008B50121042000F00D
:108D5800BFFC054B1870FFF78DFF04490870BDE88C
:108D68000840FFF7CBBF00BF581300206013002056
:108D780008B5094B187870B1FFF788FF58B1FFF7AD
:108D880065FF08B100F0A0F8FFF76AFF18B1BDE869
:108D9800084000F07DBA08BD6013002038B5064CC5
:108DA80005465E212068FCF7DFFC20682946BDE8FF
:108DB8003840FCF7D9BC00BF74130020024B5E2179
:108DC8001868FCF7D1BC00BF7413002010B50A4C1A
:108DD8005E280146206805D15D21FCF7C5FC2068A6
:108DE8003E2105E05D2903D1FCF7BEFC20683D214A
:108DF800BDE81040FCF7B8BC7413002010B5044659
:108E0800C0B2FFF7E3FFC4F30720BDE81040FFF747
:108E1800DDBF000010B5084B084C19782068FCF736
:108E2800C7FC074920680968FCF7B8FC20680421DA
:108E3800BDE8104000F0AABB6C130020741300209A
:108E48006413002037B50546042000F06FFB154C6D
:108E580001462060A0B14279134B81681A70134A09
:108E680011604FF41651FCF799FC20680221FCF7B9
:108E78009FFC2068042103B0BDE8304000F074BBBB
:108E8800AB784FF4165200930420022300F05CFCE8
:108E9800054942792060054B80680A70186003B064
:108EA80030BD00BF741300206C1300206413002031
:108EB80008B5044B1868FCF767FCD0F1010038BF0F
:108EC800002008BD741300202DE9F041FFF7F0FFE2
:108ED800002800F04081FCF7AFFCA04B1A68811A0B
:108EE8007C2940F2388118609D480478651C05701B
:108EF800002404F12406F0B2FFF750FF994B33F930
:108F08001400F7F73BFE984A05461088F7F736FE37
:108F180001462846F7F73AFF9449F7F783FEF8F732
:108F280047F8013400B2FFF769FF032CE1D1302084
:108F3800FFF734FF8E49B1F90000FFF75FFFFFF735
:108F48003DFF8748067816F0030629D1894D102081
:108F5800FFF724FF2B68642493FBF4F210B2FFF7A9
:108F68004DFF2120FFF71AFF296891FBF4F004FB5D
:108F7800101484EAE473A3EBE47318B2FFF73EFF1E
:108F88001420FFF70BFF7C4AB2F90000FFF736FF09
:108F98001C20FFF703FF3046FFF730FFFFF70EFFF7
:108FA8006F490878430740F0B080744D0220FFF7FE
:108FB800F5FEB5F900300A2593FBF5F0FFF71EFF23
:108FC8000220FAF749FD002847D06D4F6D4E3878DA
:108FD800347840F63401B4FBF0F26B4C4A432188F4
:108FE8002A2391FBF0F800FB1810B2FBF3F24FEACA
:108FF800001399B241EA022C1FFA8CFEC2F3032235
:109008004EEA02080620FFF7C9FE0FFA88F0FFF7BC
:10901800F5FE20883F78431C9AB292FBF7F107FBD4
:109028001120367820806E247443152394FBF3F4C2
:109038003A206427FFF7B2FEB4FBF7F63046FFF795
:10904800DDFE3B20FFF7AAFE07FB164291B24C1D3E
:1090580094FBF5F000B2FFF7D1FE2020FFF708FAE5
:10906800002850D0494C1320FFF798FE2568484F38
:10907800002DB8BF6D4295FBF7F630B2FFF7BEFE84
:109088001B20FFF78BFE23680A26002BB8BF5B4224
:1090980093FBF6F142F2107591FBF5F205FB121005
:1090A80000B2FFF7ABFE2320FFF778FE2368002B02
:1090B800ACBF4E205320FFF7A1FE1220FFF76EFE33
:1090C80061680029B8BF494291FBF7F210B2FFF777
:1090D80095FE1A20FFF762FE60680028B8BF40427C
:1090E80090FBF6F696FBF5F305FB136108B2FFF764
:1090F80085FE2220FFF752FE6268002AACBF452099
:109108005720FFF77BFEFFF759FE15480378282BF9
:1091180021D100240470FCF78FFB4FF47A753C24AE
:10912800B0FBF5F61720FFF739FEB6FBF4F5B5FBF3
:10913800F4F104FB1152100200B2FFF75FFE182091
:10914800FFF72CFE04FB156318B2FFF757FEBDE8C6
:10915800F041FFF733BEBDE8F08100BF7013002077
:1091680068130020501E00200400002000007A44EC
:10917800700E0020980D0020261E0020E01D002003
:1091880002000020501900206A130020D81E002079
:10919800A08601004FF4165070470000154B2DE9CA
:1091A800F04180460F4618680221FCF701FB0024B5
:1091B8002646781E84420F4D0DDA18F804102868E8
:1091C8008E190134FCF7D0FA4FF47A70B6B2FCF776
:1091D80039FBE4B2EDE7F1B22868FCF7C5FA4FF4C1
:1091E8007A70FCF72FFB28680121BDE8F041FCF7F5
:1091F800DFBA00BFA813002010B5084B084C197837
:109208002068FCF7D5FA074920680968FCF7C6FA10
:1092180020680421BDE8104000F0B8B9DA13002036
:10922800A8130020A413002013B5042000F07EF931
:10923800144C01462060A0B14279134B81681A7022
:10924800124A11604FF49641FCF7A8FA20680121F0
:10925800FCF7AEFA2068042102B0BDE8104000F027
:1092680083B900904FF496420123042000F06CFA71
:10927800054B42792060054980681A70086002B081
:1092880010BD00BFA8130020DA130020A41300208B
:10929800F8B5544C2068FCF777FA002800F0A08055
:1092A8002068FCF776FA05460520FCF7D6FA8A2DE1
:1092B80021D08E2DEDD14C4C00212E22204605F0D8
:1092C80005FA4A4A7C2323701378E0207D21E07058
:1092D80084F82C1014204FF4FA71A37723754822D0
:1092E80078232076607661836570628484F8243000
:1092F80020462E2171E02020FFF7BAF80028C8D0B8
:109308003B4C00212C22204605F0E0F9A021E17019
:10931800384B39497C207D22207084F82B2018781E
:10932800CA7A6570A076002A52D0344934480F684A
:109338006625FE0F97FBF0FC6672324E5FFA8CFCD6
:1093480006FB0C7284F8295006256A4342F2107312
:10935800B2FBF3FE03FB1E274968277391FBF0F06D
:109368003F0AC0B26773CF0F06FB00116943B1FB18
:10937800F3F5642203FB1513E9B202FB0010010A9E
:10938800E0732148217401885FFA8EFE63741B0A1A
:1093980002FB0CECA374B1FBF2F224235A4390B203
:1093A8001A4A010A1388E0712172180A18492075AF
:1093B80018480A8801884FEA1C2EE374130A84F8B7
:1093C8000AC084F80BE0A7736275A375217702E0E1
:1093D800202384F8293006482C21FFF7DFFE58E7C0
:1093E800F8BD00BFA8130020AC13002050190020BE
:1093F80078130020F01E0020031F0020D81E002034
:10940800A08601006079FEFFAE1E0020B81E002075
:10941800AA1E0020C41E00204FF49640704700008A
:1094280010B500230C245C430549DAB2615C814223
:1094380003D00133042BF5D11A46104610BD00BFE6
:10944800300000202DE9F84F0C2283460D462248B3
:109458000421224B05F0D0F900260C2373431E4A41
:1094680002EB030898F808101BEA010F2DD0D05C16
:1094780000241B4F2201BB5CBA46834203D001344F
:10948800E4B2042CF5D14FEA041940200AEB09078D
:10949800FAF7E2FA20B91AF80910881E012814D937
:1094A8006B7B13B13A7B13420FD0696878688142AD
:1094B8000BD3AA68BB689A4207D80A480470876029
:1094C800C0F80480C560BDE8F88F0136042EC4D109
:1094D8000020BDE8F88F00BF30000020F19400089C
:1094E800FC0A0108DC130020037A002023B15A1E6D
:1094F80001301340C0B2F9E70A7A22B1511E013394
:109508000A40DBB2F9E7984294BF00200120704777
:1095180000230549DAB2595C814203D00133092B93
:10952800F7D11A4610467047F10A010800220D4B80
:109538000C2101FB0233197A814211D00132D2B2D7
:10954800042AF4D10022074B0C2101FB0233197ABB
:10955800014005D10132D2B2042AF4D1084670473D
:10956800586870473000002010B50023064A0C24C4
:1095780004FB03225468844203D00133042BF5D141
:109588000022517210BD00BF300000200023074A9E
:109598000C2101FB03225168814203D00133042BC3
:1095A800F5D1002200205072704700BF3000002023
:1095B80038B5002205461A4811014318405CA842F4
:1095C80004D00132062AF6D1002038BD154C042DEE
:1095D8000FCB84E80F0016D007D8012D0DD0022D2F
:1095E8001BD111490B6898680AE0082D11D0202D6D
:1095F80013D10D490B68D86802E00B48026850681F
:109608006060A06003E0FFF75BFB6060A06020463D
:1096180038BD2046FEF7C2FFF9E7024838BD00BF53
:109628003C0B0108EC1300200C140020214B10B552
:1096380018600120FFF7BCFF01460120FFF702FF79
:1096480008B9002010BD0220FFF7B2FF0146022032
:10965800FFF7F8FE0028F4D01020FFF7A9FF014615
:109668001020FFF7EFFE04464FF48070FAF7F4F984
:1096780008B1002CE5D00820FFF79AFF0146082022
:10968800FFF7E0FE04460820FAF7E6F908B1002CD7
:10969800D7D00420FFF78CFF01460420FFF7D2FE45
:1096A80004464FF40060FAF7D7F908B1002CC8D087
:1096B800012010BD0C14002010B50446FFF778FFF8
:1096C80001462046FFF7BEFE003018BF012010BD3E
:1096D80038B505460C46FFF76BFF01462846FFF7ED
:1096E800B1FE28B14368187A04420CBF002001205B
:1096F80038BD0000F8B505460020FFF791FE104E72
:109708000C272B780F4C07FB0060E15C01720120ED
:10971800FFF786FE07FB00626878235C022013725D
:10972800FFF77EFEAA7807FB0061A05C08720320A1
:10973800FFF776FEEB7807FB0061E25C0A72F8BD82
:1097480030000020F10A01082DE9FF478146039205
:109758000C461E469DF83070FFF72AFF0146484622
:10976800FFF770FE039A054600282ED0836890F80C
:1097780000A093F80080B8F1030F26D8DFE808F0BE
:1097880002050D0F0097134801E013480097214682
:109798003346F8F7E1FB04460AE0002000E0012028
:1097A80021463B46F8F7A6FE31460446FCF700F88A
:1097B8005CB184F80480696808484C6040F82A4025
:1097C80049462046FFF7D0FE00E00024204604B0BA
:1097D800BDE8F0870038014000440040FC13002039
:1097E80038B5064C05462060FFF784FF284600F090
:1097F800FFFF2068BDE8384000F0E0BE0C140020F0
:10980800034B187808B100F0E1BD01F07BB800BF48
:109818001014002010B504462046FBF7C4FF18B901
:109828000A20FCF71AF8F7E710BD0000232801D139
:1098380000F0CCBD044B19680A7D824202D1012098
:10984800FCF732B9704700BF0C14002010B5441E55
:1098580014F8011F21B1034B1868FBF785FFF7E7E0
:1098680010BD00BF481400200148FFF7EFBF00BF3C
:10987800240D010810B50748FFF7E8FF0024064B40
:1098880006481A19E15852680C34FAF74BFCC02CF8
:10989800F5D110BD620D0108400C0108780D0108D2
:1098A80070B5FBF7C9FF244C244B4FF47A71B0FB19
:1098B800F1F11A7822482378FAF734FCFEF7F2FD22
:1098C80005462048204902682048B2FBF1F1FAF722
:1098D80029FC00241E4B53F8241051B1012000FA32
:1098E80004F0284202D01B48FAF71CFC0134E4B209
:1098F800F0E70220FEF7BCFD68B1174A174B117854
:10990800174853F82110FAF70DFC1648017A11B1DF
:109918001548FAF707FC154C1548FFF797FF2488F8
:10992800F7F7D0FE0246134821464FF46C73BDE8A2
:109938007040FAF7F7BB00BF020000205019002062
:10994800800D01086C01002040420F00BE0D010887
:10995800C01B0108DC0D0108880D0020000D01085E
:10996800E00D0108F01D0020EA0D0108600D00203F
:1099780050100108EE0D010838B50C680546204660
:1099880005F0D8FD024628682146BDE8384005F0B4
:1099980001BE000037B5037904460D46052B34D8BF
:1099A800DFE803F003060A0D1114816809782DE039
:1099B800806890F9001029E08368198826E0826899
:1099C800B2F9001022E0816809681FE080686946E2
:1099D8000068FAF78DFC01461148FAF7A3FBF5B1C8
:1099E800E068F7F7CBF86946FAF782FC01460D48BC
:1099F800FAF798FB2069F7F7C1F86946FAF778FC97
:109A080001460848FAF78EFB09E000210648FAF7F4
:109A180089FB25B10548E1682269FAF783FB3EBD59
:109A2800E70D0108E60D0108240E0108200E0108C3
:109A380008B50648FFF70AFF054B1868FFF7EAFE66
:109A48000020BDE80840FCF72FB800BF270E01082A
:109A58004814002008B50748FFF7F8FE064B93F8AE
:109A6800AC03F9F79BFFF9F7A9FFBDE80840FFF73A
:109A7800DFBF00BF360E0108541900207FB5044629
:109A880005F058FD082825D100231F49E25C086825
:109A980085186E7806F00301022908BF203AE254BF
:109AA8000133082BF1D10025665D1848314605F0D1
:109AB80065FC28B101356019314605F05FFC18B125
:109AC8001348FFF7C3FE1DE0082DEDD120461149CC
:109AD800FEF75EFE1048FFF7B9FE00230F4A04A9FF
:109AE800981890F808218818084A995C0133082BBF
:109AF80000F80C1CF2D100208DF80C0001A90848D0
:109B0800FAF710FB7FBD00BFA4010020E80A010896
:109B1800400E01085C1A0020600E0108541900204C
:109B28007B0D010808B5FDF735FD022801D0032893
:109B380004D10348BDE80840FFF788BE08BD00BF50
:109B4800750E01082DE9F041054605F0F3FC0446C1
:109B5800FAF7B8F9064694B92A48FFF777FE2A4972
:109B680051F8241049B1012202FA04F2324202D01B
:109B78002648FAF7D7FA0134F1E7254821E02846C4
:109B88002449224605F006FD58B92348FFF75EFE32
:109B9800224C54F8041F0029EFD01C48FAF7C2FAE7
:109BA800F7E72B782D2B04D10135013C4FF0010844
:109BB80001E04FF000080026134850F8267027B936
:109BC8001748BDE8F041FFF741BE2846394622460E
:109BD80005F0E0FCA0B9012000FA06F0B8F1000F8A
:109BE80003D0FAF7B9F80F4802E0F9F73FFF0E483B
:109BF800FFF72CFE0D483946BDE8F041FAF792BA56
:109C08000136D9E79B0E01089C0B0108DC0D010801
:109C180050100108A7190108AE0E0108980B010899
:109C2800C30E0108DD0E0108E70E01087B0D0108CF
:109C380010B504460848FFF709FE084A08480949CC
:109C48000023036013700B70FCF7F4FD2046BDE899
:109C58001040FFF7FFBE00BFF00E010811140020EE
:109C6800441400201014002008B50448FFF7EEFD46
:109C7800F9F704FFBDE80840FFF7DABE080F01084E
:109C88002DE9F04389B0044605F054FCC6B2002E15
:109C98006AD17A48FFF7DAFD794C20690021F7F795
:109CA80055F938BB013677483146FAF73BFA20694F
:109CB80004A9FAF71DFB01467348FAF733FA6069FD
:109CC80004A9FAF715FB01466F48FAF72BFAA069C1
:109CD80004A9FAF70DFB01466B48FAF723FAE06985
:109CE80004A9FAF705FB01466848FAF71BFA10348D
:109CF8000C2ED2D10025664C2F46A8464FF00009FD
:109D08001034B14514DA404654F8101CF6F782FEB8
:109D180054F80C1C80462846F6F77CFE54F8081CBC
:109D280005463846F6F776FE09F101090746E7E7E2
:109D38005848CDF8048002950397FFF787FD002463
:109D480001A82358544923F00040F7F727F953494D
:109D5800534A0434002814BF10460846FFF776FD1E
:109D68000C2CEDD14F4871E020464F49052205F0F3
:109D780011FC38B9424B0022C1181030C0280A61C2
:109D8800F8D177E020464949042205F003FC05464E
:109D980020460DBB202105F0F1FA00286AD0461CA8
:109DA800304605F0C7FB2C460746414850F824507A
:109DB8000DB940484AE030462946FAB205F0EAFBB8
:109DC80040B920463C49FCF7D1FD3C482946FAF702
:109DD800A9F947E00134E8E704F078FB461E0B2EAA
:109DE800074643DC2046202105F0C8FA054640B165
:109DF800451C2846FAF7E4FA214B3F01D8510124C3
:109E080000E004462846202105F0B8FA054640B18E
:109E1800451C2846FAF7D4FA1949013401EB061211
:109E280050612846202105F0A9FA054640B1451C95
:109E38002846FAF7C5FA124B013403EB061188617C
:109E48002846202105F09AFA18B91D48FFF7FEFCAC
:109E580010E00130FAF7B4FA094A032C02EB0616AF
:109E6800F061F2D11748FFF70BFF03E016480C2109
:109E7800FAF758F909B0BDE8F08300BF290F0108C7
:109E880054190020540F01085A0F01087B0D0108CE
:109E9800681900205E0F01080AD7233C250F010826
:109EA800210F0108501001086D0F0108730F0108F8
:109EB800E40B0108780F010864190020900F0108CD
:109EC800A30F01088F120108DD0F0108F8B5074636
:109ED80005F030FB044638B91A491B4B4A791B4830
:109EE800511E53F8211028E038461949224605F03A
:109EF80051FB60B91748FFF7A9FC174C54F8041F29
:109F080019B11648FAF70EF9F8E7154805E00025E3
:109F18000D4B53F8256026B91248BDE8F840FFF705
:109F280095BC38463146224605F034FB01350028F9
:109F3800EED10448314645710B48BDE8F840FAF7C0
:109F4800F1B800BF54190020E40B010805100108FE
:109F5800A719010819100108E00B0108DC0D010818
:109F680050100108780F01082C1001082DE9F0475E
:109F7800064605F0DFFA054620B1012819D13378E5
:109F88002A2B16D14748FFF761FC002414266643A4
:109F9800454F4648F159FAF7C5F8B8192946FFF769
:109FA800F9FC01344248FFF751FC722CEED1BDE8B0
:109FB800F08730463D2105F0E1F9002857D0441CD0
:109FC800204604F083FA82462046FAF7F9F900277A
:109FD800054614247C43DFF8D09054F809804046A5
:109FE80005F0A8FA41460246304605F0D3FA0028A3
:109FF80035D14C44E068F6F7C1FD01462846F6F72E
:10A00800C3FF002829D02069F6F7B8FD0146284685
:10A01800F6F7B0FF002820D020792279052818BF4C
:10A028005546052A0FD8DFE802F003030606090C97
:10A03800A1680D7007E0A268158004E0A0680560BB
:10A0480001E0A1680D6041461A48FAF76BF820460E
:10A058000021BDE8F047FFF79DBC174803E0013732
:10A06800722FB6D11548BDE8F047FFF7EFBB04469D
:10A07800142565430C4F314655F80780404605F0D6
:10A088005BFD50B109484146FAF74CF878190021B0
:10A09800FFF780FC0648FAF745F80134722CE7D13F
:10A0A800BDE8F0873E100108E01B010818120108FE
:10A0B80050100108531001085E10010883100108B0
:10A0C80010B50446204605F035FA10F0FF0F07D109
:10A0D8000B490C4891F8AC13BDE81040FAF722B8C8
:10A0E800204604F0F3F9022808D8054B064C83F8FB
:10A0F800AC03F9F763FCF9F7A1FEE3E710BD00BF75
:10A1080054190020A01001088F12010870B50446E8
:10A1180005F010FA08B9204830E020461F4905F03C
:10A1280081FE00242646254678B12CB1012C06D1A3
:10A1380004F0CCF9064602E004F0C8F90546002010
:10A148001649013405F06EFEEEE70B2D05D91448CB
:10A158000C21BDE87040F9F7E5BF012C08DC114A75
:10A16800114832F915202946BDE87040F9F7DABFE1
:10A17800A6F57A73B3F57A7F04D90C48BDE8704028
:10A18800F9F7D0BF0A4829463246F9F7CBFF054808
:10A1980020F8156070BD00BFB610010859120108FB
:10A1A800F0100108801E0020161101082E11010868
:10A1B8005011010838B5054605F0BCF9C0B268B9B8
:10A1C80004461249124801EB4402B2F846202146DF
:10A1D8000134F9F7A7FF152CF3D138BD284604F050
:10A1E80075F9142804460BDC2021284605F0C6F82A
:10A1F80004F06CF9054B03EB4404A4F8460038BDA1
:10A2080004481521BDE83840F9F78CBF081D002027
:10A2180069110108751101082DE9F043584885B006
:10A22800584CF9F77FFF5848FFF7C4FF6279574B3E
:10A23800511E574853F82110F9F774FF206900217F
:10A24800F6F784FE002858D10025266900213046FB
:10A25800F6F77CFE00284CD101354E482946D4F843
:10A268001490D4F81880E769F9F75CFF30460021AC
:10A27800F6F776FE10B14848F9F754FF69463046BC
:10A28800FAF736F801464548F9F74CFF48460021E9
:10A29800F6F766FE10B14048F9F744FF69464846AC
:10A2A800FAF726F801463D48F9F73CFF40460021F9
:10A2B800F6F756FE10B13848F9F734FF69464046BC
:10A2C800FAF716F801463548F9F72CFF3846002109
:10A2D800F6F746FE10B13048F9F724FF69463846CC
:10A2E800FAF706F801462E48F9F71CFF10340C2D32
:10A2F800ABD12C48691CF9F715FFF9F7E3FD2A4C97
:10A30800064654F8041F19B12848F9F70BFFF8E777
:10A318000D46274850F8251049B1012202FA05F2E6
:10A32800324202D02348F9F7FDFE0135F1E7154B1B
:10A33800214ACE1896F808418B5C04A8013105190A
:10A34800082905F8103CF2D100241C4869468DF80C
:10A358000840F9F7E7FE14256543194E1948A9592D
:10A36800F9F7E0FE00217019FFF714FB01341648D5
:10A37800FFF76CFA722CEED105B0BDE8F08300BF90
:10A388009B110108541900208F120108E40B0108E1
:10A39800CB110108D611010859120108E70D01086F
:10A3A8007B0D0108DE110108980B0108F011010866
:10A3B8009C0B0108FE110108E80A01080B120108AC
:10A3C800E01B01081412010850100108F0B56D4B8C
:10A3D80087B01A787AB96C4C01201870022120686D
:10A3E800FFF7C2F82068F9F7C7FE6848FFF72EFAAA
:10A3F8006748FFF72BFA644C2068FBF7C5F900287B
:10A4080000F0BD802068FBF7C4F909280146614ABD
:10A4180001D03F2851D1002517685F4C2E462FB137
:10A428005E4821683A4605F0B5F810B9254606B9E0
:10A4380026465B490C348C42F1D3C6B13468D5F852
:10A4480000E03B46E05C1EF8031081420DD1534A00
:10A4580041B92D2B06D820244E48D454013303602B
:10A46800D15404E0D0540133ECE74A490B60494A1F
:10A4780014681CB1AE4201D13C4612E04948FFF7CE
:10A48800E5F9AE4209D856F80C0BFFF7DFF93E4B59
:10A4980009211868FBF768F9F3E73D48FFF7D6F993
:10A4A80000243C4B18688442A5D237493B4A0868C7
:10A4B800115DFBF759F90134F3E713682BB9042848
:10A4C80038D13648FFF7B4FB59E00C2801D136489B
:10A4D8008CE70A2901D00D2948D12E4D3348FFF7C2
:10A4E800B5F92E4C2A6832480023A35404930090EF
:10A4F800294903A810220C23039403F0EBFF054617
:10A5080038B1006805F016F8411CAA686018904731
:10A5180002E02848FFF79AF9002130221F4804F08A
:10A52800D5F818491B4B0A7800201860002A7FF4D8
:10A538005FAF24E00C28CAD07F2903D15BE72F2B1B
:10A548003FF659AF1F297FF656AF7E293FF653AF26
:10A5580013B920293FF44FAF104C581CE1540A4A54
:10A568000C4B18601068FBF7FFF844E77F29E6D129
:10A578000A4C581E0021106021540F4839E707B0D3
:10A58800F0BD00BF10140020481400201E1201085E
:10A598005612010844140020400C01081114002030
:10A5A800000D01085B120108601201085010010833
:10A5B800819900086B1201088C12010837B505460D
:10A5C8000220FEF7B3FF064C0146206030B9009028
:10A5D800AA6802200323FFF7B7F820603EBD00BF3A
:10A5E80048140020F8B5174E174C184D0746C1B24D
:10A5F80030682170FBF7B8F822782B78C7F3072169
:10A6080082EA0300287030682170FBF7ADF82178E2
:10A618002A78306881EA0203C7F307412B7021705A
:10A62800FBF7A2F82078297880EA0102390E306811
:10A6380021702A70FBF798F82B78207880EA0301BC
:10A648002970F8BD54140020501400204C14002028
:10A65800F8B50D4E0D4D0E4CC1B207463068297045
:10A66800FBF782F82A782378391282EA03002070EF
:10A6780029703068C9B2FBF777F823782A7882EA1C
:10A6880003002070F8BD00BF5414002059140020A6
:10A698004C140020054B10B5044621461868FBF7FA
:10A6A80063F8034802785440047010BD5414002025
:10A6B8004C140020034B04491A78885C01321A7044
:10A6C800704700BF4D1400207114002010B5FFF72B
:10A6D800F1FF0446FFF7EEFF04EB002080B210BD47
:10A6E80010B5FFF7F3FF0446FFF7F0FF04EB004057
:10A6F80010BD000038B5044624200D46FFF7CAFFF8
:10A708004D20FFF7C7FF002C0CBF3E202120FFF78C
:10A71800C1FF064B002228461A70FFF7BBFF04480A
:10A728000078BDE83840FFF7B5BF00BF4C140020E3
:10A738005A14002001460020FFF7DCBF0146012023
:10A74800FFF7D8BF014B1878FFF7A4BF4C140020BF
:10A7580070B5054608460E46FFF7ECFF2C46721901
:10A76800D0B2E3B2984204D014F8010BFFF792FF7D
:10A77800F5E770BD10B5441E14F8010F10B1FFF7CE
:10A7880089FFF9E710BD00002DE9F84300270124EF
:10A798000025144B187885421CDA1349134B15F819
:10A7A80001800C2202FB0830406804F0C3FE814699
:10A7B8000CB13F180CE026464E4509DA0B4A0C212D
:10A7C80001FB08235868805DFFF764FF0136F3E753
:10A7D8000135DEE724B1F8B2FFF7ACFF0024D7E774
:10A7E800BDE8F8834E1400205B14002060000020B0
:10A7F800F7B5404DFF2115220746284603F066FFAE
:10A80800002302202B70FDF733FE012418B102202B
:10A818006C70A87003240420FDF72AFE68B1354E39
:10A8280003214FF400503155651CF9F715F918B19B
:10A8380004227255023400E02C460220FDF718FE6F
:10A8480048B12C4B05201E19062107251855717093
:10A85800B570033404E00820FDF70AFE0028F0D1A3
:10A868002020F9F7F9F818B1224B08221A550134BB
:10A878004FF48070F9F7F0F830B11E480A26011934
:10A888000B2506554D7002341B4A1A4B507908287F
:10A8980001D00E2802D10C261E5501340D210420AA
:10A8A8001955651CF9F7D8F818B112481122425504
:10A8B800A51C1149132391F839210E4E6C1C101C4C
:10A8C80018BF01207355F9F7C7F810B11420305597
:10A8D800AC1C0A4B01201C70FEF728FE084C0146F0
:10A8E800206030B900907A6801200323FEF72CFF1E
:10A8F8002060FEBD5B140020541900204E14002077
:10A9080054140020F8B5B54C2068FAF73DFF00282C
:10A9180000F02F852068FAF73CFFB14A034611780A
:10A9280071B9B0F124014B4253EB01041470002CAF
:10A93800E9D1AC4A51780029E5D1FEF777FFE2E783
:10A94800012904D14D280CBF0223002321E002294C
:10A9580004D13C280CBF032300231AE003290FD19C
:10A9680040284FF0000401D91470CCE79E489F4955
:10A9780003709F480C7004709E4C2370042308E0F9
:10A98800042908D19B4C9C48217803704B402370C4
:10A9980005231370B7E70529B5D19448924C01787F
:10A9A80022788A42934A07D914785C401470934AF3
:10A9B800535401310170A6E71078984240F0D484CE
:10A9C8008D4B19787B2900F01B8300F2C5806E2916
:10A9D80000F0658360D8682900F02E8325D86529A2
:10A9E80000F0028219D8642940F0B9840720844C09
:10A9F800FFF7A0FEE620FFF74DFE6079FFF74AFE5D
:10AA08000020FFF747FE94F819017E4B7E4A002884
:10AA18000CBF1046184600F055BC662900F062824B
:10AA2800672940F09C84794807E36B2900F0158377
:10AA380023D8692900F005836A2940F09084102002
:10AA4800FFF778FE6748724CC07AFFF723FE71491A
:10AA58000878FFF71FFE2068FFF7C4FD6068FFF75E
:10AA6800C1FD6D4AB2F90000FFF7F2FD6B4BB3F977
:10AA78000000FFF7EDFD6A4A0EE36C2900F0FF8243
:10AA88006D2940F06C840620FFF754FE654908687C
:10AA9800FFF7A8FD644AFFE2732900F06D833CD8F4
:10AAA800702900F02B83C0F00B83712900F03983E3
:10AAB800722940F05484524C1620FFF73BFE0020C8
:10AAC800FFF7C6FDB4F9D000FFF7C2FD574DB4F942
:10AAD800D200FFF7BDFDB4F9D400FFF7B9FDB5F911
:10AAE800BA00FFF7B5FD0020FFF7B2FD0020FFF721
:10AAF80079FDB5F928000A2390FBF3F0FFF7A8FDCC
:10AB080094F80401FFF7C6FD94F80601FFF7C2FDAB
:10AB180094F80501FFF7BEFD5DE3762900F0378361
:10AB28000DD8742900F01583752940F018842F205A
:10AB3800FFF700FE3E48FFF71DFE00F013BC772923
:10AB480000F00A83782940F00A84384C3820FFF74F
:10AB5800F1FD04F1400503E2D02900F0718300F211
:10AB6800C680CA2900F0018168D8A42900F0D683DC
:10AB780010D8A02940F0F3832E4C0C20FFF7DAFD03
:10AB88002068FFF72FFD4FF080510868FFF72AFD76
:10AB9800206897E3C82900F0DA80C92940F0DF83EC
:10ABA800FFF788FD0F4A1A4CD072FFF783FD194B47
:10ABB8001870FFF795FD2060FFF792FD6060FFF7C2
:10ABC80085FD15490880FFF781FD144A10801A4851
:10ABD800037843F002040470D6E000BF5414002048
:10ABE8004F140020031F0020581400207014002068
:10ABF8004D1400204C1400205A1400207114002019
:10AC0800541900201C000080140000801800002047
:10AC1800D81E0020F01E0020AA1E0020AE1E002014
:10AC2800F8100020481E0020700E0020081D00208B
:10AC3800C8240108030000102E110020CD2900F0BF
:10AC4800098322D8CB2900F0A180CC2940F0878342
:10AC5800FFF730FDCC4CE077FFF72CFD84F820009F
:10AC6800FFF728FD84F82300FFF724FD84F824006B
:10AC7800FFF720FD84F82500FFF71CFD84F821006C
:10AC8800FFF718FD84F822007EE0CE2900F0EC8260
:10AC9800CF2940F06483FFF719FDFFF717FDBB4C80
:10ACA800B94DA4F8D000FFF711FDA4F8D200FFF7C2
:10ACB8000DFDA4F8D400FFF709FDA5F8BA00FFF7C9
:10ACC80005FDFFF70DFDFFF701FD0A22504328851A
:10ACD800FFF7F0FC84F80401FFF7ECFC84F80601A8
:10ACE800FFF7E8FC84F80501FFF7E4FC4CE0D52900
:10ACF80000F094810FD8D22961D0C0F07082D32996
:10AD08006DD0D42940F02B839F4C0020FFF712FD13
:10AD180004F1400556E1F02900F0C7820CD8D62985
:10AD280044D0EF2940F01B83FFF7D0FC964CA08558
:10AD3800FFF7CCFC608527E0FA2900F09D82FE2908
:10AD480040F00D830820FFF7F5FC0024A5E200245D
:10AD5800FFF7BCFC8E4908530234102CF8D10020B0
:10AD6800FFF7E8FCFDF72EFDFCE28A4C04F10A052A
:10AD7800FFF7A0FC01346070FFF79CFCE072FFF75E
:10AD880099FCAC426075F3D1002083E2002482482C
:10AD980003789C42F8D2814D655DFFF797FC7A49AC
:10ADA800013401EB4505A5F84600F0E70024FFF75C
:10ADB8008DFC7B4908530234102CF8D1E4E7794C18
:10ADC8006478002CE0D1FFF775FC704B022883F8FB
:10ADD800AC0388BF83F8AC43F8F7F0FD37E2FFF720
:10ADE80075FC714A1080CFE7704D0B20FFF7A2FC6D
:10ADF800B5F90000FFF72CFCF6F764FC00B2FFF78A
:10AE080027FC0220FDF734FB05460420FDF730FB44
:10AE180004460820FDF72CFB820042EA440129433E
:10AE280020208CB2FDF724FB44EAC00084B2102035
:10AE3800FDF71EFB44EA001318B2FFF709FC594A54
:10AE48001079D17884005378907944EA4101194304
:10AE580041EAC0045179537A44EA411040EA831424
:10AE68005348C17944EAC113047A417A43EA042376
:10AE780043EA4124D379117A44EA8324927A44EA52
:10AE8800C123417B43EA0234827B44EA4133017C9B
:10AE980043EA8234027944EA0143417C43EA0214DA
:10AEA800827C44EA4143C17C43EA8244007D44EA0F
:10AEB800C142394B42EA00540020197803468B42BC
:10AEC8000AD2364D01225D5D02FA05F525421CBF06
:10AED8009A4010430133F2E72C4CFFF783FB94F8B8
:10AEE800AC0379E11220FFF725FC32490C88B4F550
:10AEF800806F314CB4F9000008D8FFF7A9FBB4F90A
:10AF08000200FFF7A5FBB4F904000EE0082590FB4A
:10AF1800F5F0FFF79DFBB4F9020090FBF5F0FFF7A1
:10AF280097FBB4F9043093FBF5F0244CFFF790FB42
:10AF3800B4F90000FFF78CFBB4F90200FFF788FBB7
:10AF4800B4F904001E4CFFF783FBB4F90000FFF7C7
:10AF58007FFBB4F90200FFF77BFBB4F90400AEE114
:10AF6800B4F97800FFF774FBB4F97A00FFF770FBC7
:10AF7800B4F97C00FFF76CFB94F87E000834FFF707
:10AF880089FBAC42ECD1EDE1081D002054190020EA
:10AF98005A1F0020071D00204E1400205B140020BB
:10AFA800801E0020031F0020141E0020600D0020BA
:10AFB800141F002004000020501E0020940E0020C2
:10AFC800FC1D0020FFF782FBA4F87800FFF77EFB4A
:10AFD800A4F87A00FFF77AFBA0F57A73072899B2EC
:10AFE80098BF84F87F00B1F57A7F98BFA4F87C00F9
:10AFF800FFF760FB84F87E000834AC42E2D1B1E18F
:10B008000820FFF797FB0024B049621892F87F00E8
:10B018000834FFF73FFB402CF6D1A3E10020FFF7EF
:10B0280089FB0024FFF746FBA84962180834402C26
:10B0380082F87F00F6D195E1A5481021FFF788FB3B
:10B0480090E11020FFF776FB0024A248005F02344D
:10B05800FFF7FEFA102CF8D184E10520FFF76AFB10
:10B068009D4BB3F90000FFF7F3FA9C48B0F90000D4
:10B07800FFF7EEFA9A490A7802F00100ACE0994C21
:10B088000620FFF757FBB4F90000FFF7E1FAB4F91F
:10B098000200FFF7DDFA944AB2F900000FE1072039
:10B0A800FFF748FB91480078FFF7F4FA0020FFF714
:10B0B800CFFA8F4BB3F90000FFF7CAFA0020FEE081
:10B0C800824C0720FFF736FBE07FFFF7E3FA94F89E
:10B0D8002000FFF7DFFA94F82300FFF7DBFA94F873
:10B0E8002400FFF7D7FA94F82500FFF7D3FA94F86D
:10B0F8002100FFF7CFFA94F822006DE01E20FFF739
:10B1080019FB7C4C04F10A0501346078FFF7C2FA98
:10B11800E07AFFF7BFFA607DFFF7BCFAAC42F3D1E3
:10B1280020E175490A78540004F0FE00FFF702FB9D
:10B138000024714803789C4280F014816F49634869
:10B14800625C013400EB4203B3F94600FFF780FA72
:10B15800EFE7FFF719FB05E1674900240878FFF7D7
:10B16800E9FA654A1078844280F0FC80634B185DE8
:10B17800FFF790FA0134F4E70820FFF7DBFA01241F
:10B18800E0B20134FFF786FA092CF9D1EAE0FFF7BB
:10B1980091FA06461220FFF7CDFA0EB9584902E097
:10B1A800102E03D157490D684C6801E0002425464C
:10B1B8003046FFF76FFA2846FFF714FA2046FFF7E4
:10B1C80011FA514A1068FFF70DFA0020FFF740FA0C
:10B1D8000020FFF73DFA0020FFF75CFAC2E0FFF716
:10B1E80069FA0546FFF77CFA0746FFF779FA06463B
:10B1F800FFF776FA0446FFF769FAFFF767FAFFF7F1
:10B2080059FA65B93E48414B012107604660DD7136
:10B218001973002C3FF4B8AD3B4A1460B4E5102D07
:10B228007FF4B2AD3748076046600CB1364B1C60FE
:10B23800374A344802211170011DFCF701FAA3E5D1
:10B2480032484378002B7FF49FADF8F717FCF8F7E6
:10B25800F5FD99E52D4C6278002A7FF495AD4FF401
:10B26800C870FAF701F88FE528484378002B7FF477
:10B278008BAD0121817387E5244A5478002C6ED167
:10B28800244B93F8AC03F8F789FBF8F797FBF8F72A
:10B29800D5FD2046FFF74EFA64E01F48005F0234F0
:10B2A800FFF7D6F9082CF8D15CE0084C0420FFF72A
:10B2B80041FAB4F92C00FFF7CBF9B4F92A00FFF7EB
:10B2C800C7F94FE0FFF78EF94CE000BF081D0020DA
:10B2D800681E00205A1F0020B81E0020C41E00202F
:10B2E8002E110020A00E0020261E0020501900203C
:10B2F800EA1D0020071D00204E1400205B140020CA
:10B30800BC1E0020B01E00204C1E0020031F002081
:10B31800B810002054190020E21D0020154C227896
:10B328009000431CD8B2FFF705FA2078FFF7B2F96E
:10B33800002410490A78944214D20F48005DFFF7A0
:10B34800A9F90E4B185DFFF7A5F90D49085DFFF740
:10B35800A1F90C4A105DFFF79DF90134E9E70020D7
:10B36800FFF7ECF9FFF7EEF9074B00201870FFF72D
:10B37800CABAF8BDF11E0020981E0020C61E002083
:10B38800E01E0020F21E00204F1400202DE9F0419D
:10B398000746884616460024B4421AD00025BD4206
:10B3A80011D00D4B01359A8AEDB290B280F48851D4
:10B3B80099820120FAF70CFA4046FAF74EFA002073
:10B3C800FAF706FAEBE73C200134FAF746FAE4B25A
:10B3D800E2E7BDE8F08100BF00100048F0B50023A7
:10B3E8000E681A46012505FA02F505EA0604AC427C
:10B3F80032D10D796F1E012F1BD84FF0030C0CFAB8
:10B4080003FC876827EA0C0791F805C087600CFAE7
:10B4180003FC87684CEA070787608788BFB227EA7A
:10B42800040484808C79878804FA02F43C43A7B228
:10B438008780032404FA03F405FA03F50768E44354
:10B448002740076007683D430560C5682C40CD79F3
:10B4580005FA03F52C43C46001320233102AC1D126
:10B46800F0BD00214FF6FF730222036001714271A3
:10B478008171C1717047816170470185704701F022
:10B48800070330B59B000F2404FA03F402FA03F211
:10B49800C908083150F8215025EA040440F8214031
:10B4A80050F82140144340F8214030BD124B1A682F
:10B4B80042F0010018605968104A0A405A6018683A
:10B4C80020F0847121F480321A60186820F48021F9
:10B4D80019605A6822F4FE005860D96A21F00F02F8
:10B4E800DA62186B06490022014019639A60054B1D
:10B4F8004FF0006098607047001002400CC07FF861
:10B50800CCFC00FF00ED00E082B00023254800934A
:10B518000193026842F480310160224B186800F4FC
:10B52800003201920099481C0090019A1AB90099BA
:10B53800B1F5A04FF1D11B6813F4003018BF0120FA
:10B548000190019A012A2AD1174B12211960A3F5FB
:10B5580080504268426041684160436843F48062B9
:10B568004260416821F47C134360426842F4E81168
:10B578004160036843F0807202600168094A8901EA
:10B58800FBD5506820F003035360516841F0020076
:10B598005060044A536803F00C010829F9D102B03D
:10B5A800704700BF0010024000200240A44B2DE964
:10B5B800F0435A6802F00C02042A05D0082A06D083
:10B5C800A0490160B2B916E09E4C046012E05D68C3
:10B5D8005C68C5F38346B71CE20301D49A4A06E0C7
:10B5E800DB6A984D03F00F02511CB5FBF1F27A4368
:10B5F800026000E00022924F944D7E68C6F3031368
:10B60800EC5C036823FA04F141607E68C6F3022605
:10B61800AE5D21FA06F68660D7F804C0CCF3C228DE
:10B6280015F80850DFF828C221FA05F1C160D7F8EB
:10B638002C90C9F3041808F00F093CF819C018F049
:10B64800100F1FFA8CFC07D0BCF1000F04D0B2FB1E
:10B65800FCF8C0F8108000E00361FF6AC7F3442CCF
:10B668007B4F0CF00F0837F818701CF0100FBFB2A2
:10B6780004D01FB1B2FBF7F7476100E04361704F98
:10B68800D7F830C01CF0100F0ABFDFF8B8C18361CB
:10B69800C0F818C03F6BBF0656BF6A4FC361C76189
:10B6A800674FD7F830C01CF0400F0ABFDFF894C1CD
:10B6B8000362C0F820C03F6BFF0506D5934204D152
:10B6C800A54202D15F00476200E041625C4FD7F8B3
:10B6D80030C01CF4805F08D0934206D1A54204D143
:10B6E8004FEA430CC0F828C000E081623F6BBF05F9
:10B6F80006D5934204D1A54202D15F00C76200E09B
:10B70800C1624F4FD7F830C01CF4806F08D0934205
:10B7180006D1A54204D14FEA430CC0F844C000E06A
:10B7280041643F6B3F0506D5934204D1A54202D13F
:10B738005F00876400E08164414FD7F830C01CF493
:10B74800005F06D0934204D1A54202D15A00C264D8
:10B7580000E081643C6B3A4A14F0030F01D10163A5
:10B7680015E0116B01F00301012901D103630EE01B
:10B77800116B01F00301022902D14FF4004205E0E8
:10B78800126B02F00301032901D12E4A02632C4AED
:10B79800116B11F4403F01D1466318E0116B01F4BD
:10B7A8004031B1F5803F01D1436310E0116B01F4E2
:10B7B8004031B1F5003F02D14FF4004106E0116B72
:10B7C80001F44031B1F5403F01D11E494163126B8C
:10B7D8001B4912F4402F01D1866318E00A6B02F46A
:10B7E8004022B2F5802F01D1836310E00A6B02F486
:10B7F8004022B2F5002F02D14FF4004106E0096B58
:10B8080001F44022B2F5402F01D10E4981630C4A60
:10B81800116B11F4401F01D1C66323E0116B01F4D1
:10B828004011B1F5801F01D1C3631BE0116B01F416
:10B838004011B1F5001F0DD14FF4004111E000BFD8
:10B848000010024000127A0000093D00900100201B
:10B8580070010020116B01F44011B1F5401F01D1B6
:10B868001149C163126B114912F4400F02D10664E9
:10B87800BDE8F0830A6B02F44002B2F5800F0FD0E6
:10B888000B6B03F44002B2F5000F02D14FF40043F2
:10B8980006E0096B01F44003B3F5400F01D1024BF8
:10B8A8000364BDE8F08300BF00127A000010024074
:10B8B800030F064BDA6A14BF22F4785222F4F872A6
:10B8C800DA62D96A0843D862704700BF00100240A4
:10B8D800020F012A0A4B0AD005D3022A0BD1196B91
:10B8E80021F0400206E0196B21F0100202E01A6B09
:10B8F80022F020021A63196B08431863704700BFCF
:10B9080000100240044B5A6909B1104301E022EAD1
:10B9180000005861704700BF00100240044B9A694C
:10B9280009B1104301E022EA00009861704700BFA6
:10B9380000100240044BDA6909B1104301E022EA21
:10B948000000D861704700BF00100240044BDA685D
:10B9580009B1104301E022EA0000D860704700BF37
:10B9680000100240044B1A6909B1104301E022EAB1
:10B9780000001861704700BF00100240024B5A6A6D
:10B9880042F08070586270470010024008B5154BAD
:10B9980098420BD101214FF48050FFF7D7FF4FF4A5
:10B9A80080500021BDE80840FFF7D0BF0E4988420B
:10B9B80007D14FF480400121FFF7D4FF4FF48040B6
:10B9C80009E00A4A90420BD14FF400400121FFF7E9
:10B9D800C9FF4FF400400021BDE80840FFF7C2BF8F
:10B9E80008BD00BF0030014000380040003C004066
:10B9F8004A8830B5B2F5827F1BD10488CB8804F41D
:10BA080041520C881C4344F482730C8923434C89AB
:10BA180023438C892343CC8923431A4393B203805D
:10BA2800828822F470631A04130C8A881343838073
:10BA380019E0838823F4706425048C882B0C234335
:10BA480083800B8805881343CA8805F441540D89FF
:10BA580013434A892B438D891343CA892B431343C4
:10BA680023439AB20280838B098A23F40062130469
:10BA78001A0C8283018230BD038819B199B241F052
:10BA8800400303E023F040010A04130C03807047CD
:10BA9800838823F4805213041A0C828083889AB214
:10BAA8001143818070470173704781817047007B23
:10BAB8007047808980B27047038919420CBF002003
:10BAC80001207047C2680D4B10B5134091E814006F
:10BAD80014438A681443CA6814430A6914434A69B8
:10BAE80014438A6922431343C360026B097F22F01F
:10BAF8000F024B1E1343036310BD00BF07C0FFFDB9
:10BB080000230121036043608360C36003614361D4
:10BB18008361017770470000B0F1A04F10B502D0E3
:10BB2800114B984201D1114A00E0114A9468114B17
:10BB3800B0F1A04F03EA040391E8140044EA0204B8
:10BB48008A6844EA0204CA68097C44EA023242EA82
:10BB5800012242EA030302D00349884201D1034883
:10BB680000E00348836010BD00010050000300504E
:10BB780000070050E010FCFF00230360436083606F
:10BB8800C36003747047836811B143F0010101E099
:10BB980043F0020181607047836843F0004181608F
:10BBA8007047836823F0804282608368194381600C
:10BBB80070478068C00F7047836823F040528260E6
:10BBC800836811B143F0805101E043F00051816076
:10BBD8007047042A70B54FF006040BD862431F243F
:10BBE80004FA02F401FA02F2056B25EA040414438C
:10BBF800046329E0092A0CD862431F241E3A04FA78
:10BC080002F401FA02F2456B25EA04041443446382
:10BC18001AE00E2A0CD862431F243C3A04FA02F4B4
:10BC280001FA02F2856B25EA0404144384630BE0ED
:10BC380062431F245A3A04FA02F401FA02F2C56B6D
:10BC480025EA04041443C46309294FF003020FD9F9
:10BC58004A4307211E3A01FA02F103FA02F3846902
:10BC6800846924EA0104846184692343836170BD83
:10BC780044694C1E5443382606FA04F4514303FA27
:10BC880001F3456925EA0404446144692343436197
:10BC980070BD836843F0040181607047C36811B1C7
:10BCA80043F0010101E023F00101C1607047C3685E
:10BCB80023F00202C260C3681943C1607047036879
:10BCC80019420CBF00200120704730B5046A41F0CA
:10BCD800010124F0010505628569046A25F0F30570
:10BCE8002A4342EA031324F00A0241EA0204836168
:10BCF800046230BD30B5056A4FF6EF742C4004621B
:10BD08008469090124F47344056A44EA022242EA78
:10BD180003334FF65F7441F010022C4091B20C438C
:10BD28008361046230BD0000204A038890429BB2C0
:10BD38000ED002F5006290420AD0B0F1804F07D0D1
:10BD4800A2F59832904203D002F58062904203D166
:10BD58004A8823F070031343154A904208D002F52D
:10BD68008062904204D023F440730A899BB2134343
:10BD780003804B680A88C3620C4B028598420FD037
:10BD880003F5006290420BD002F54063984207D059
:10BD980003F58062904203D002F58063984201D196
:10BDA8004989018601224261704700BF002C014089
:10BDB8000010004000214FF0FF33436001800181F3
:10BDC80041804181704741627047038819B199B237
:10BDD80041F0010303E023F001010A04130C03807E
:10BDE80070470000036A30B523F001020262036A5B
:10BDF8004268856923F0020325F4803424F0730532
:10BE08000C682C438D892B438D882B43134DA842F6
:10BE18000FD005F50065A8420BD005F54065A8428E
:10BE280007D005F58065A84203D005F58065A842CE
:10BE38000DD1CD8923F008032B43CD8823F00403CB
:10BE48002B430D8A22F440722A434D8A2A4389687B
:10BE5800426084614163036230BD00BF002C014031
:10BE6800036A70B523F010020262056A42688469A9
:10BE780025F0200524F080760C6826F4E64343EA92
:10BE880004248E898B88334345EA03130E4DA84258
:10BE980003D005F50065A84210D123F08006CB89B0
:10BEA80022F4406246EA0315CB8825F0400646EAAC
:10BEB80003134D8A0E8A354342EA85028968426037
:10BEC80084618163036270BD002C0140036A70B510
:10BED80023F480720262056A4268C4690B6824F020
:10BEE800730646EA03048E898B8825F4007533436C
:10BEF80045EA03230E4DA84203D005F50065A84284
:10BF080010D123F40066CB8922F4405246EA032577
:10BF1800CB8825F4806646EA03234D8A0E8A35438A
:10BF280042EA051289684260C461C163036270BD58
:10BF3800002C0140036A70B523F480520262056A3E
:10BF48004368C4690A6824F4E64646EA02228C88F3
:10BF58008E8925F40055344345EA0434084DA84237
:10BF680003D005F50065A84204D10D8A23F4804367
:10BF780043EA851389684360C2610164046270BD45
:10BF8800002C0140002303608380C3808360838189
:10BF9800C381038243827047836923F008021143F7
:10BFA80081617047836923F4006242EA012181615B
:10BFB8007047C36923F008021143C1617047C36920
:10BFC80023F4006242EA0121C16170470023012283
:10BFD800038043808280C38003817047406B704731
:10BFE800806B7047C06B7047006C7047836923F0A3
:10BFF8000C0282618369194381617047836923F464
:10C0080040628261836943EA012181617047C269A4
:10C018004FF6F3731340C361C2691143C16170479E
:10C02800C2694FF2FF331340C361C26909028BB280
:10C038001A43C2617047F8B50B880D460446498813
:10C04800AA8843B92B89FFF740FEE9882046BDE856
:10C05800F840FFF7CBBF042B08D12B89FFF74AFE26
:10C06800E9882046BDE8F840FFF7C8BF082BB5F8B7
:10C0780008C0066A1BD14FF6FF6737400762C369DD
:10C088004FF60C77066A1F404FF2FF53334042EADF
:10C098000C1243EA012141F480731743E988BFB2C7
:10C0A8009AB2C7610262BDE8F840FFF7B0BF4EF62A
:10C0B800FF7737400762C36940F6FF46076A1202F6
:10C0C8001E4045F6FF733B4042EA0C3C1FFA8CF2D7
:10C0D80043EA0131164341F48052E98893B2C661BC
:10C0E8000362BDE8F840FFF79BBF436C11B143F40E
:10C0F800004201E059044A0C42647047C3680AB11F
:10C10800194302E0C94389B21940C1607047036905
:10C11800C26811EA030003D011420CBF00200120BD
:10C128007047C9438AB2026170470000C37810B5EE
:10C1380003B3164CE168CB43C3F302244178C4F13E
:10C14800040201FA02F10F2222FA04F28478037839
:10C1580022400A43110103F16043CAB203F5614169
:10C1680081F800230078012200F01F03410902FA38
:10C1780003F007E00078012200F01F03410902FAEA
:10C1880003F02031024B43F8210010BD00ED00E020
:10C1980000E100E0036830B5044623F001002060A8
:10C1A80062680D46AB6822F4405141EA03006060C2
:10C1B8002268EB6822F4B0516A6821F00C0043EA67
:10C1C80002012B6995B041EA030202432260A0688C
:10C1D8006B6920F4407141EA03026846A260FFF7E8
:10C1E800E5F91848844201D10C9A0EE016498C42B0
:10C1F80001D10D9A09E0154B9C4201D10E9A04E039
:10C20800134884420CBF0F9A109A2168286811F4C9
:10C21800004F18BF5200B2FBF0F300FB13212A684D
:10C228002068B1EB520F28BF0133020406D54FF640
:10C23800F072C3F342011A4041EA020398B2A081A6
:10C2480015B030BD003801400044004000480040AF
:10C25800004C0040036811B143F0010101E023F0F4
:10C26800010101607047C905CA0D028570478368DE
:10C278000AB1194301E023EA010181607047C1F363
:10C28800072310B5C9B20124022B04FA01F101D128
:10C29800043002E0032B08BF0830036812B143EAF8
:10C2A800010201E023EA0102026010BD090C01232A
:10C2B80003FA01F202627047044B1A69120604D5A8
:10C2C800034800F1883158605960704700200240E7
:10C2D80023016745024B1A6942F0800018617047D4
:10C2E80000200240014BD860704700BF0020024088
:10C2F800084BDA68D20709D4D868C00608D4D968C8
:10C3080011F0040F0CBF0420032070470120704770
:10C31800022070470020024010B50446FFF7E8FFEE
:10C32800012806D11CB1FFF7E3FF013CF8E705201F
:10C3380010BD002C08BF052010BD000073B50023F8
:10C3480006464FF430200D460193FFF7E5FF042819
:10C3580019D10D4CAAB2206940F0010121614FF4B6
:10C3680030203280FFF7D8FF042808D10236019622
:10C37800019B2D0C1D804FF43020FFF7CDFF216964
:10C3880021F0010222617CBD0020024038B505463B
:10C398004FF43020FFF7C0FF042811D1094C23695E
:10C3A80043F002002061656121694FF4302041F0BB
:10C3B80040022261FFF7B0FF236923F002012161E7
:10C3C80038BD00BF00200240036823F0010202606C
:10C3D8000268144B13408A6843EA02234A681343ED
:10C3E8000A68036022F070630361026842F0010387
:10C3F8000022036082608B69C2600A691A43826006
:10C40800836843F400428260CB68026849691A4332
:10C418000260436823F0784222F400430B434360F0
:10C42800704700BFFFE0CF0000234FF400420360D5
:10C4380043608360C360036142618361704703683E
:10C4480011B143F0010101E023F0010101607047DF
:10C4580030B54568064C890543EA91532C40039949
:10C468001C4344EA010343EA0242426030BD00BF74
:10C47800009800FC81627047406AC0B270478369C7
:10C4880019420CBF002001207047C16170470000AD
:10C4980002684FF6FE73134003602D4B002198424B
:10C4A800016041608160C16022D02A49884229D058
:10C4B800294B984230D02949884237D0284B984296
:10C4C8003ED0284B984206D153F8681C41F47000BE
:10C4D80043F8680C70472449884206D151F87C0C0F
:10C4E80040F0706241F87C2C7047204B984206D18E
:10C4F80053F8042C42F00F0143F8041C70471C4900
:10C50800884206D151F8183C43F0F00041F8180C65
:10C518007047184B984206D153F82C2C42F470619E
:10C5280043F82C1C70471449884206D151F8403C06
:10C5380043F4704041F8400C7047104B984205D1C5
:10C5480053F8542C42F4702143F8541C704700BF30
:10C55800080002401C000240300002404400024033
:10C56800580002406C00024080000240080402406B
:10C578001C040240300402404404024058040240B3
:10C5880070B506688C680D6A26F4FF4222F07006C2
:10C598000A6945EA04034C6913438A692343CC6951
:10C5A80013431C434B6A44EA03028B6A1A4332431F
:10C5B80002608B890A68496843608260C16070BD07
:10C5C8000023036043608360838103614361836167
:10C5D800C361036243628362704719B1016841F025
:10C5E800010303E002684FF6FE73134003607047CF
:10C5F80041607047406880B2704703680AB11943C8
:10C6080001E023EA0101016070470000C3004CBF4C
:10C61800014B024B58607047000402400000024082
:10C6280000B540F6D87320F00042C3F649739A4229
:10C6380083B0014615DDB2F1FF4F03DBF4F7E8F9EB
:10C6480003B000BD694600F095FB00F00302012A23
:10C65800009801990ED0022A07D082B900F0A0FDF7
:10C66800EEE7002100F09CFDEAE700F099FD00F1FB
:10C678000040E5E701F040FC00F10040E0E701225E
:10C6880001F03AFCDCE700BF30B5C0F3C754A4F1B1
:10C698007F031E2B83B0014621DC581C1DDBCD0F08
:10C6A800162B0CDD21F07F4323F4000040F400003A
:10C6B800963C00FA04F005B1404203B030BD114881
:10C6C80050F825402046F4F7A5F901902146019835
:10C6D800F4F79EF920F0004121B90020EDE7F4F7C6
:10C6E80067FCEAE720F07F4222F40003C0F3C7505A
:10C6F80043F40001C0F1960221FA02F0002DDCD0CB
:10C70800DAE700BFA825010800B540F6D87320F085
:10C718000042C3F649739A4283B0014616DDB2F16E
:10C72800FF4F03DBF4F774F903B000BD694600F06E
:10C7380021FB00F00300012815D002280BD0B8B95E
:10C7480000980199012201F0D7FBEDE700210022B2
:10C7580001F0D2FBE8E700980199012201F0CCFB37
:10C7680000F10040E0E70098019900F019FDDBE7CF
:10C778000098019900F014FD00F10040D4E700BFD3
:10C7880070B58AB0064600F09BF8224C054694F92D
:10C798000030013303D0304601F0B0FD10B928460F
:10C7A8000AB070BD304601F05BFD4FF07E51F4F7E2
:10C7B800F5FB0028F3D0184A0121002530460192E4
:10C7C80000910895F3F76AFE02460B461348CDE937
:10C7D8000423CDE9022301F011FC94F90030CDE9DE
:10C7E8000601022B0BD0684601F006FC38B1089808
:10C7F80050B9DDE90601F4F7B7F80546CFE701F0CF
:10C8080089FE21210160F2E701F084FE089A0260A6
:10C81800EFE700BFA0010020B0250108B8250108F6
:10C8280000F002BA70B58AB0054600F04FFC224C01
:10C83800064694F90030013308D0284601F05EFD21
:10C8480020B128460021F4F78BFB10B930460AB016
:10C8580070BD1A4A012128460026009101920896C7
:10C86800F3F71CFE2478CDE90401CDE902017CB977
:10C8780000220023CDE90623684601F0BDFB88B1FC
:10C888000898A0B9DDE90601F4F76EF80646DDE779
:10C898000020002102460B46F3F77EFF022CCDE96B
:10C8A8000601E9D101F036FE21230360E8E701F033
:10C8B80031FE08990160E5E7A0010020BC250108C8
:10C8C800F8B520F00043B3F17E5F044613D00BDCCB
:10C8D800B3F17C5F14DAB3F10C5F00F3A48040F687
:10C8E800DB70C3F6C970F8BD0146F4F791F801464C
:10C8F800F4F74CFAF8BD002840F30E810020F8BD8B
:10C908000028C0F20E8101464FF07E50F4F780F8FF
:10C918004FF07C51F4F786F9044600F0D7FB4EF649
:10C928000871064620F47F65C3F611012046F4F726
:10C9380079F947F60471C3F64F21F4F76BF82146ED
:10C94800F4F770F941F24611C3F62451F4F760F890
:10C958002146F4F767F940F6A821C3F64E61F4F7CB
:10C9680059F82146F4F75EF94BF29001C3F6A66137
:10C97800F4F74EF82146F4F755F94AF6AB21C3F619
:10C988002A61F4F747F82146F4F74CF94CF22E6186
:10C998000746C3F69D512046F4F744F943F2613146
:10C9A800C3F63071F4F734F82146F4F73BF945F251
:10C9B8002D71C4F20101F4F72DF82146F4F732F98C
:10C9C8004DF23911C4F21901F4F722F82146F4F7AF
:10C9D80029F94FF07E51F4F71DF801463846F4F76F
:10C9E800D5F93146F4F71EF925F00F050746294613
:10C9F8002846F4F717F901462046F4F709F82946BE
:10CA080004463046F4F706F801462046F4F7BEF926
:10CA180001463846F3F7FEFF2946F3F7FBFF0146C8
:10CA2800F3F7F8FFF8BD0146F4F7FCF84EF6087185
:10CA3800C3F611010546F4F7F5F847F60471C3F695
:10CA48004F21F3F7E7FF2946F4F7ECF841F24611D6
:10CA5800C3F62451F3F7DCFF2946F4F7E3F840F670
:10CA6800A821C3F64E61F3F7D5FF2946F4F7DAF8A3
:10CA78004BF29001C3F6A661F3F7CAFF2946F4F713
:10CA8800D1F84AF6AB21C3F62A61F3F7C3FF29466A
:10CA9800F4F7C8F84CF22E610646C3F69D512846B5
:10CAA800F4F7C0F843F26131C3F63071F3F7B0FF21
:10CAB8002946F4F7B7F845F22D71C4F20101F3F7EE
:10CAC800A9FF2946F4F7AEF84DF23911C4F219015D
:10CAD800F3F79EFF2946F4F7A5F84FF07E51F3F7D8
:10CAE80099FF01463046F4F751F901462046F4F71C
:10CAF80099F8014642F26810C3F2A230F3F788FFB2
:10CB080001462046F3F784FF014640F6DA70C3F683
:10CB1800C970F3F77DFFF8BD40F6DB70C4F2490039
:10CB2800F8BD4FF07E51F3F775FF4FF07C51F4F7E5
:10CB380079F84EF60871C3F611010446F4F772F855
:10CB480047F60471C3F64F21F3F764FF2146F4F763
:10CB580069F841F24611C3F62451F3F759FF21460B
:10CB6800F4F760F840F6A821C3F64E61F3F752FFD8
:10CB78002146F4F757F84BF29001C3F6A661F3F794
:10CB880047FF2146F4F74EF84AF6AB21C3F62A616F
:10CB9800F3F740FF2146F4F745F80646204600F033
:10CBA80095FA4CF22E610546C3F69D512046F4F7DE
:10CBB80039F843F26131C3F63071F3F729FF2146A2
:10CBC800F4F730F845F22D71C4F20101F3F722FFB2
:10CBD8002146F4F727F84DF23911C4F21901F3F799
:10CBE80017FF2146F4F71EF84FF07E51F3F712FFB6
:10CBF80001463046F4F7CAF82946F4F713F842F22A
:10CC08006811C3F2A231F3F703FF01462846F3F790
:10CC180001FF0146F3F7FEFE014640F6DA70C4F262
:10CC28004900F3F7F5FEF8BDF8B521F00044B4F17A
:10CC3800FF4F034617DC20F00045B5F1FF4F0646CD
:10CC480011DCB1F17E5F42D08F1707F0020040EA95
:10CC5800D37775B9022F35D0032F08D140F6DB738F
:10CC6800CCF2490303E01846F3F7D4FE034618460E
:10CC7800F8BDD4B1B4F1FF4F2DD0B5F1FF4F14D0AA
:10CC88002C1BE4153C2C18DC002952DB1846F4F761
:10CC98007DF801F0E5FA01F0B7F9012F46D0022F2F
:10CCA80035D0002F25D10346E1E7002E40F6DB738F
:10CCB8001CDBC3F6C9731846F8BD40F6DB70C3F633
:10CCC800C970EAE740F6DB73C4F24903CFE7BDE871
:10CCD800F84001F099B9B5F1FF4F2FD0022FF1D0EC
:10CCE800032FBBD0012F34D00023C0E7CBF6C97384
:10CCF800BDE74BF62E51C3F2BB31F3F78BFE40F67E
:10CD0800DB71C4F24901F3F783FE0346AFE74BF644
:10CD18002E51C3F2BB31F3F77DFE014640F6DB70BE
:10CD2800C4F24900F3F774FE0346A0E700F100439C
:10CD38009DE714F13C0FA9DA0020AEE7022F13D0CB
:10CD4800032F0CD0012F40F6DB7305D0C3F64973CF
:10CD58008DE74FF000438AE7CBF6497387E74CF637
:10CD6800E433CCF2160382E74CF6E433C4F216033C
:10CD78007DE700BF2DE9F04F40F6D87320F000445E
:10CD8800C3F649739C4289B006460D4640F38B8032
:10CD98004CF6E331C4F216018C4226DC4FF478617C
:10CDA8000028C3F6C97140F32B81F3F731FE4FF425
:10CDB8007D6224F00F04C3F6C9729442064600F05F
:10CDC800818044F24341C3F23571F3F721FE0146F5
:10CDD80028603046F3F71CFE44F24341C3F2357134
:10CDE800F3F716FE0127686061E04FF47867C4F234
:10CDF8004937BC4240F38180B4F1FF4F5BDA4FEA18
:10CE0800E459A9F18609A4EBC9542046F4F7D0F8EF
:10CE1800F3F7B4FE0246014620460592F3F7F8FD03
:10CE28004FF08741F3F7FEFE0746F4F7C1F8F3F732
:10CE3800A5FE0146044638460694F3F7E9FD4FF08F
:10CE48008741F3F7EFFE00210790F4F77FF80028F9
:10CE580000F0F6800327204600210DF11808013F55
:10CE6800F4F774F840B158F8044D00212046013F0A
:10CE7800F4F76CF80028F6D1924B02200090019349
:10CE880005A83B4629464A4600F066FA002E0746A2
:10CE98000DDA95E80C0002F1004103F10042296027
:10CEA8006A60474203E00023286000274B60384649
:10CEB80009B0BDE8F08F0146F3F7AAFD00276860C6
:10CEC8002860F4E74FF48841C3F23571F3F7A0FD09
:10CED8004AF20831C2F685610446F3F799FD014626
:10CEE80028602046F3F794FD4AF20831C2F68561BE
:10CEF800F3F78EFD01276860D9E701F0B1F94FF625
:10CF08008411C3F622718046F3F78CFE4FF07C51F2
:10CF1800F3F780FDF4F74CF80746F3F72FFE4FF4CC
:10CF28007861C3F6C9718346F3F77CFE0146404633
:10CF3800F3F76EFD44F243418146C3F2357158461A
:10CF4800F3F770FE1F2F8246514648461FDC5E4BA2
:10CF58007A1E53F8223024F0FF029A4217D0F3F7D2
:10CF680057FD8046C5F8008041464846F3F750FD16
:10CF78005146F3F74DFD002E686098DA08F1004835
:10CF880000F10041C5F8008069607F428FE7F3F740
:10CF98003FFDE3158046C0F3C750191A0829E1DDA3
:10CFA8004FF48841C3F2357158460393F3F73AFEBC
:10CFB800824651464846F3F72BFD0446214648462B
:10CFC800F3F726FD5146F3F723FD4AF2083181466F
:10CFD800C2F685615846F3F725FE4946F3F718FD72
:10CFE800824651462046F3F713FD039BC0F3C75210
:10CFF8008046981A192841DCC5F80080A146B3E795
:10D00800F3F708FD4FF47D6724F00F04C3F6C977E2
:10D01800BC42064616D044F24341C3F23571F3F7D9
:10D02800F9FC014628603046F3F7F2FC44F243412C
:10D03800C3F23571F3F7EEFC4FF0FF37686036E75F
:10D04800032719E74FF48841C3F23571F3F7E2FC7F
:10D058004AF20831C2F685610446F3F7DBFC014663
:10D0680028602046F3F7D4FC4AF20831C2F68561FD
:10D07800F3F7D0FC4FF0FF37686018E74FF423410F
:10D08800C2F685615846F3F7CDFD804641462046F5
:10D09800F3F7BEFC814649462046F3F7B9FC414602
:10D0A800F3F7B6FC43F232110446C2F28D415846FA
:10D0B800F3F7B8FD2146F3F7ABFC824651464846E4
:10D0C8004DE700BF44260108C425010820F00042AE
:10D0D800B2F1FF4FF8B50446034646D2002A42D0C3
:10D0E800002852DBC415B2F5000F09D210F4000570
:10D0F80053D15B0001351902FBD5C5F10100241895
:10D1080023F07F417F3C21F40006E20746F400004B
:10D1180048BF400043004FF08072002760109A42D9
:10D128003C462CDD5B004FF400021825A618510878
:10D138009E4205F1FF3502DCB4189B1BBF185B004B
:10D1480062189A4202DC9B1A54187F185B004A083E
:10D15800013DEBD113B107F001017F187C1004F1F8
:10D168007C5303EBC0542046F8BD0146F3F75AFD43
:10D1780001462046F3F74EFC04462046F8BD4FF022
:10D18800007403F17F431746CCE70146F3F740FCF0
:10D198000146F3F7FBFD0446E5E70120AFE700BFD2
:10D1A8002DE9F84320F00046B6F1485F05460F46E2
:10D1B8005BDAF3F7FDFE002800F0CA80294628460E
:10D1C800F3F730FD4DF24E71CAF647510446F3F7B6
:10D1D80029FD47F2F641C3F20F11F3F71BFC214674
:10D1E800F3F720FD4FF27C21C3F29341F3F710FCD3
:10D1F8002146F3F717FD40F60151C3F2D071F3F75A
:10D2080009FC2146F3F70EFD40F66131C3F6B6215D
:10D21800F3F7FEFB2146F3F705FD4AF6AB21C3F60B
:10D228002A51F3F7F7FB2146F3F7FCFC804620462A
:10D238004FF07C51F3F7F6FC414606462046F3F7DB
:10D24800F1FC394604462846F3F7ECFC0146204633
:10D25800F3F7DEFB01463046F3F7DAFB01464FF001
:10D268007E50F3F7D5FBBDE8F8830146F3F7DAFC07
:10D278004DF24E71CAF647510446F3F7D3FC47F214
:10D28800F641C3F20F11F3F7C5FB2146F3F7CAFCC9
:10D298004FF27C21C3F29341F3F7BAFB2146F3F72F
:10D2A800C1FC40F60151C3F2D071F3F7B3FB21463C
:10D2B800F3F7B8FC40F66131C3F6B621F3F7A8FBE3
:10D2C8002146F3F7AFFC4AF6AB21C3F62A51F3F730
:10D2D800A1FB2146F3F7A6FC49F69913C3F6996317
:10D2E8009E428046A3DD0020C3F64870864227DCB4
:10D2F80006F17F464FF07E503146F3F789FB8146B1
:10D3080020464FF07C51F3F78DFC3146F3F780FB54
:10D31800414606462046F3F785FC3946044628462A
:10D32800F3F780FC01462046F3F772FB01463046CE
:10D33800F3F76EFB01464846F3F76AFBBDE8F8834E
:10D348004FF000090026C3F63879C3F69066D7E790
:10D358004FF07E50BDE8F8832DE9F04FDFB00C9315
:10D368000C9D224B689C0A91691ED61E48BF161D4B
:10D37800834653F82400F71027EAE77308900491CE
:10D3880004980D93089DDC43DDF834C002EBC40219
:10D3980041190792C0EB0C0750D47E18699BC7EB64
:10D3A80006090136002F03EB870522AC09F0010AB4
:10D3B800C0F2FE822868F3F7E1FB0137B74220602C
:10D3C8004FF004083AD0BAF1000F26D0002FC0F26F
:10D3D800F18255F80800F3F7D1FB0137B74244F85A
:10D3E800080008F1040818D128E000BF5C290108EA
:10D3F80055F80800F3F7C2FB013708F1040944F8AF
:10D40800080013D455F80900F3F7B8FB0137B74201
:10D4180044F8090009F1040810D0002FE8DA0020C8
:10D42800013708F1040944F80800EBD5013700205A
:10D43800B74244F8090009F10408EED1089A002A15
:10D44800C0F2458508990C9E8D004AAB5C1903957E
:10D4580049AF02944FEA860A049A002AC0F29682DB
:10D468000DF1880808EB860555F8041CAAF1040399
:10D47800DBF80000C3F38009F3F7D4FB0146002072
:10D48800F3F7C8FA0424043D544580462BD0B9F17B
:10D49800000F0DD055F8041DDBF80400F3F7C2FBAC
:10D4A80001464046F3F7B6FA0824544580461AD098
:10D4B80055F8041C5BF80400F3F7B4FB014640463A
:10D4C800F3F7A8FA0434804655F8081C5BF8040002
:10D4D800F3F7A8FB01464046F3F79CFA0434083DED
:10D4E80054458046E4D1029847F8048F01368742B4
:10D4F800B2D1039F0EA9CE190996089EB2005EAB61
:10D508009D18002E029255F8509C7DDD0DF5947CF7
:10D518004FF06E5148460DACA7180CEB0205F3F717
:10D5280081FBF3F745FDF3F729FB4FF087410190A5
:10D53800F3F778FB01464846F3F76AFAF3F738FD44
:10D548000EAC20600198014655F8040DF3F762FA15
:10D55800BC428146C7F3800156D0E9B14FF06E5105
:10D56800F3F760FBF3F724FDF3F708FB4FF087416F
:10D578000190F3F757FB01464846F3F749FAF3F7EA
:10D5880017FD019A0FAC2060114655F8040DF3F70A
:10D5980041FABC42814637D04FF06E514846F3F706
:10D5A80041FBF3F705FDF3F7E9FA4FF087418046B1
:10D5B800F3F738FB01464846F3F72AFAF3F7F8FC85
:10D5C8004146606055F8040DF3F724FA4FF06E51A8
:10D5D8008146F3F727FBF3F7EBFCF3F7CFFA4FF0AD
:10D5E80087418046F3F71EFB01464846F3F710FAD9
:10D5F800F3F7DEFC4146A06055F8040DF3F70AFA8C
:10D608000834BC428146C7D10799484600F0A2FEBB
:10D618004FF078510546F3F705FB00F025FE4FF073
:10D628008241F3F7FFFA01462846F3F7F1F9074676
:10D63800F3F7BEFC8146F3F7A1FA01463846F3F743
:10D64800E7F907990746002940F33981721E0EACA5
:10D65800079D54F82230C5F1080043FA00F101FA99
:10D6680000F0C5F107041B1A43FA04F40DF1380C55
:10D6780089444CF82230002C55DD002E09F10109AF
:10D6880040F39481029D0EABDDF808C053F8042BDB
:10D69800281F0DF1380E00250EEB0C01C0F3800099
:10D6A80022B1C2F5807243F8042C01258B4226D0A2
:10D6B80060B10F9A0433002D40F0F38022B1C2F517
:10D6C800807543F8045C01258B4218D053F8042B6D
:10D6D800002D40F0EC80C2F5807012B143F8040CC4
:10D6E800012553F8042B002D40F0DB80C2F5807033
:10D6F800002AE9D001258B4243F8040CE6D10799AA
:10D7080000290DDD012900F0E280022908D1701EF0
:10D718000DF1380E5EF8202002F03F034EF820305D
:10D72800022C00F0E08038460021F3F70FFC0028B7
:10D7380000F0F3800898751EA84225DC029B0DF1C5
:10D74800380E0EEB03010B46DDF824C053F8042D08
:10D75800CCEB0100011F6345C1F3800011D030B14B
:10D7680053F8041DDDF824E00A43734509D0099FE6
:10D7780053F8040D53F8041D0243BB4242EA010268
:10D78800F6D1002A40F01A81089F0EAD781E55F890
:10D798002020002A40F0108105EB8004012354F872
:10D7A800041D01330029FAD0F018771C87420B902A
:10D7B80075DCDDF810E00D9D0B9B0C9C0EEB070251
:10D7C800DDF808C0699F991B06EB05094AA8A61948
:10D7D80022AB07EB890900EB0C05571C8A0003EB09
:10D7E8008601029506920591002659F8040FF3F771
:10D7F800C5F9059CA051049800285EDB22AD05EB15
:10D808008702AAF10403C3F3800452F8041CDBF86E
:10D8180000000394141FF3F705FA01460020F3F7FC
:10D82800F9F84FF00408D04505462DD0039971B199
:10D8380054F8041DDBF80400F3F7F4F90146284610
:10D84800F3F7E8F84FF00808D04505461CD054F81F
:10D85800041C5BF80800F3F7E5F901462846F3F7DE
:10D86800D9F808F10408054654F8081C5BF80800C4
:10D87800F3F7D8F901462846F3F7CCF808F104087D
:10D88800083CD0450546E2D1DDF808E006980436A4
:10D898004EF8045F01378642CDF808E0A5D10B9E0B
:10D8A8002CE6C2F1FF0243F8042C01250CE7C2F173
:10D8B800FF0543F8045C012513E70025E4E75ED182
:10D8C800701E0DF1380E5EF820301C12D3E6711E62
:10D8D8000DF1380C5CF82100022C00F07F024CF8A6
:10D8E80021207FF420AF39464FF07E50F3F790F8AF
:10D8F8000746002D3FF417AF07994FF07E5000F010
:10D9080029FD01463846F3F783F8074638460021D3
:10D91800F3F71CFB00287FF40DAF0294079C3846F0
:10D928006142CDF8109000F015FD4FF08741054693
:10D93800F3F72AFB002800F0D2824FF06E512846F8
:10D94800F3F770F9F3F734FBF3F718F94FF0874161
:10D958000746F3F767F901462846F3F759F8F3F74E
:10D9680027FB0EA941F826003846F3F721FB079A52
:10D97800013608320EAC079244F8260034E04FF026
:10D988007C51F3F701FB58B90024CCE64FF00008AE
:10D99800029847F8048F013687427FF45DADA8E509
:10D9A8000224002E09F101093FF76CAE0025A6E616
:10D9B800002002E5002010E50123F5E6079A0EAEE7
:10D9C80056F82530083ACDF8109002940792002BAB
:10D9D80040F08E8206EB85042E4654F8045D013E25
:10D9E800083A002DF9D007924FF07E50079900F0C1
:10D9F800B1FC002E0446C0F2AC804FEA860AC6EBA2
:10DA0800867B0EAF4FEA8B095744C9F100034AA938
:10DA1800386801EB0A08C3F3800BF3F7AFF8214627
:10DA2800F3F700F94FF06E51C8F800002046F3F7FD
:10DA3800F9F8A9F104096FF0030ACA45054631D07F
:10DA4800BBF1000F0BD057F8040CF3F797F82946F1
:10DA5800F3F7E8F86FF0070A48F8040C1AE057F8EB
:10DA68000A00F3F78BF82946F3F7DCF84FF06E510C
:10DA780048F80A002846F3F7D5F8AAF10404054641
:10DA88003859F3F77BF82946F3F7CCF8AAF1080AD6
:10DA980048F8040028464FF06E51F3F7C3F8CA451A
:10DAA8000546DCD1701CDFF84C94DDF820A003900B
:10DAB80000270596BAF1000FC0F20582002FC0F2C8
:10DAC8000282002600241AF0010F354620D0D8F82B
:10DAD8000010D9F80000F3F7A5F801462046F2F740
:10DAE80099FF0125AA45044626DB0426BD420FDD21
:10DAF80022E0BB4520DC58F8021059F80200F3F781
:10DB080091F801462046F2F785FFBD42044613DC32
:10DB180058F8061059F80600F3F784F8014620462D
:10DB2800F2F778FF05F1010B06F104020235DA4538
:10DB3800044602F10406DCDA5EABDDF80CC003EB48
:10DB480087010137674541F8A04CA8F10408B1D115
:10DB5800059E689C032C16D8DFE814F085011F0188
:10DB68001F011B0000230299002900F00B81379C3C
:10DB7800369804F100420A9C00F1004503F1004385
:10DB880025606260A360049D05F007005FB0BDE8F2
:10DB9800F08F002EE6DD06F1FF3836AF07EB880977
:10DBA8004D4655F804290DF1D40AD5F808B01046A9
:10DBB80059460192F2F72EFF804641460198F2F746
:10DBC80027FF01465846F2F725FF5545C9F380035C
:10DBD800A860C5F8048044D0BBB155F80429D5F82D
:10DBE80008B0104659460192F2F714FF0199804691
:10DBF80008464146F2F70CFF01465846F2F70AFF7D
:10DC08005545C5F80480A8602BD02C4654F8043933
:10DC1800D4F808B0184659460193F2F7FBFE80463F
:10DC280041460198F2F7F4FE01465846F2F7F2FE33
:10DC3800C4F80480A06055F804BC251FD5F80880F6
:10DC480058464146F2F7E6FE044621465846F2F7A2
:10DC5800DFFE01464046F2F7DDFE55456C60A860E0
:10DC6800D3D1012E7FF77EAF4D4655F804B9C7EBE7
:10DC7800090ED5F808A058465146AEF10409F2F746
:10DC8800C9FE804641465846F2F7C2FE0146504654
:10DC9800F2F7C0FEBD42C9F38009C5F80480A86048
:10DCA80043D0B9F1000F15D055F804A9D5F808905C
:10DCB80050464946F2F7AEFE804641465046F2F7D6
:10DCC800A7FE01464846F2F7A5FEBD42C5F8048006
:10DCD800A8602AD02C4654F804A9D4F808905046D5
:10DCE8004946F2F797FE804641465046F2F790FEC5
:10DCF80001464846F2F78EFEC4F80480A06055F845
:10DD0800049C251FD5F8088048464146F2F782FE54
:10DD1800044621464846F2F77BFE01464046F2F7A4
:10DD280079FEBD426C60A860D4D1013607EB860746
:10DD380008353E467A1B131F56F8041D0020C3F30E
:10DD48008007F2F767FEAE4203463FF40CAF3FB1DF
:10DD580056F8041DF2F75EFEAE4203463FF403AFE9
:10DD6800184656F8041C341FF2F754FE083E54F8BF
:10DD7800041CF2F74FFEAE42F3D102990346002984
:10DD88007FF4F5AEDDF828C036993798CCF8001046
:10DD9800CCF80400CCF80830F5E60023002E29DB87
:10DDA80036AF751C07EB85042546E21B55F8041DA4
:10DDB800A2F1040E0020CEF38008F2F72BFEBD423C
:10DDC800034617D0B8F1000F06D055F8041DF2F736
:10DDD80021FEBD4203460DD0184655F8041C2C1FE1
:10DDE800F2F718FE083D54F8041CF2F713FEBD4282
:10DDF800F3D103460299002967D003F10040DDF80A
:10DE080028C01946CCF800003698F2F701FE002E1B
:10DE1800034621DD36AF07EB8606F51B2A1F379927
:10DE2800C2F38007F2F7F6FD37ACB442034613D0CD
:10DE380037B16168F2F7EEFD38ACB44203460BD057
:10DE4800184654F8041FF2F7E5FD54F8041FF2F7DA
:10DE5800E1FDB442F5D10346029909B103F100434B
:10DE68000A9C63608FE6002E40DB36AF013607EB75
:10DE780086000546C21B55F8041D0020141FF2F742
:10DE8800C9FDBD42C4F38006034615D036B155F826
:10DE9800041DF2F7BFFDBD4203460DD0184655F8E4
:10DEA800041C2C1FF2F7B6FD083D54F8041CF2F7C9
:10DEB800B1FDBD42F3D10346029909B103F1004314
:10DEC8000A9C23605FE6002436E6184697E7DDF8EB
:10DED80030E0900003904FEA8E0AFFF70ABB28460D
:10DEE800F3F766F80EAB43F826007DE50023E3E779
:10DEF8002E4679E5682901082DE9F84320F000430A
:10DF0800B3F1485F04460F46904603DAF3F750F83A
:10DF1800002859D021462046F2F784FE21460546BE
:10DF2800F2F780FE4CF6D311C2F62E71064628464B
:10DF3800F2F778FE42F63471C3F2D721F2F768FDA2
:10DF48002946F2F76FFE4EF61B71C3F23861F2F7FD
:10DF580061FD2946F2F766FE40F60151C3F65011FD
:10DF6800F2F756FD2946F2F75DFE48F68901C3F639
:10DF78000841F2F74FFD8146B8F1000F27D04FF066
:10DF88007C513846F2F74EFE494680463046F2F755
:10DF980049FE01464046F2F73BFD2946F2F742FEAC
:10DFA8003946F2F735FD4AF6AB210546C3F62A6134
:10DFB8003046F2F737FE01462846F2F72BFD0146B8
:10DFC8002046F2F725FD04462046BDE8F8830146C1
:10DFD8002846F2F727FE4AF6AB21C3F62A61F2F784
:10DFE80017FD3146F2F71EFE01462046F2F712FDF4
:10DFF80004462046BDE8F883002070470021002031
:10E00800C7F6F871704700BF2DE9F04120F00045D0
:10E01800B5F1A14F044606460DDBB5F1FF4F00F3FD
:10E028009C80002840F6DB7440F3D480C3F6C974A2
:10E038002046BDE8F0814FF6FF73C3F6DF639D42CB
:10E0480000F3A280B5F1445FC0F28E804FF0FF3735
:10E0580021462046F2F7E6FD01468046F2F7E2FD4A
:10E0680046F6D711C3F685410546F2F7DBFD4DF6B6
:10E078005921C3F64B51F2F7CDFC2946F2F7D2FDF0
:10E0880046F63531C3F68851F2F7C4FC2946F2F753
:10E09800C9FD42F66E61C3F6BA51F2F7BBFC2946D8
:10E0A800F2F7C0FD44F62511C3F61261F2F7B2FC8F
:10E0B8002946F2F7B7FD4AF6AB21C3F6AA61F2F793
:10E0C800A9FC4146F2F7AEFD4AF221218046CBF683
:10E0D80015512846F2F7A6FD4FF26B11C3F66E51A3
:10E0E800F2F796FC2946F2F79DFD48F29571C3F6C2
:10E0F8009D51F2F78DFC2946F2F794FD48F63861F8
:10E10800C3F6E351F2F784FC2946F2F78BFD4CF68F
:10E11800CD41C3F64C61F2F77BFC2946F2F782FD4C
:10E128007B1C0146404658D0F2F774FC2146F2F7B2
:10E1380079FD494B53F82710F2F76AFC2146F2F7AC
:10E1480067FC0146454850F82700F2F761FC002EAD
:10E158003DDB04462046BDE8F0810146F2F75AFC53
:10E1680004462046BDE8F0814FF2CA21C7F24911A2
:10E17800F2F750FC4FF07E51F2F710FF00283FF401
:10E1880065AF2046BDE8F08100F06AF84FF6FF71F0
:10E19800C3F697718D4204464FF6FF7228DCC3F62A
:10E1A8002F72954246DC0146F2F734FC4FF07E515F
:10E1B800F2F72EFC4FF0804105462046F2F72AFC84
:10E1C80001462846F2F7E2FD0027044640E700F141
:10E1D80000442DE7CBF6C9742AE7F2F71BFC214669
:10E1E800F2F720FD01462046F2F712FC04461FE72D
:10E1F800C4F21B02954214DC4FF07F51F2F708FC81
:10E208004FF07F5105462046F2F70CFD4FF07E5146
:10E21800F2F700FC01462846F2F7B8FD022704464B
:10E2280016E700202146CBF68070F2F7AFFD0327F2
:10E2380004460DE74FF07E51F2F7EAFB4FF07E51AE
:10E2480007462046F2F7E6FB01463846F2F79EFD00
:10E2580001270446FCE600BF94290108A429010807
:10E2680020F00040704700BFF8B520F00046F50DDB
:10E278007F3D162D014604461BDC002D074620DB9A
:10E288004FF6FF73C0F27F0343FA05F606420ED03D
:10E298004FF2CA21C7F24911F2F7BCFB0021F2F78D
:10E2A8007DFE18B1002C1BDB27EA06042146084630
:10E2B800F8BDB6F1FF4FFAD3F2F7ACFB01460846BA
:10E2C800F8BD4FF2CA21C7F24911F2F7A3FB0021AA
:10E2D800F2F764FE0028E9D0002C07DB0024E5E70C
:10E2E8004FF4000040FA05F56719DDE70021CBF689
:10E2F8008071002E18BF0C46D8E700BF08B902206D
:10E308007047B0F1004FFAD0A0F500026FF001435A
:10E318009A4201D80420704700F1FF419942F9D987
:10E328004FF6FE73421EC0F27F039A4201D80320C3
:10E33800704700F100414A1E9A42F8D9B0F1FF4FE8
:10E3480005D010F5000F14BF0020012070470120F0
:10E35800704700BF38B530F00044034602460D460A
:10E368000FD0B4F1FF4F0ED2B4F5000F11D3E40D66
:10E378006419FE2C33DC002C1BDD22F0FF4141EA3E
:10E38800C453184638BD0146F2F744FB0346184605
:10E3980038BD4FF09841F2F745FC43F6B041CFF64F
:10E3A800FF718D42034612DBC0F3C7540246193C85
:10E3B800DEE714F1160F21DA4CF250329542194675
:10E3C8000EDC44F26020C0F6A25000F023F844F2BC
:10E3D8006021C0F6A251F2F725FC0346D1E71946A1
:10E3E8004FF2CA20C7F2491000F014F84FF2CA21C0
:10E3F800C7F24911F2F716FC0346C2E722F0FF43C1
:10E4080004F1190043EAC0504FF04C51F2F70AFCEE
:10E418000346B6E701F0004120F00040084370478A
:10E428002DE9F041274C84B025680746D5F84841C6
:10E43800002C41D066681F2E1CDD234810B94FF010
:10E44800FF301FE04FF4C870039102920193AFF3BD
:10E45800008003990446029A019B0028EFD0D5F862
:10E468004861002060602660C5F84841C4F888010A
:10E47800C4F88C01656847B9A81C013544F8201018
:10E488006560002004B0BDE8F081012000FA05F0C5
:10E49800D4F8886104EB85080643022FC8F8882061
:10E4A800C4F88861C8F80831E6D1D4F88C3143EA59
:10E4B8000002C4F88C21DFE705F5A674C5F84841C9
:10E4C800B8E700BFBC2A01080000000000210A22AA
:10E4D80001F07ABD2DE9F84FDDF828B081468A466B
:10E4E80098469AB193B11646002503E00FD0651CF3
:10E4F800AE420BD97419640808FB04A7484639468C
:10E50800D8470028F2DA2646AE42F3D80027384624
:10E51800BDE8F88F40F2D053C2F200031868704784
:10E52800114B124A70B5981A831018D0591E02EB75
:10E5380083040D4654F8042D01F00106904775B187
:10E5480026B154F8040D8047013D08D054F8043D25
:10E558009847013D54F8041D8847013DF6D1BDE8B0
:10E56800704004F0AFBA00BFE42A0108E02A0108AD
:10E578000F2A2DE9F00340F2A18041EA00039B072E
:10E5880040F09E800C68A2F1100504604B68AC4610
:10E5980043608C68BCF10F0F8460CC68C5F300152C
:10E5A800C46000F1100301F110042BD975B125687E
:10E5B800ACF1100C1D6065685D60A5689D60E5683C
:10E5C8001034DD601033BCF10F0F1BD9276804F13C
:10E5D80010061F60676803F110055F60A768ACF15B
:10E5E800200C9F60E768DF6024691C61776806F18A
:10E5F80010046F60B7682033AF60F668BCF10F0F86
:10E60800EE60E3D8A2F1100828F00F0302F00F041F
:10E6180003F1100C032C00EB0C0301EB0C0851D98F
:10E62800211F4FEA9109444608EB890C54F8046B02
:10E63800C8EB0C010CF1040C1D46644545F8046B4D
:10E64800C1F3800112D029B154F8041B644545F880
:10E65800041B0BD0274657F8041B2E4646F8041B0C
:10E6680064686C603C1D351D6445F3D109F1010CEB
:10E678004FEA8C0902F0030208EB09014B44D2B1BE
:10E688000D789A18DC4303F8015B1419934204F0DF
:10E69800010410D02CB111F8014F03F8014B93423B
:10E6A80009D04D781C4604F8015B8D7802315D7005
:10E6B800631C9342F5D1BDE8F00370470346DEE7DB
:10E6C8000346DDE741462246D9E700BFF0B4840798
:10E6D800034600F08D80541E002A00F08780E5076D
:10E6E800CEB211D41A4602F8016B134615469207AA
:10E6F80010D0621E002C79D003F8016B14469A07DB
:10E708001D4607D0013CEDE7034603F8016B9A0765
:10E718001D46F7D1032C52D9CEB246EA06270F2C54
:10E7280047EA07432DD9A4F1100217460F2FC2F369
:10E7380000162B606B60AB60EB6005F1100216D918
:10E748003EB1103F136053609360D36010320F2FB7
:10E758000DD9203F02F11006136053609360D36017
:10E76800136153619361D36120320F2FF1D8A4F163
:10E77800100222F00F0204F00F041032032C15448B
:10E788001DD9271F3E462A46032E42F8043BC7F3ED
:10E7980080070DD927B1043E032E42F8043B07D960
:10E7A800174647F8043B083E53603A1D032EF7D836
:10E7B800231F23F00302131D04F00304ED18ACB16A
:10E7C800C9B2EA432C1905F8011BA318A54203F0A6
:10E7D80001020BD01AB105F8011BA54206D02B4641
:10E7E80003F8011B69705D1CA542F8D1F0BC7047A5
:10E7F800054614468EE700BF2DE9F04F89B0144650
:10E808008046019202EB4202A508500004F003047E
:10E8180018F0030F0291994603950694079040F06B
:10E82800D6800699002940F05A82019A151F18BF10
:10E8380001250095029D062D40F2CF80DDF808C025
:10E84800019F64464FEA5C06072C07FB068A40F0E6
:10E85800E281DDF81CC008EB0C06009B002B40F0A1
:10E86800FB81D8F80010DAF80030C8F80030CAF890
:10E8780000100198DDF804A008EB000549460022C5
:10E8880005952F4604953446CAF1000A91460D466F
:10E89800A74240F213812B464D469946002D00F0C1
:10E8A800C183DDF810B00299CBEB070AC8EB0B0265
:10E8B8005245A8BF5246DDF804C0002A0CFB018B64
:10E8C8003ADD009BB91A022B404640F0D28210F87C
:10E8D800015B91F800C0029500F801CCDDF808C092
:10E8E8000B468A18CD4303F801CBAD18013093428B
:10E8F80005F0010520D04DB110F8015C497800F809
:10E90800011C03F8015B0130934215D0014611F850
:10E91800015C93F800C0184601F801CC00F8015BCF
:10E9280011F8015B93F801C0034601F801CC03F824
:10E93800015B01319342EAD10199C6EB0B03341B09
:10E94800581AA04228BF204600282FDD009DC0EBA2
:10E958000B02022D40F053821578FB4339783818A2
:10E9680007F8015B874203EB0005134603F8011B18
:10E9780005F001011AD039B155783A7807F8015BEA
:10E98800874203F8012B11D03D781E781A46394684
:10E9980001F8016B02F8015B5B787D780F4607F898
:10E9A800013B8742134603F8015BEDD1019D5545B4
:10E9B800C0F08C81DDF804C0A4457CD2C4EB0B0800
:10E9C80018F0030FB4FBFCF402943FF42AAF029D45
:10E9D8000223062D00933FF631AFDDF804C00CFB8F
:10E9E800058A08EB0C01514565D2019CDDF804B09D
:10E9F80065420434009E02940091CDF810A04F4661
:10EA0800DDF80090C14509D84DE0D9F8000021682B
:10EA1800C9F8001020604445A14644D909EB050413
:10EA280020464946B84700283DDD002EEDD0012E8E
:10EA380000F0A7831BF804E094F800900BF1FF3175
:10EA48000BEB04000246234601F0010C002902F8F2
:10EA5800019B03F801EBDEDDBCF1000F09D0407823
:10EA680094F801E00139002902F801EB03F8010BE1
:10EA7800D1DD93F800A092F80090944618460CF85F
:10EA880001AB00F8019B92F801E093F801A002396C
:10EA980062460346002902F801AB03F801EBE8DC03
:10EAA8004445A146BAD8DDF800C0049BDC449C4527
:10EAB800CDF800C0A4D309B0BDE8F08F3846414670
:10EAC800A84700280BDC8CE02068326822603060A0
:10EAD80056444FF001095444A7423FF6DCAE2046A5
:10EAE8004146A8470028C0F29A83F4D1009B002B26
:10EAF800EAD00099012935D0DDF804E0207896F8AD
:10EB080000C00EF1FF312246334601F00109002909
:10EB180002F801CB03F8010BDADDB9F1000F09D0D7
:10EB2800107893F800C00139002902F801CB03F8E6
:10EB3800010BCDDD93F800B092F800E0944618463A
:10EB48000CF801BB00F801EB92F8019093F801B0C2
:10EB5800023962460346002902F801BB03F8019B0B
:10EB6800E8DCB5E721463346DDF80CE053F8042B22
:10EB780051F8040B0EF1FF3C41F8042C0CF0010293
:10EB880043F8040C04310433BCF1000FA0DD72B16A
:10EB980051F8040C53F8042C0CF1FF3C41F8042CF8
:10EBA80043F8040C04310433BCF1000F90DD53F832
:10EBB800042C51F8049C084641F8042C1A4643F8E2
:10EBC800049C50F8043B52F8041BACF1020C40F8CA
:10EBD800041C011D42F8043C131DBCF1000FE6DCC7
:10EBE80076E714D1009A002A7CD104983B68026821
:10EBF800DDF810C0CCF800303A60DDF810E0DDF840
:10EC080004900EEB090CCDF810C04FF00109DDF8A7
:10EC180004E077443CE602980199431E282801FB4A
:10EC2800038600F2AB803446454651462846C8471D
:10EC3800002821465046C0F29580C84700283FF773
:10EC48000CAE28462146C847009B34EA200A28BF54
:10EC5800AA46002B3FF405AE00994246012900F070
:10EC68004781DDF804C012F8015B9AF800400CF106
:10EC7800FF3102F8014C574601F00100013200292A
:10EC880007F8015B7FF7F5AD58B13D7812F8013C04
:10EC9800013902F8015C0132002907F8013B7FF7CE
:10ECA800E8AD12F8014C3B78384602F8013C00F810
:10ECB800014B12F8014B7D78023902F8015C0746D6
:10ECC8000132002907F8014BEBDCD2E5019D4046F3
:10ECD800BAFBF5F12A464B46FFF78EFD6AE6022499
:10ECE8000094A7E50098012800F03B81DDF810E0CA
:10ECF800DDF804B039789EF800000BF1FF3B72464E
:10ED080002F8011B3B460BF00101BBF1000F03F8B1
:10ED1800010B7FF772AF59B1117818780BF1FF3BEF
:10ED2800BBF1000F02F8010B03F8011B7FF765AF79
:10ED380092F800C093F800901046194600F8019B1D
:10ED480001F801CB92F801E093F801C0ABF1020B96
:10ED580002460B46BBF1000F02F801CB03F801EBAA
:10ED6800E6DC4AE7C8470028FFF677AD2846214683
:10ED7800C84735EA200A28BFA2466EE5019AC408AA
:10ED880002FB04F408EB04054FEA440B294640460D
:10ED9800CDF810B0C84708EB0B07002839462846BD
:10EDA800C0F23481C847002840F33182C4F1000B17
:10EDB8000AEB0B0751463846C847544400282146F9
:10EDC8005046C0F21781C847002840F318820498BB
:10EDD80006EB0B04371A21463846C8470028314647
:10EDE8002046C0F2FB80C84700283FF71EAF3846D0
:10EDF8003146C84736EA200428BF3C4615E739465D
:10EE0800134653F8042B51F8045B8008013841F885
:10EE1800042C00F0010243F8045C04310433002898
:10EE28007FF7C4AD6AB151F8045C53F8042C01387B
:10EE380041F8042C43F8045C0431043300287FF7BC
:10EE4800B5AD51F8046C53F8042C0D4641F8042C68
:10EE580043F8046C1A4652F8041B55F8046B023840
:10EE680045F8041C131D291D002842F8046CE8DC31
:10EE78009CE50B4653F8045B50F8041B920802F11A
:10EE8800FF3C40F8045C021D0CF0010543F8041C2B
:10EE98000433BCF1000F7FF74FAD7DB152F8041C6D
:10EEA80053F8040C0CF1FF3C42F8040C43F8041C22
:10EEB80004320433BCF1000F7FF73EAD52F8045C16
:10EEC80053F8040C114642F8040C43F8045C184645
:10EED80050F8042B51F8045BACF1020C41F8042CF7
:10EEE800031D0A1DBCF1000F40F8045CE6DC23E5B5
:10EEF8005746039952F8043B57F8040B013942F876
:10EF0800040C01F0010447F8043C04323B1D0029BD
:10EF18007FF7AFAC6CB152F8045C53F8047C01394C
:10EF280042F8047C43F8045C0432043300297FF778
:10EF3800A0AC52F8045C53F8040C144642F8040CD4
:10EF48001F4643F8045C57F8042B54F8045B023955
:10EF580044F8042C3B1D221D002947F8045CE8DC1A
:10EF680087E404993B46DDF80C9053F8042B51F8DC
:10EF780004EB09F1FF3041F8042C00F0010243F8DA
:10EF880004EC0431043300287FF737AE6AB151F836
:10EF980004CC53F8042C013841F8042C43F804CC71
:10EFA8000431043300287FF728AE53F8042C51F8B5
:10EFB80004EC894641F8042C1A4643F804EC59F845
:10EFC800043B52F8041B023849F8041C42F8043C7C
:10EFD800131D002809F10401E7DC0EE6C8470028E4
:10EFE800FFF623AE38463146C84737EA200428BF23
:10EFF80034461AE6C8470028FFF6E9AE38462146E7
:10F00800C84737EA200A28BFA246E0E6C8470028D2
:10F01800FFF6CCAE40463946C84738EA200528BF37
:10F028003D46C3E60298019C059D04FB008A5545B0
:10F03800BFF441AD019FDDF814B03C1D009ECDF832
:10F0480000B0DDF804B07D420494CDF808A01F4656
:10F05800DDF80090C84509D34CE0D9F800002168D4
:10F06800C9F8001020604445A14643D909EB0504BE
:10F0780020464946B84700283CDD002EEDD0012E39
:10F0880041D01BF804E094F800900BF1FF310BEB32
:10F0980004000246234601F0010C002902F8019BF6
:10F0A80003F801EBDFDDBCF1000F09D0407894F8DC
:10F0B80001E00139002902F801EB03F8010BD2DD68
:10F0C80093F800A092F80090944618460CF801AB0B
:10F0D80000F8019B92F801E093F801A0023962461A
:10F0E8000346002902F801AB03F801EBE8DC4445CC
:10F0F800A146BBD8DDF800C0029BDC449C45CDF896
:10F1080000C0A5D3D7E4DDF81090234609EB04022C
:10F11800DDF80CE053F8041B52F804CC0EF1FF3074
:10F1280042F8041C00F0010143F804CC0432043313
:10F13800002898DD61B152F8049C53F8041C01388A
:10F1480042F8041C43F8049C0432043300288ADD86
:10F1580053F8041C52F804EC944642F8041C19466F
:10F1680043F804EC5CF8043B51F8042B02384CF8E3
:10F17800042C41F8043C0B1D00280CF10402E7DCC8
:10F1880071E7029A23461219DDF80C9053F8041B14
:10F1980052F804CC09F1FF3042F8041C00F00101D8
:10F1A80043F804CC0432043300287FF734AC69B147
:10F1B80052F804EC53F8041C013842F8041C43F8D4
:10F1C80004EC0432043300287FF725AC53F8041C00
:10F1D80052F8049C944642F8041C194643F8049CCF
:10F1E8005CF8043B51F8042B02384CF8042C41F825
:10F1F800043C0B1D00280CF10402E7DC0BE4384644
:10F208002146C84734EA200A28BFBA46DFE5404607
:10F218003946C84737EA200528BF4546C6E5A7420C
:10F228003FF639AB009B63B9386822683A602060C2
:10F23800DDF804E04FF001097744CEEB0404FFF752
:10F2480027BB0098012833D0DDF80490207897F880
:10F2580000E009F1FF313A4602F8010B234601F0BC
:10F268000100002903F801EBE2DD48B1107893F8BA
:10F2780000C00139002902F801CB03F8010BD7DDE2
:10F2880093F800B092F800E0944618460CF801BBD9
:10F2980000F801EB92F8019093F801B00239624648
:10F2A8000346002902F801BB03F8019BE8DCBFE72D
:10F2B80039462346DDF80CE053F8042B51F8040BCB
:10F2C8000EF1FF3C41F8042C0CF0010243F8040C49
:10F2D80004310433BCF1000FAADD72B151F8040CFB
:10F2E80053F8042C0CF1FF3C41F8042C43F8040CAF
:10F2F80004310433BCF1000F9ADD53F8042C51F8A3
:10F30800049C084641F8042C1A4643F8049C50F81B
:10F31800043B52F8041BACF1020C40F8041C011D1C
:10F3280042F8043C131DBCF1000FE6DC80E700BF87
:10F33800830770B5064614D10368A3F1013222EAA7
:10F34800030010F0803F0CD1331D1A4653F8044BCC
:10F35800A4F1013525EA040414F0803FF5D01046E5
:10F3680000E0304603782BB1421C14781046013275
:10F37800002CFAD100F080F8304670BDC9B2F0B464
:10F3880000294BD082070FD00278002A71D0914211
:10F3980042D0431C05E013F8012B002A3BD09142D0
:10F3A8003AD09A071846F6D1036841EA0127A3F133
:10F3B800013222EA030212F0803F47EA07471CD1D4
:10F3C8007B40A3F1013222EA030313F0803F14D1FA
:10F3D800021D02E014F0803F0FD1104652F8043BA2
:10F3E800A3F1013687EA030426EA0303A4F10135F1
:10F3F80013F0803F25EA0404ECD00278002A38D0C4
:10F40800914209D0431C01E0914205D0184613F8F7
:10F41800012B002AF8D11046F0BC704783070BD0A7
:10F428000278002AF8D0431C03E001780133002950
:10F43800F2D099071846F8D10168A1F1013323EAFF
:10F44800010212F0803F0AD1031D184653F8041B2D
:10F45800A1F1013424EA010212F0803FF5D00378CB
:10F46800002BD9D0421C1178104601320029FAD15C
:10F47800D2E71046D0E700BF80EA0102844612F0C6
:10F48800030F4FD111F0030F32D14DF8044D11F095
:10F49800040F51F8043B0BD0A3F101329A4312F048
:10F4A800803F04BF4CF8043B51F8043B16D100BF21
:10F4B80051F8044BA3F101329A4312F0803FA4F1B2
:10F4C80001320BD14CF8043BA24312F0803F04BF39
:10F4D80051F8043B4CF8044BEAD023460CF8013BA6
:10F4E80013F0FF0F4FEA3323F8D15DF8044B704750
:10F4F80011F0010F06D011F8012B0CF8012B002A8E
:10F5080008BF704711F0020FBFD031F8022B12F07C
:10F51800FF0F16BF2CF8022B8CF8002012F47F4F37
:10F52800B3D1704711F8012B0CF8012B002AF9D13F
:10F53800704700BF20F0030110F00300C0F1000085
:10F5480051F8043B00F1040C4FEACC0C6FF00002B8
:10F558001CBF22FA0CF213434FF0010C4CEA0C2C9E
:10F568004CEA0C4CA3EB0C0222EA030212EACC127E
:10F5780004BF51F8043B0430F4D013F0FF0F1FBF51
:10F58800013013F47F4F013013F47F0F18BF01309F
:10F59800704700BFF0B4002A63D0344B04461B68A0
:10F5A80014F8010B571E1D186E7807F0010706F0B6
:10F5B8000305012D58D011F8015B5E19767806F025
:10F5C8000306012E08BF2035401B4BD1002D49D022
:10F5D800013A47D02FB314F8010B1D186E7806F0C6
:10F5E8000305012D11F8015B08BF20305E197678FC
:10F5F80006F00306012E08BF2035401B32D18DB31B
:10F60800013A0ED12EE011F8012B9E18767806F0FB
:10F618000306012E08BF2032801A23D112B36A1EB6
:10F6280020D014F8010B1D186E7806F00305012D83
:10F6380011F8015B08BF20305E19767806F00306E2
:10F64800012E08BF2035401B0CD15DB114F8010B09
:10F65800551E1A18567806F00302012AD3D1203015
:10F66800D1E71046F0BC70472030A4E7A401002081
:10F6780041EA00039B07F0B474D1032A72D90C46FF
:10F6880054F8045B161FA5F1013727EA050717F0A0
:10F69800803F0346C6F3800C31D10346032E324621
:10F6A80043F8045B2AD9BCF1000F0AD0214654F86C
:10F6B800045BA5F1013626EA050616F0803F18D04E
:10F6C8001DE0264656F8045B2146A5F1013727EAD6
:10F6D800050717F0803F12D143F8045B656831468F
:10F6E800A5F1013626EA0506043A0C1D16F0803FFE
:10F6F80005D1043A032A43F8045BE2D821467AB3D9
:10F708000D78013A03F8015B9DB112F0010F1C4618
:10F718002AD1234622B311F8015F013A03F8015BAD
:10F728003DB111F8015F013A65705C1C2346002D5C
:10F73800EFD1AAB100219C18DA4303F8011BA218E3
:10F74800A34202F001020BD01AB103F8011BA34235
:10F7580006D01A4602F8011B5970531CA342F8D16F
:10F76800F0BC70470346CAE711F8015F1C4604F86D
:10F77800015B013A2346002DCBD1DAE72DE9F007EA
:10F7880001273C4600254FF0FF3663198B4200EBFA
:10F79800060C0DD21CF804A010F80380D0452ED218
:10F7A80001241D469F1B63198B4200EB060CF1D305
:10F7B8004FF0010A1760544600254FF0FF3C6319CB
:10F7C800994200EB0C080ED918F8048010F8039041
:10F7D800C1451AD901241D46CCEB030A6319994285
:10F7E80000EB0C08F0D80CF101000136B0423CBF28
:10F7F800BA463046C2F800A0BDE8F00770470BD003
:10F8080001272E463C46ED19BFE709D04FF0010A03
:10F81800AC4654465544D2E7BC4205D00134B4E75F
:10F82800544505D00134CAE727461D460124ACE7F4
:10F83800A2461D460124C2E72DE9F04FADF2244D42
:10F848001546064689461046194607AA1C46FFF77C
:10F8580095FF07AB82460DF21C411A1D5C60083308
:10F868008B425460F9D114B301232F78611E08A884
:10F87800A34240F8271001EA030218D032B16A788F
:10F8880002234F1EA34240F8227010D0B046A4466F
:10F898005C1C15F803E0CE1A2A5D02330F1B634582
:10F8A80040F82E6040F82270F2D146466446079927
:10F8B80028466918524600F045FC002840F0B680FA
:10F8C8000AF1FF3E05EB0E0CCDF808E0CAF1010E77
:10F8D800834604F1FF38CDF80CC0CDF814E0074694
:10F8E800CDF810A04A460095019408E027B1079F7B
:10F8F800BB4201D20199CB1B9B4400272246019CA5
:10F90800B0185C440021A21A00F07CFB002840F0EB
:10F918008780002C00F08480301910F8013C08A979
:10F9280051F82330002BE1D1049B9F4228BF3B466E
:10F93800434527D2DDF8009006EB0B0119F8035078
:10F94800CA5C09EB0300954266D1DD43454415F0D6
:10F95800010F024613D00133434513D24078CD5CE2
:10F96800013285420BD057E012F8010FCD5C854279
:10F9780052D1013312F8010FCD5C85424CD10133CD
:10F988004345F1D3DDF81090029B4F4528BF4B4605
:10F9980039D2DDF808C0DDF8009006EB0B0519F840
:10F9A8000C1015F80C00814240F0C080DDF80CE026
:10F9B80009EB070ACAEB0E01C80772461ED5DDF827
:10F9C800089009F1FF31DDF80C90685C19F801CC5A
:10F9D80009F1FF32844516D10B460FE012F8019C5D
:10F9E80015F800E04A1EF1450DD10346013815F817
:10F9F80000C011F8011C614505D10346581E524547
:10FA080002F1FF31EAD101379F4200F29180079F4E
:10FA1800019ABB44D71B71E7DDF814E0F3446BE7A8
:10FA2800002009B00DF5806DBDE8F08FCAEB040029
:10FA3800504538BF5046CAF10102431C0AF1FF3C49
:10FA480005EB0A0704F1FF3B019200944A4607932D
:10FA5800B1464FF0000864463E46009909EB0200A3
:10FA680008EB0107BA1A002100F0CCFA0028D7D118
:10FA7800002FD5D009EB070010F8013C08AA52F86E
:10FA8800230000284AD1DA4509EB08002AD210F8E9
:10FA98000A303178994218BF534642D16FEA0A03B7
:10FAA80003EB0B01C9073246534618D50AF1010387
:10FAB8005B4517D2324612F8011F10F803E08E4555
:10FAC8000DD02EE012F8011F10F803C08C4528D184
:10FAD800013312F8011F10F803E08E4521D10133DC
:10FAE8005B45EFD3621C23469BD0295D025D9142A2
:10FAF80013D1E10709D5631EE95CC25C914204D0C9
:10FB08000BE0E95CC25C914207D15A1E002B88D0F9
:10FB1800A95C825C023B9142F3D0079880443A4644
:10FB28009BE7DDF804C0E0449844F8E7049B6AE7E3
:10FB380006EB0B0075E700BF2DE9F04F037889B09D
:10FB480080460D46002B00F065810A789AB18446FC
:10FB58000131012602E011F8012B5AB1934214BF7A
:10FB6800002606F001061CF8013F0C46002BF2D1D6
:10FB7800207820B936B1404609B0BDE8F08F4FF083
:10FB88000008F8E708F101002978FFF7F7FB641B84
:10FB980006460028F3D0012C00F0B580A04440456B
:10FBA80094BFC0EB080701271F2C06D939462A46FF
:10FBB8002346FFF741FE8046DDE7214607AA28468F
:10FBC800FFF7DCFD0799039069182846039A00F0AF
:10FBD800B9FA002840F09980DDF80CC0DDF80C90E7
:10FBE8000CF1FF3E05EB0E01C9F1010C8346CDF87F
:10FBF80008E080460491CDF814C03A46B146019514
:10FC080008EB040609EB02000021B21A00F0FAF929
:10FC18000028B4D1002EB2D0039B9B4528BF5B4679
:10FC28009C4227D9019D09EB030010F80820E95CE4
:10FC3800E81891425FD1DD432D1915F0010F0246F6
:10FC480009EB080113D001339C4213D94078CD5CED
:10FC5800013285420BD04EE012F8010FCD5C85428F
:10FC680049D1013312F8010FCD5C854243D10133EC
:10FC78009C42F1D8DDF80CE0029ADE4540F2CD80D6
:10FC8800019B09EB0805995CA85C814240F0C5809E
:10FC9800DDF804A0049BDA44CAEB0301C8071AD5AF
:10FCA800029FDDF810C0791E685C1CF8017C0CF11D
:10FCB800FF33874214D10A460DE013F801EC2F5C9C
:10FCC8004B1EBE450CD1024601382F5C11F8011CB1
:10FCD800B94205D10246501E534503F1FF31ECD11C
:10FCE8000BF1010B934500F29A80079A9044C2EBFE
:10FCF800040B324684E7059D05EB080B0BEB030864
:10FD08004FF0000BF5E7804635E7DDF80CA00399C6
:10FD1800CAEB0403534538BF5346CAF1010B581CBC
:10FD280006EB0A0205EB0A08CDF808B03B46079037
:10FD38004FF00009019201F1FF3B37468A4609EB73
:10FD48000406F8180021F21A00F05CF900287FF484
:10FD580016AF002E3FF413AF544598BF07EB0900C8
:10FD68002CD9DDF804E098F800001EF80930984214
:10FD78004AD16FEA0A021119C9074246534607EBEE
:10FD8800090018D50AF101039C4217D9424612F816
:10FD9800011F10F803C08C450DD036E012F8011F82
:10FDA80010F803E08E4530D1013312F8011F10F826
:10FDB80003C08C4529D101339C42EFD8BBF1FF3FEA
:10FDC8005B463FF4F8AE15F80B1010F80B20914283
:10FDD80016D11BF0010F0AD00BF1FF33E95CC25CAE
:10FDE800914204D00CE0E95CC25C914208D15A1EF1
:10FDF800002B3FF4E0AEA95C825C023B9142F2D05A
:10FE08000798814433469AE75346DDF808E0F14401
:10FE18009944F7E70C460126AAE6039A60E74E469E
:10FE2800C844A8E640F2D053C2F200031A6801237E
:10FE38005C3200F001B800BFF0B4002825D00746B6
:10FE480038463E780D46013715F8014B3CB1A642BD
:10FE5800FAD1002BF4D1176007F8013C11E0C6B1C4
:10FE68003D4600E01BB915F8016B0C46284614F80E
:10FE7800013B9E42F6D136B1002105F8011C106005
:10FE8800781EF0BC70473046F9E710680028D6D1D4
:10FE9800F7E716603046F4E72DE9F00F494C82B0D9
:10FEA800D4F800C001900F463C4614F8015B0CEBF7
:10FEB80005004678274606F00800C6B2002EF3D1A2
:10FEC8002D2D61D02B2D04BF244614F8015BB346B9
:10FED800002B41D1302D43D00A239A46BBF1000FA5
:10FEE8000CBF6FF000474FF00047B7FBFAF90AFB69
:10FEF80019700090002080460CE0303DAB421BDDBD
:10FF0800461C05D0C84539D835D00AFB0858012009
:10FF180014F8015B0CEB0506767806F00407FFB2CF
:10FF2800002FEAD116F0030606D0012E14BF57267B
:10FF38003726AD1BAB42E3DC431C2AD0BBF1000FD4
:10FF480001D0C8F10008002A31D0D0B9404611606C
:10FF580002B0BDE8F00F7047102BBED1302DBCD1D8
:10FF68002578782D25D0582D23D043BB4FF0080A8B
:10FF780030255346B2E700988542C6DD4FF0FF3082
:10FF8800C6E74046611EE2E714F8015B4FF0010B3B
:10FF98009EE7BBF1000F01990CBF6FF000404FF0D6
:10FFA800004022230B60002AD2D0611ECFE74046D2
:10FFB800CEE74FF0100A6578534602348EE79A462A
:10FFC80030258BE7A401002070B440F2D054C2F26F
:10FFD800000406460D462068134631462A4670BC82
:10FFE800FFF75ABF024B13B1024800F005B870473B
:08FFF8000000000029E50008EB
:020000040801F1
:100000000146002002460346FEF70EBA8307F0B40D
:10001000C9B200F09680531E002A00F09480027846
:100020008A420BD0421CD8071AD512F0030F104693
:100030001CD01478013B01328C4211D1F0BC7047C6
:10004000002B7CD01278013B8A42F7D014F0030FCA
:10005000204604F1010209D02478013B8C42EDD006
:1000600012F0030F104602F10104E9D1032B3FD92E
:10007000046841EA012545EA054585EA0407A7F138
:10008000013222EA07021E1F041D12F0803FC6F350
:1000900080072DD1032E334629D967B12668204623
:1000A00085EA0602A2F1013626EA0202043412F0C1
:1000B000803F19D01CE020462468061D85EA040212
:1000C000A2F1013424EA020212F0803F10D1346818
:1000D000043B85EA0402A2F1013424EA0202341D41
:1000E00012F0803F304603D1043B032BE3D8204677
:1000F0005D1E23B303788B42A0D0431C0022E80787
:1001000014D51C781846012201338C4296D09542B2
:10011000184603F1010402F102020ED01B788B4253
:100120008CD020462478431C8C4287D095421846B8
:1001300003F1010402F10202F0D100207EE718462B
:100140007CE7134692E7104678E700BF032AF0B435
:1001500031D941EA00039C072ED106680F68151FAC
:10016000031D0C1DBE42C5F3800C24D1032D2A466D
:100170001FD9BCF1000F08D01E682568214618461B
:1001800004340433AE4211D015E0214618461C68F1
:100190000B68051D0E1D9C420DD1314628462E6868
:1001A0000D68043A031D0C1DAE4204D1043A032A23
:1001B000EBD8214618461AB303780C78A3420AD12B
:1001C000551E0022EB0714D510F8013F11F8014F1E
:1001D0000122A3420DD0181B10E010F8013F11F8C6
:1001E000014FA342F7D110F8013F11F8014FA3428C
:1001F000F1D1AA4202F10202EFD10020F0BC704717
:100200001046FBE71E1E64646464646400100048CA
:1002100000110102001000480044010200100048D3
:100220000022110202031048494A4B4C4D444546F6
:1002300047FF1048498A8B8C8D84858687FF000094
:1002400050020108260201085F020108320201087B
:10025000202122232425262748494A4B4C4DFF20A4
:100260002122232425262748498A8B8C8DFF0000D4
:1002700041210008011F00082F1F0008F920000875
:10028000171F0008E12000089D2400084B240008E7
:100290006F240008192600080D240008092400080E
:1002A000002C01400000004800010000001B010A72
:1002B0000044014000040048000100000019000A49
:1002C000004801400004004800020000001A000A33
:1002D000003401400008004840000000002E010AE0
:1002E000003401400008004880000000042E010A8C
:1002F000003401400008004800010000082E010AF7
:100300000004004000040048020000000C1D000A28
:10031000000400400000004810000000041D000A16
:1003200000080040000C004800100000001E000201
:1003300000080040000C004800200000041E0002DD
:1003400000080040000C004800400000081E0002A9
:1003500000080040000C0048008000000C1E000255
:10036000000000400000004802000000041C0002E1
:10037000000000400000004804000000081C0002CB
:10038000002C014000000040000400400008004034
:1003900000340140004401400048014000000400D6
:1003A00008000C00D0073200320032003200320068
:1003B00032003200C800640000004145545231321E
:1003C00033340030313233343536373839414243F3
:1003D0004445464748494A4B4C4D4E4F5051525365
:1003E0005455565758595A00F544000839450008E5
:1003F000154500085145000879450008CD4500081D
:1004000001450008454600080000803FF704353FDD
:10041000F70435BF0000803F0000803FF70435BF80
:10042000F70435BF0000803F0000803FF70435BF70
:10043000F704353F0000803F0000803FF704353F60
:10044000F704353F0000803F0000803F00000000BF
:10045000000080BF000080BF0000803F000080BF20
:1004600000000000000080BF0000803F000000008E
:100470000000803F000080BF0000803F0000803F00
:1004800000000000000080BF0000803F0000803FAF
:10049000000000BF0000803F0000803F000000BF60
:1004A000000080BF0000803F0000803F000080BF50
:1004B0000000003F0000803F0000803F0000003F40
:1004C0000000803F0000803F0000803F0000003FB0
:1004D000000080BF000080BF0000803F000080BFA0
:1004E000000000BF000080BF0000803F000000BF90
:1004F0000000803F000080BF0000803F0000803F80
:100500000000003F000080BF0000803F00000000AE
:100510000000803F0000803F0000803F000080BF5F
:10052000000080BF000000000000803F00000000CD
:100530000000803F000080BF0000803F0000803F3F
:10054000000080BF000000800000803F000000002D
:10055000A8AAAA3F000000000000803F000080BF62
:10056000B0AA2ABF000000000000803F0000803FCA
:10057000B0AA2ABF000000000000803F0000803FBA
:1005800000000000000000000000803F000080BF6D
:1005900000000000000000000000803F000000009C
:1005A00000000000000080BF0000803F000000004D
:1005B000000000000000803F00000000000000007C
:1005C000030100004805010804000000F0070108CD
:1005D000040000005007010802010000780501082E
:1005E000000100000000000006000000D008010823
:1005F0000600000090070108010100000000000053
:1006000004000000900801080600000030080108FE
:1006100008000000D00601080800000008040108D6
:10062000080000008804010801010000000000002B
:1006300000010000000000000001000000000000B8
:10064000040000000805010806000000700601080B
:1006500000010000000000000201000098050108F0
:100660000101000000000000000000000000000088
:100670000000803F000080BF0000803F000080BF7E
:100680000000803F000080BF000080BF0000803F6E
:100690000000803F0000803F0000803F0000803F5E
:1006A0000000803F0000803F000080BF000080BF4E
:1006B0000000803F0000000000000000000000007B
:1006C0000000803F0000000000000000000000006B
:1006D0000000803F000080BF0000803F000080BF1E
:1006E0000000803F000080BF000080BF0000803F0E
:1006F0000000803F0000803F0000803F0000803FFE
:100700000000803F0000803F000080BF000080BFED
:100710000000803F000080BF0000803F0000803F5D
:100720000000803F000080BF000080BF000080BF4D
:100730000000803F0000803F0000803F000080BF3D
:100740000000803F0000803F000080BF0000803F2D
:100750000000803F000080BF0000803F000080BF9D
:100760000000803F000080BF000080BF0000803F8D
:100770000000803F0000803F0000803F0000803F7D
:100780000000803F0000803F000080BF000080BF6D
:100790000000803FD0B35DBF0000003F0000803FFD
:1007A0000000803FD0B35DBF000000BF000080BFED
:1007B0000000803FD0B35D3F0000003F0000803F5D
:1007C0000000803FD0B35D3F000000BF000080BF4D
:1007D0000000803F00000000000080BF0000803F5C
:1007E0000000803F000000000000803F000080BF4C
:1007F0000000803F000000000000803F000080BF3C
:100800000000803F000080BF000000000000803F2B
:100810000000803F0000803F000000000000803F9B
:100820000000803F00000000000080BF000080BF8B
:100830000000803F000000BFD0B35D3F0000803F5C
:100840000000803F000000BFD0B35DBF0000803FCC
:100850000000803F0000003FD0B35D3F000080BF3C
:100860000000803F0000003FD0B35DBF000080BFAC
:100870000000803F000080BF00000000000080BF3B
:100880000000803F0000803F000000000000803F2B
:100890000000803F000000000000803F000080BF9B
:1008A0000000803F000080BF000080BF000000000B
:1008B0000000803F000000000000803F0000803FFB
:1008C0000000803F0000803F000080BF000000006B
:1008D0000000803F00000000A8AAAA3F0000803F5F
:1008E0000000803F000080BFB0AA2ABF000080BF88
:1008F0000000803F0000803FB0AA2ABF000080BFF8
:100900000000803F00000000A8AAAA3F000080BFAE
:100910000000803F000080BFB0AA2ABF0000803FD7
:100920000000803F0000803FB0AA2ABF0000803F47
:1009300024505542582C34312C312C303030332C4B
:10094000303030312C3131353230302C302A314595
:100950000D0A0024504D544B3235312C3131353293
:1009600030302A31460D0A0024505542582C34317B
:100970002C312C303030332C303030312C35373670
:1009800030302C302A32440D0A0024504D544B3262
:1009900035312C35373630302A32430D0A00245099
:1009A0005542582C34312C312C303030332C3030EF
:1009B00030312C33383430302C302A32360D0A00A6
:1009C00024504D544B3235312C33383430302A32A8
:1009D000370D0A0024505542582C34312C312C301C
:1009E0003030332C303030312C31393230302C3003
:1009F0002A32330D0A0024504D544B3235312C31FC
:100A0000393230302A32320D0A00B5620601030055
:100A1000F00500FF19B56206010300F00300FD15A3
:100A2000B56206010300F00100FB11B56206010387
:100A300000F00000FA0FB56206010300F00200FCAE
:100A400013B56206010300F00400FE17B56206014B
:100A500003000102010E47B5620601030001030114
:100A60000F49B56206010300010601124FB5620687
:100A70000103000112011E67B56206160800030794
:100A800003000000000031E5B56206080600C8005A
:100A900001000100DE6A00000000000000C2010049
:100AA00030090108530901080100000000E10000BD
:100AB000680901088A090108020000000096000088
:100AC0009E090108C009010803000000004B000056
:100AD000D4090108F609010804000000802500007F
:100AE0008F1201088F1201084145525431323334BC
:100AF000000027100804230220010000000000006D
:100B00008025000000C2010002000000010000007A
:100B10008025000000C20100030000000200000068
:100B200080250000004B00000500000003000000CD
:100B300080250000004B00000500000002000000BE
:100B40008025000000C2010000000000100000002D
:100B50008025000000C2010001000000200000000C
:100B60008025000000C2010000000000010000001C
:100B70008025000000C20100000000000800000005
:100B80008025000000C201000003000004000000F6
:100B900080250000004B000000000000301B010811
:100BA000371B01083C1B01084D1B0108571B01089E
:100BB000621B01086D1B0108781B0108421A01081D
:100BC000811B01083C1A01088A1B0108941B0108BB
:100BD0009F1B0108A51B0108A81B0108B81B0108E1
:100BE00000000000821A0108861A01088C1A010808
:100BF000921A0108951A01089C1A01089F1A010807
:100C0000A41A0108B01A0108B31A0108B91A010898
:100C1000C01A0108CA1A0108D41A0108DD1A01080D
:100C2000EB1A0108F71A0108FE1A0108041B010853
:100C3000111B01081C1B0108291B010800000000F2
:100C40008C18010890180108BDA10008B718010808
:100C5000BC180108899C0008D0180108D91801089F
:100C6000719C0008F6180108FB18010821A2000871
:100C70002A1901088F120108399C00082F19010850
:100C8000371901084D9B00084B1901085A19010832
:100C90002D9B0008741901088F1201087D98000827
:100CA000791901087D190108859A0008CA180108F8
:100CB00099190108D59E0008AC190108B21901085C
:100CC00015A10008CD190108D5190108C9A000080F
:100CD000E4190108E91901085D9A00086F0F01087D
:100CE000F9190108759F0008271A01081B1A010845
:100CF000A9980008721401088F1201087198000861
:100D00008F1201084E1A0108561A01085E1A0108CE
:100D1000661A01086D1A0108781A01087D1A01087F
:100D2000000000004166726F333220434C49207648
:100D3000657273696F6E20322E32204D61792031D9
:100D4000322032303134202F2031333A32343A30AD
:100D500039202D2028636C65616E666C6967687444
:100D60002900417661696C61626C6520636F6D6D0D
:100D7000616E64733A0D0A0025730925730D0A002C
:100D800053797374656D20557074696D653A2025CB
:100D900064207365636F6E64732C20566F6C74618E
:100DA00067653A202564202A20302E3156202825D8
:100DB00064532062617474657279290D0A0043508E
:100DC000552025644D487A2C2064657465637465EC
:100DD000642073656E736F72733A20002573200070
:100DE00041434348573A202573002E256300437939
:100DF000636C652054696D653A2025642C20493266
:100E000043204572726F72733A2025642C20636F01
:100E10006E6669672073697A653A2025640D0A0059
:100E2000202564202564000D0A5265626F6F746985
:100E30006E672E2E2E00536176696E672E2E2E0061
:100E40004D75737420626520616E79206F726465E0
:100E500072206F662041455452313233340D0A00FE
:100E600043757272656E742061737369676E6D6528
:100E70006E743A20004572726F723A20456E61625C
:100E80006C6520616E6420706C756720696E204708
:100E900050532066697273740D0A00456E61626C6E
:100EA00065642066656174757265733A20004176E9
:100EB00061696C61626C65206665617475726573E9
:100EC0003A2000496E76616C6964206665617475CC
:100ED0007265206E616D652E2E2E0D0A00446973B9
:100EE00061626C65642000456E61626C656420001F
:100EF0000D0A4C656176696E6720434C49206D6F21
:100F000064652E2E2E0D0A00526573657474696E29
:100F10006720746F2064656661756C74732E2E2E65
:100F2000004E4709004F4B0900437573746F6D20E5
:100F30006D697865723A200D0A4D6F746F720954AD
:100F4000687209526F6C6C09506974636809596161
:100F5000770D0A002325643A0900257309005361BF
:100F60006E69747920636865636B3A090072657312
:100F70006574006C6F616400496E76616C69642011
:100F80006D6978657220747970652E2E2E0D0A00B9
:100F90004C6F61646564202573206D69782E2E2E58
:100FA0000D0A0057726F6E67206E756D6265722054
:100FB0006F6620617267756D656E74732C206E6547
:100FC000656473206964782074687220726F6C6C39
:100FD000207069746368207961770D0A004D6F7421
:100FE0006F72206E756D626572206D75737420620C
:100FF00065206265747765656E203120616E6420BE
:1010000025640D0A0043757272656E74206D6978EF
:1010100065723A2025730D0A00417661696C616240
:101020006C65206D69786572733A20004D6978654A
:10103000722073657420746F2025730D0A00437548
:101040007272656E742073657474696E67733A208A
:101050000D0A0025732073657420746F20004552BB
:10106000523A2056616C75652061737369676E6DC5
:10107000656E74206F7574206F662072616E67658F
:101080000D0A004552523A20556E6B6E6F776E20F6
:101090007661726961626C65206E616D650D0A0032
:1010A00043757272656E742070726F66696C653A12
:1010B0002025640D0A0055736167653A0D0A6D6F4E
:1010C000746F7220696E646578205B76616C7565FB
:1010D0005D202D2073686F77205B6F7220736574BD
:1010E0005D206D6F746F722076616C75650D0A00FE
:1010F0004E6F2073756368206D6F746F722C20754E
:1011000073652061206E756D626572205B302C20E6
:1011100025645D0D0A004D6F746F7220256420698F
:1011200073207365742061742025640D0A00496E74
:1011300076616C6964206D6F746F722076616C7576
:10114000652C20313030302E2E323030300D0A00F8
:1011500053657474696E67206D6F746F72202564B7
:1011600020746F2025640D0A006175782025752094
:1011700025750D0A00496E76616C696420466561CB
:101180007475726520696E6465783A206D75737444
:10119000206265203C2025750D0A0043757272653A
:1011A0006E7420436F6E6669673A20436F707920D2
:1011B00065766572797468696E672062656C6F77B1
:1011C00020686572652E2E2E0D0A006D6978657295
:1011D0002025730D0A00636D697820256400636D16
:1011E000697820256420302030203020300D0A001E
:1011F00066656174757265202D25730D0A0066653C
:1012000061747572652025730D0A006D617020256B
:10121000730D0A00736574202573203D20000D0AAC
:10122000456E746572696E6720434C49204D6F644A
:10123000652C20747970652027657869742720747F
:101240006F2072657475726E2C206F72202768652E
:101250006C70270D0A000D0A2320000D1B5B4B004C
:101260001B5B324A1B5B313B3148004552523A20EE
:10127000556E6B6E6F776E20636F6D6D616E642C53
:1012800020747279202768656C7027000820080098
:101290006C6F6F7074696D6500656D665F61766F08
:1012A0006964616E6365006D69647263006D696E87
:1012B000636865636B006D6178636865636B006D7F
:1012C000696E7468726F74746C65006D61787468AF
:1012D000726F74746C65006D696E636F6D6D616EB5
:1012E00064006465616462616E6433645F6C6F772F
:1012F000006465616462616E6433645F6869676835
:10130000006E65757472616C33640064656164625B
:10131000616E6433645F7468726F74746C65006DC1
:101320006F746F725F70776D5F7261746500736563
:1013300072766F5F70776D5F72617465007265744D
:1013400061726465645F61726D00666C6170735F89
:10135000737065656400666978656477696E675F58
:10136000616C74686F6C645F646972007365726944
:10137000616C5F706F72745F315F7363656E617211
:10138000696F0073657269616C5F706F72745F3250
:101390005F7363656E6172696F0073657269616C1A
:1013A0005F706F72745F335F7363656E6172696FD4
:1013B0000073657269616C5F706F72745F345F7324
:1013C00063656E6172696F007265626F6F745F63EF
:1013D0006861726163746572006D73705F626175DC
:1013E000647261746500636C695F626175647261E7
:1013F0007465006770735F706173737468726F7582
:1014000067685F6261756472617465006770735FBD
:1014100070726F7669646572006770735F696E6978
:101420007469616C5F62617564726174655F696E35
:101430006465780073657269616C72785F70726F51
:1014400076696465720074656C656D657472795F48
:1014500070726F76696465720074656C656D657431
:1014600072795F737769746368006672736B795F12
:10147000696E76657273696F6E007662617473630C
:10148000616C6500766261746D617863656C6C7621
:101490006F6C7461676500766261746D696E636517
:1014A0006C6C766F6C7461676500706F7765725FE6
:1014B0006164635F6368616E6E656C00616C69672F
:1014C0006E5F6779726F00616C69676E5F616363FD
:1014D00000616C69676E5F6D616700616C69676E62
:1014E0005F626F6172645F726F6C6C00616C6967E0
:1014F0006E5F626F6172645F706974636800616CD3
:1015000069676E5F626F6172645F796177006D61B8
:10151000785F616E676C655F696E636C696E61743C
:10152000696F6E006779726F5F6C7066006D6F72C5
:101530006F6E5F7468726573686F6C640067797250
:101540006F5F636D70665F666163746F7200677969
:10155000726F5F636D70666D5F666163746F72005A
:10156000616C745F686F6C645F7468726F74746CC4
:10157000655F6E65757472616C00616C745F686F35
:101580006C645F666173745F6368616E6765007445
:1015900068726F74746C655F636F7272656374698F
:1015A0006F6E5F76616C7565007468726F74746CD1
:1015B000655F636F7272656374696F6E5F616E679A
:1015C0006C65007961776465616462616E6400795D
:1015D00061775F636F6E74726F6C5F64697265636D
:1015E00074696F6E007961775F64697265637469AD
:1015F0006F6E007472695F756E61726D65645F73A2
:101600006572766F0072635F726174650072635F0A
:101610006578706F007468725F6D696400746872D9
:101620005F6578706F00726F6C6C5F70697463686F
:101630005F72617465007961775F726174650074CF
:1016400070615F72617465007470615F6272656180
:101650006B706F696E74006661696C736166655F5B
:1016600064656C6179006661696C736166655F6F62
:1016700066665F64656C6179006661696C7361665A
:10168000655F7468726F74746C65006661696C7311
:101690006166655F6465746563745F7468726573C1
:1016A000686F6C6400727373695F6175785F6368FB
:1016B000616E6E656C0067696D62616C5F666C611E
:1016C0006773006163635F6861726477617265006C
:1016D0006163635F6C70665F666163746F72006103
:1016E000636378795F6465616462616E64006163FD
:1016F000637A5F6465616462616E64006163635F05
:10170000756E61726D656463616C006163635F74C3
:1017100072696D5F7069746368006163635F74729E
:10172000696D5F726F6C6C006261726F5F74616291
:101730005F73697A65006261726F5F6E6F6973656E
:101740005F6C7066006261726F5F63665F76656C86
:10175000006261726F5F63665F616C74006D6167E8
:101760005F6465636C696E6174696F6E0067707346
:101770005F706F735F70006770735F706F735F6926
:10178000006770735F706F735F64006770735F7082
:101790006F73725F70006770735F706F73725F69F1
:1017A000006770735F706F73725F64006770735F60
:1017B0006E61765F70006770735F6E61765F69005F
:1017C0006770735F6E61765F64006770735F7770D8
:1017D0005F726164697573006E61765F636F6E74CA
:1017E000726F6C735F68656164696E67006E6176C5
:1017F0005F73706565645F6D696E006E61765F73BF
:10180000706565645F6D6178006E61765F736C65AD
:10181000775F72617465007069645F636F6E747284
:101820006F6C6C657200705F706974636800695FEB
:10183000706974636800705F726F6C6C00695F72CE
:101840006F6C6C00705F79617700695F7961770018
:10185000705F616C7400695F616C7400645F616CDF
:101860007400705F6C6576656C00695F6C657665A9
:101870006C00645F6C6576656C00705F76656C000B
:10188000695F76656C00645F76656C0061757800F1
:10189000666561747572655F6E616D6520617578EE
:1018A000666C6167206F7220626C616E6B20666F80
:1018B00072206C69737400636D6978006465736984
:1018C000676E20637573746F6D206D697865720043
:1018D00064656661756C74730072657365742074F9
:1018E0006F2064656661756C747320616E6420722C
:1018F00065626F6F740064756D70007072696E74EC
:1019000020636F6E666967757261626C65207365CE
:101910007474696E677320696E20612070617374DE
:1019200061626C6520666F726D006578697400662F
:10193000656174757265006C697374206F72202D17
:1019400076616C206F722076616C006770737061D5
:1019500073737468726F756768007061737374680D
:10196000726F7567682067707320746F207365727B
:1019700069616C0068656C70006D6170006D61700C
:1019800070696E67206F66207263206368616E6E97
:10199000656C206F72646572006D69786572206E87
:1019A000616D65206F72206C697374006D6F746F68
:1019B00072006765742F736574206D6F746F722089
:1019C0006F75747075742076616C75650070726FD8
:1019D00066696C6500696E64657820283020746FD4
:1019E0002032290073617665007361766520616E2F
:1019F00064207265626F6F74006E616D653D766123
:101A00006C7565206F7220626C616E6B206F722046
:101A10002A20666F72206C6973740073686F772078
:101A200073797374656D20737461747573004759AD
:101A3000524F00414343004241524F00534F4E41E9
:101A40005200475053004750532B4D4147004144EB
:101A5000584C333435004D505536303530004D4DEF
:101A6000413834357800424D41323830004C534DC6
:101A7000333033444C48430046414B45004E6F6E73
:101A8000650054524900515541445000515541445C
:101A9000580042490047494D42414C0059360048E0
:101AA00045583600464C59494E475F57494E470006
:101AB0005934004845583658004F43544F58380061
:101AC0004F43544F464C415450004F43544F464CA3
:101AD00041545800414952504C414E450048454CF4
:101AE000495F3132305F4343504D0048454C495FB8
:101AF00039305F44454700565441494C340048450D
:101B00005836480050504D5F544F5F534552564F22
:101B1000004455414C434F505445520053494E47A1
:101B20004C45434F5054455200435553544F4D007C
:101B300052585F50504D005642415400494E464C59
:101B4000494748545F4143435F43414C0052585F0B
:101B500053455249414C004D4F544F525F53544FDF
:101B60005000534552564F5F54494C5400534F4612
:101B70005453455249414C004C45445F52494E47ED
:101B8000004641494C534146450054454C454D455E
:101B900054525900504F5745524D455445520056E6
:101BA0004152494F0033440052585F504152414C1A
:101BB0004C454C5F50574D0052585F4D53500000FC
:101BC0002E1A0108331A0108371A01084A1A0108A7
:101BD0003C1A0108421A0108461A010800000000D8
:101BE00090120108020000006019002000000000AF
:101BF000282300009912010800000000621900204B
